:100000000C948A0E0C9490860C94BB0E0C94BB0E30
:100010000C94BB0E0C944A520C946B9E0C94BB0E29
:100020000C94BB0E0C94BB0E0C94BB0E0C94BB0E2C
:100030000C94BB0E0C94BB0E0C94BB0E0C94BB0E1C
:100040000C94BB0E0C9407410C94CE510C94BB0E37
:100050000C94BB0E0C94BB0E0C94BB0E0C948284BF
:100060000C94BB0E0C94C9490C94A0490C94BB0E83
:100070000C94BB0E0C94BB0E0C94BB0E0C94BB0EDC
:100080000C947F920C94BB0E0C94BB0E0C94BB0E84
:100090000C9477490C944E490C94BB0E0C94BB0EF7
:1000A0000C94BB0E0C94BB0E0C94BB0E0C94BB0EAC
:1000B0000C94BB0E0C943E880C94BB0E0C94BB0E9F
:1000C0000C94BB0E0C94BB0E0C94BB0E0C942549E7
:1000D0000C94FC480C94BB0E0C94D3480C94AA4886
:1000E0000C94BB0E8C1B8F1B961B991B9C1B9F1B80
:1000F000A61BAD1BB01BB71BBE1BC51B69219721DF
:10010000CE210522E0221723452373233A243A24E3
:100110003A243A243A243A243A243A243A243A24EF
:100120003A243A243A243A243A243A243A243A24DF
:100130003A243A243A243A243A243A243A243A24CF
:100140003A243A243A243C227322AB22A123CF231F
:10015000072438263E2644264A26502656265C2664
:10016000622668266E2674267A268C269226982683
:10017000B026B626BC26C226C826CE26D426DA2627
:10018000E026E626EC26F226F826FE260A27162783
:100190001C2722272827402746274C275227582745
:1001A0005E274E2854285A286C28722878288A28D6
:1001B000902896289C28A228A828D228D828022946
:1001C00008290E2914292C29322938293E29D32916
:1001D000D329D329D329D329D329D329D3295429BE
:1001E00058295C29622966296A296E29722976298B
:1001F0007A2980299E29A429AA292E2764276A27DB
:10020000702776277C2782271A2920292629442926
:100210004A295029B029B629BC29AE28B4288827F4
:100220008E2794279A27A027A62760287E281027A4
:100230008026862634273A27C229C829CE290427B2
:10024000DE28E428EA28F028F628FC28AC27B22784
:10025000B827BE27C427CA27D027D627DC27E227FE
:10026000E827EE27F427FA27002806280C2812286A
:100270001E2824282A28302836283C2842284828A6
:1002800092298C2986299829662884289E26A426C6
:10029000AA26BA281828C028C628CC28AE308B3009
:1002A0006430CB302231EA3019310831D331B631E4
:1002B0008F312332F031F0311232FB31B938B93895
:1002C000C838B938D538EE380939243976457945F2
:1002D00068456C457245B0457D45814587458B45F0
:1002E0008F45954599459D45B045A345A745AB45E7
:1002F000334B384B3D4B474B514BCA4B5B4B634BDE
:100300006B4B754B7F4B894B984BA24BCA4BAC4BFD
:10031000B64BC04B9C62A062A462A862AC62B062A1
:10032000B462B862BC62C062C462F062F462FB6232
:100330000863156328633B6354636D638B63A16338
:10034000146848687D689D68D2683A694A69746A29
:10035000BE69C869FC69316A3F6A746A06696D885A
:1003600076887E889288A488B688C188549A6B9AC9
:10037000829A999AB09ADE9AF59A0C9B239B429B9B
:100380005A9B719B909BA69BC79A05A84CCDB2D453
:100390004EB93836A9020C50B9918688083CA6AAF5
:1003A000AA2ABE000000803F3400330032004E6FA6
:1003B0006E650053746F70706564004E657574727D
:1003C000616C205475726E004D6F76696E672052B5
:1003D000657665727365004D6F76696E6720466F4E
:1003E0007277617264004272616B696E670054419A
:1003F0004E4B20524553544F52454400250048650A
:10040000616C7468204C6576656C3A2000564548EE
:1004100049434C452052455041495220434F4D508D
:100420004C4554450054414E4B2044455354524F83
:100430005945440025004865616C7468204C657618
:10044000656C3A2000290056454849434C452052E6
:1004500045504149522053544152544544202800AC
:10046000524550414952204F5045524154494F4EF8
:100470002043414E43454C4C45440029004D4143E7
:1004800048494E452047554E2048495421202800D0
:10049000524550414952204F5045524154494F4EC8
:1004A0002043414E43454C4C454400290043414EB6
:1004B0004E4F4E20484954212028005475727265D1
:1004C0007420726F746174696F6E206973206E6F2F
:1004D00074206F66207479706520536572766F2E74
:1004E000204E6F20736574757020617661696C6150
:1004F000626C652E004E6F207374656572696E675D
:1005000020736572766F2061737369676E65642C02
:100510002072652D636865636B2076656869636C1E
:100520006520747970652E0054757272657420654B
:100530006C65766174696F6E206973206E6F7420CC
:100540006F66207479706520536572766F2E204E29
:100550006F20736574757020617661696C61626C7F
:10056000652E00546F70204C65667400546F7020C7
:1005700043656E74657200546F70205269676874C9
:10058000004D6964646C65204C656674004D696457
:10059000646C652043656E746572004D6964646CBB
:1005A0006520526967687400426F74746F6D204CE7
:1005B00065667400426F74746F6D2043656E746578
:1005C0007200426F74746F6D2052696768740046E0
:1005D00049524D574152452056455253494F4E3A84
:1005E00020006942757300534275730050504D00EE
:1005F0004E6F6E6520446574656374656400417A6E
:10060000696D7574682020202000456C65766174E2
:10061000696F6E2020005475726E202020202020EB
:1006200020005468726F74746C652020200053742D
:1006300069636B202020202020204D696E2020201F
:100640002043656E7465722020204D617820202043
:10065000204465616462616E642020526576657233
:1006600073656400524144494F20494E464F202D46
:1006700020004E4F542044455445435445440049BE
:10068000474E4F52454400416E616C6F67004469AC
:10069000676974616C00417578204368616E2E2033
:1006A00020204D696E20202020204D6178202020C0
:1006B000202054797065004368616E6E656C73200C
:1006C0007574696C697A65643A20004368616E6E7E
:1006D000656C732064657465637465643A200020FA
:1006E0002844697361626C656429002028456E6145
:1006F000626C656429004D656368616E6963616C55
:10070000207265636F696C00416972736F66740073
:100710004D656368616E6963616C204261727265E8
:100720006C3A200020284D31290020284D32290024
:10073000202842290042617272656C20456C657602
:100740006174696F6E3A20200020284D3029002006
:10075000284D312900202841290054757272657492
:1007600020526F746174696F6E3A2020200020411E
:100770006D70732900202843757272656E74204C69
:10078000696D69743A20004472697665204D6F7412
:100790006F72733A202020202020004D4F544F527A
:1007A00020545950455300496E646570656E646508
:1007B0006E7420547265616420436F6E74726F6C46
:1007C0000054616E6B202854616D69796120444D3D
:1007D00044290054616E6B2028444B4C4D204765E2
:1007E0006172626F7829004361720048616C6674BF
:1007F0007261636B0054616E6B00554E4B4E4F57E8
:100800004E00596573004E6F002900252C20446569
:1008100063656C65726174696F6E20666163746F85
:1008200072200020284B69636B6261636B207370D8
:100830006565642000547261636B205265636F6963
:100840006C20456E61626C65643A202020004E2F5A
:100850004120666F722076656869636C65207479E3
:100860007065005475726E204D6F64653A202020CB
:100870002020202020202020202020004E2F41203A
:10088000666F722076656869636C6520747970653F
:1008900000596573202854616D697961290025002C
:1008A000202D20004E65757472616C205475726E37
:1008B00020416C6C6F7765643A20202000207365BE
:1008C00063005472616E736D697373696F6E204457
:1008D000656C61793A202020202000207365630038
:1008E000456E67696E652050617573652054696D4A
:1008F000653A202020202020002073656300536883
:100900006966742054696D653A20202020202020DB
:10091000202020202020004175746F6D6174696370
:10092000004D616E75616C005472616E736D697318
:1009300073696F6E20547970653A20202020202042
:10094000002500596573202D20005265766572736D
:1009500065205370656564204C696D697465643AFF
:100960002020002500596573202D2000466F7277E6
:10097000617264205370656564204C696D697465AB
:10098000643A202000206D73290025207468726F5E
:1009900074746C6520666F7220002028004D6F749F
:1009A0006F72204E7564676520456E61626C656488
:1009B0003A202020200029004E6F6E65004E6F6E99
:1009C00065002C205072657365743A200029002060
:1009D0002841646A757374656420746F2000202850
:1009E0004C6576656C3A2000446563656C20526105
:1009F0006D7020456E61626C65643A202020202075
:100A00000029004E6F6E65004E6F6E65002C205001
:100A100072657365743A20002900202841646A7564
:100A20007374656420746F200020284C6576656CB3
:100A30003A2000416363656C2052616D7020456E01
:100A400061626C65643A2020202020004163746953
:100A500076652044726976696E672050726F6669A8
:100A60006C653A200056656869636C65205479703E
:100A7000653A2020202020202020202020004452E1
:100A80004956452053455454494E475300207365F9
:100A900063005265636F696C2064656C61793A200C
:100AA0002020202020202020202020202020202046
:100AB0002020002500596573202D200042617272AC
:100AC000656C20456C65766174696F6E2053706546
:100AD0006564204C696D697465643A20002500598D
:100AE0006573202D200054757272657420526F74E6
:100AF0006174696F6E205370656564204C696D691F
:100B00007465643A20200054555252455420534590
:100B10005454494E475300556E6B6E6F776E0045C7
:100B200078706572696D656E74616C005365706193
:100B300072617465204865617420262046616E00EC
:100B4000436F6D62696E656420486561742026207C
:100B500046616E00250044697361626C65640053F0
:100B60006D6F6B65207768656E2064657374726F56
:100B70007965643A200046616E206D61782073705B
:100B80006565643A20202020202020200046616EE8
:100B900020666173742069646C6520737065656498
:100BA0003A20200046616E2069646C652073706590
:100BB00065643A20202020202020002028637572C0
:100BC00072656E746C792064697361626C65642906
:100BD00000207365636F6E6473004E2F4100507286
:100BE000652D686561742064656C61793A20202008
:100BF0002020202000536D6F6B6572205479706542
:100C00003A2020202020202020202000536D6F6BD0
:100C10006572206F757470757420636F6E74726F77
:100C20006C6C6564206D616E75616C6C7900534D00
:100C30004F4B455200556E6B6E6F776E0048656185
:100C40007679004D656469756D004C69676874005C
:100C5000437573746F6D00556E6B6E6F776E004EDB
:100C60006F6E65004F70656E2050616E7A65720020
:100C700054616D6979612053706563002073656309
:100C8000207265636F766572792900207365632031
:100C900072656C6F61642C2000204D472068697478
:100CA000732C20002063616E6E6F6E206869747310
:100CB0002C2000280057656967687420436C6173B5
:100CC000733A20202020200044616D616765205028
:100CD000726F66696C653A20202000596573202880
:100CE00000416363657074204D472044616D616706
:100CF000653A200059657320280053656E64204DC5
:100D00004720495220436F64653A2020004E2F410E
:100D10000052657061697265642062793A20202012
:100D2000202020004E2F41004869742050726F74BB
:100D30006F636F6C20323A20202000290020285455
:100D400065616D2000466972652050726F746F6333
:100D50006F6C3A2020202000466972652050726F27
:100D6000746F636F6C3A2020202000497320526515
:100D7000706169722054616E6B3F202020004952DF
:100D800020262054616E6B20426174746C696E671A
:100D90002044697361626C656400424154544C455F
:100DA00020494E464F00554E4B4E4F574E00426520
:100DB0006E6564696E6920544253204D6963726F99
:100DC0000042656965722055534D2D52432D320006
:100DD00054616967656E20536F756E64204361725C
:100DE00064004F70656E2050616E7A657220536F9B
:100DF000756E6420436172640042656E6564696E5D
:100E00006920544253204D696E6900536F756E64BA
:100E100020636172643A2000534F554E4420434191
:100E2000524400556E6B6E6F776E00426172726550
:100E30006C20456C65766174696F6E20436F6D6DD3
:100E4000616E640054757272657420526F746174BF
:100E5000696F6E20436F6D6D616E640053746565DC
:100E600072696E6720436F6D6D616E6400566568D0
:100E700069636C6520537065656400456E67696ED3
:100E800065205370656564005468726F74746C6596
:100E900020436F6D6D616E640053706565642064FE
:100EA00065637265617365732062656C6F7720009E
:100EB000537065656420696E637265617365732044
:100EC00061626F766520005475726E2053746F7086
:100ED000706564004C656674205475726E2053749E
:100EE0006172746564005269676874205475726E2B
:100EF00020537461727465640056656869636C653B
:100F00002053746F70706564004D6F76696E672052
:100F100052657665727365004D6F76696E6720461F
:100F20006F727761726400456E67696E65205374F5
:100F30006F7000456E67696E65205374617274004E
:100F400043616E6E6F6E2052656C6F616465640004
:100F500056656869636C652044657374726F796562
:100F6000640043616E6E6F6E204869740042726166
:100F70006B6573204170706C6965640056617269BD
:100F800061626C6500290020286F662000506F7335
:100F90002000417578204368616E6E656C200056B4
:100FA00061726961626C65004F6E004F6666004257
:100FB00000410045787465726E616C20496E7075F1
:100FC000742000070809090B0C0C0B0C0C547572EB
:100FD00072657420537469636B202D200046756E12
:100FE0006374696F6E202300202D3E2000207365FE
:100FF0006300547572726574206D6F76656D656EF1
:10100000742064656C61793A2020004E6F6E650033
:101010005965730054757272657420737469636BDB
:101020002066756E6374696F6E733A200046554E84
:101030004354494F4E205452494747455253007636
:10104000206375746F666629002028004C56432083
:10105000456E61626C65643A202020202020007675
:1010600000566F6C746167653A2020202020202094
:1010700020202000596573004E6F00426174746532
:1010800072792044657465637465643A2000424156
:1010900054544552590053657269616C2033205491
:1010A0007820426175643A202000417578205365AC
:1010B0007269616C20426175643A202020004D6F96
:1010C000746F722053657269616C20426175643A75
:1010D00020005553422053657269616C204261754E
:1010E000643A202020004241554420524154455347
:1010F00000212000464143544F5259205245534548
:101100005421200000002100240027002A002D0087
:101110003000330001010000040107010A01000052
:101120002200250028002B002E003100340002018F
:101130000000050108010B0100002000230026002B
:1011400029002C002F0032000001000003010601DD
:10115000090105050505070508080808020202023D
:101160000A0A080804040404010101010101010143
:101170000303030303030303040707070C0C0C0C0E
:101180000C0C0C0C020202020606060606060606F7
:101190000B0B0B0B0B0B0B0B010210202008081084
:1011A00020401020408002010201080402010102D7
:1011B00004081020408080402010080402018004B0
:1011C000020180402010080402010804020101020B
:1011D0000408102040800102040810204080000014
:1011E0000A0B02090C0D0E080703040100000000A1
:1011F00000000000000000000000000000000000EF
:1012000000000000000000000000121110000000AB
:1012100000000000000000000000000000000000CE
:1012200000000000556E6B6E6F776E004465746150
:10123000636865642F4E41005265636F696C20538B
:101240006572766F0050616E20536572766F005341
:101250006572766F2F455343004F6E626F61726403
:10126000204D6F746F7220447269766572004F7002
:10127000656E2050616E7A65722053636F757420BD
:1012800053657269616C2045534300536162657216
:10129000746F6F74682053657269616C00506F6C75
:1012A0006F6C752053657269616C00536572766F5F
:1012B000203100536572766F203200536572766F6D
:1012C000203300536572766F203400536572766F59
:1012D000203500536572766F203600536572766F45
:1012E000203700536572766F203800494F20506FC9
:1012F00072742042202D2050756C73656400494F34
:1013000020506F72742042202D205374617274201B
:10131000426C696E6B696E67005573657220467525
:101320006E6374696F6E2031005573657220467567
:101330006E6374696F6E203200466F7277617264FB
:101340002047656172004E65757472616C20476557
:10135000617200526576657273652047656172003F
:1013600053657420416363656C2052616D70204C3D
:101370006576656C3A200053657420446563656C3E
:101380002052616D70204C6576656C3A2000416E8C
:10139000616C6F6720557365722046756E63746962
:1013A0006F6E2031202D2000416E616C6F672055DB
:1013B0007365722046756E6374696F6E2032202DDE
:1013C00020002D00202D20002000545255450046BD
:1013D000414C534500250057616974696E6720666A
:1013E0006F7220726164696F2E2E2E200020287784
:1013F0006974682049522900466972652043616E0C
:101400006E6F6E0046697265205265706169722068
:101410005369676E616C00416972736F6674202D49
:10142000204D616E75616C2054726967676572004A
:101430004D656368616E6963616C205265636F69B5
:101440006C202D204D616E75616C20547269676748
:10145000657200536572766F205265636F696C2008
:101460002D204D616E75616C2054726967676572DD
:10147000004869676820496E74656E7369747920E5
:10148000466C61736820556E6974202D204D616E25
:1014900075616C2054726967676572004D4720530F
:1014A00074617274004D472053746F70004952206C
:1014B0004E4F5420656E61626C6564202D206E6F06
:1014C0002049522070726F746F636F6C7320736564
:1014D0006C65637465642E00556E61626C65207482
:1014E0006F20656E61626C6520495200495220652B
:1014F0006E61626C65640049522064697361626C5C
:10150000656400417578204F757470757420466C61
:10151000617368656400417578204F7574707574E7
:1015200020496E766572736520466C6173686564E8
:101530000053746F7020417578204F757470757406
:1015400020426C696E6B696E670053746F70205235
:1015500065766F6C76696E6720417578204C696797
:1015600068740053746F7020416C6C205573657201
:1015700020536F756E647300494F20506F72742052
:1015800041202D2050756C73656400494F20506FC9
:1015900072742041202D20537461727420426C6952
:1015A0006E6B696E6700416972736F6674202D20DF
:1015B00044697361626C6564004D656368616E695E
:1015C00063616C205265636F696C202D20446973E0
:1015D00061626C656400436F6D6D73206368616E5A
:1015E00067656420746F2055534200436F6D6D73BF
:1015F000206368616E67656420746F20536572694B
:10160000616C20310044726976696E672050726F98
:1016100066696C652073657420746F202300250053
:101620005370656564207265647563656420746FCA
:101630002000537065656420726573746F72656411
:10164000005475726E20456E67696E65204F6E009E
:10165000207365636F6E64732061676F202D207344
:101660006D6F6B6572207072656865617420736B55
:10167000697070656400456E67696E65206C6173A2
:10168000742073746F707065642000207365636FDD
:101690006E647300536D6F6B6572207072652D6898
:1016A0006561742073746172746564202D20656EA9
:1016B00067696E652077696C6C207475726E206F37
:1016C0006E20696E20004D616E75616C20747261D0
:1016D0006E736D697373696F6E202D207075742041
:1016E000696E206E65757472616C20676561722029
:1016F0006265666F7265207374617274696E6720CB
:10170000656E67696E652100456E67696E6520418B
:1017100075746F2053687574646F776E00456E67DB
:10172000616765205472616E736D697373696F6E62
:1017300000446973656E67616765205472616E73FA
:101740006D697373696F6E00536574205475726EA2
:10175000204D6F64653A20310053657420547572D2
:101760006E204D6F64653A203200536574205475C5
:10177000726E204D6F64653A203300456E61626C75
:1017800065204E65757472616C205475726E7300BD
:1017900044697361626C65204E65757472616C207A
:1017A0005475726E7300401F7017D007A00FA00F02
:1017B000DC05D007C40910278813983A102758026F
:1017C0006C0258026C0258026C0258026C025802F9
:1017D0006C0258026C0258026C0258026C025802E9
:1017E000B0366C023A026C023A026C023A026C02A7
:1017F000B036384A5C121C255C125C121C255C1247
:10180000BC7FC7F2C07887A5B7C5A00F8813B80BF7
:10181000401FB80BB80B7017401F494F20506F7214
:10182000742041204F7574707574202D204F6E0008
:10183000494F20506F72742041204F757470757439
:10184000202D204F666600494F20506F7274204251
:10185000204F7574707574202D204F6E00494F20F5
:10186000506F72742042204F7574707574202D2053
:101870004F6666004C56432045786974202D2056EB
:101880006F6C7461676520526573746F7265640074
:101890007629004C5643207468726573686F6C64D7
:1018A0002072656163686564212028004C6967685F
:1018B000742031204F6E004C696768742031204FCE
:1018C0006666004C696768742032204F6E004C6970
:1018D0006768742032204F666600326E64204D4780
:1018E0002053746F7000326E64204D472053746132
:1018F00072740052756E6E696E67204C6967687409
:1019000073204F6E0052756E6E696E67204C69676A
:10191000687473204F666600417578204F75747047
:101920007574204F6E00417578204F757470757412
:10193000204F66660053746F70205265766F6C7628
:10194000696E6720417578204C696768740053742C
:101950006F7020417578204F757470757420426CDB
:10196000696E6B696E6700417578204F757470758C
:1019700074205072657365742044696D00537461FE
:10198000727420417578204F757470757420426CA4
:10199000696E6B696E6700526164696F20526561A0
:1019A0006479202D200052657665727365643A2053
:1019B00020004D61782050756C73653A20004D69A8
:1019C0006E2050756C73653A2000456E6420566138
:1019D0006C75657300456E64205265636F696C2099
:1019E000536572766F20536574757000456E642080
:1019F000526F746174696F6E20536572766F2053F5
:101A00006574757000456E64205374656572696E07
:101A10006720536572766F20536574757000456E4C
:101A200064205374656572696E6720536572766FC2
:101A300020536574757000456E6420456C65766151
:101A400074696F6E20536572766F2053657475707C
:101A500000536572766F20756E2D726576657273B0
:101A6000656400536572766F207265766572736582
:101A7000640052657665727365643A2020004D619A
:101A8000782050756C73653A20004D696E20507552
:101A90006C73653A200053746172742056616C75E2
:101AA000657300494E56414C494420534552564FA8
:101AB0002E204E4F2053455455502E0053657475BB
:101AC00070205265636F696C20536572766F0053A6
:101AD000657475702054757272657420526F7461EC
:101AE00074696F6E2050616E20536572766F00537B
:101AF00065747570205374656572696E67205365EF
:101B000072766F20284F75747075742032290053D7
:101B100065747570205374656572696E67205365CE
:101B200072766F20284F75747075742034290053B5
:101B3000657475702054757272657420456C657695
:101B40006174696F6E20536572766F0048656174C9
:101B500020416D743A2000486561743A2000536159
:101B60006D652061732066616E005374617274202C
:101B70005265766F6C76696E6720417578204C6986
:101B800067687400536D6F6B657220656E61626C7F
:101B9000656400536D6F6B65722064697361626C7C
:101BA00065640053657420766F6C756D653A20002E
:101BB000202D2053746172742052657065617469C0
:101BC0006E6700202D2053746F700055736572206E
:101BD000536F756E64200041202D200042202D207F
:101BE00000536F756E642042616E6B2000506C6113
:101BF000792F53746F7000506C61792052616E645C
:101C00006F6D00506C61792050726576696F7573E5
:101C100000506C6179204E65787400546169676585
:101C20006E2056322F563300536F6E790052435454
:101C300041204D616368696E652047756E00436C95
:101C400061726B204D616368696E652047756E0037
:101C500052435441205265706169720049425520D7
:101C600052657061697200436C61726B20526570DD
:101C7000616972004F70656E50616E7A65720056D0
:101C80007354616E6B00464F560054616967656E10
:101C90002056310048656E67204C6F6E67005461B6
:101CA0006D69796120312F33350054616D69796137
:101CB00020322D53686F740054616D69796100554D
:101CC0006E6B6E6F776E003A200042697420004799
:101CD00061703A2000416972736F6674202D20454F
:101CE0006E61626C6564004D656368616E69636115
:101CF0006C205265636F696C202D20456E61626CAB
:101D0000656400524144494F204641494C53414685
:101D100045000BB511241FBECFEFD1E2DEBFCDBF12
:101D200000E00CBF17E0A0E0B2E0E8EBF0EB01E070
:101D30000BBF02C007900D92AA30B107D9F724E17A
:101D4000AAE0B7E001C01D92A83CB207E1F71EE08F
:101D5000CAE8DEE000E006C021970109802FFE01FD
:101D60000E9494C4C938D10780E00807A9F70E94EF
:101D700071A20C94E7C60C9400002F923F924F92F0
:101D80005F926F927F928F929F92AF92BF92CF920B
:101D9000DF92EF92FF920F931F93CF93DF93CDB714
:101DA000DEB7E6970FB6F894DEBF0FBECDBF8091C9
:101DB0008513909186130E947E470E9402576FEC14
:101DC00075E080918513909186130E9476486BE6AA
:101DD00076E0CE0101960E94FE4680918513909197
:101DE0008613DC01ED91FC914D815E8169817A81E0
:101DF0000280F381E02D199563E776E080918513E9
:101E0000909186130E9475482AE041EE51E060E00F
:101E100070E080918513909186130E9436476DEB98
:101E200076E080918513909186130E948147CE01C0
:101E300001960E94A2460E94AD97809185139091D1
:101E40008613DC01ED91FC910680F781E02D199558
:101E500080918513909186130E947E470E940257BD
:101E600064E676E080918513909186130E9476480F
:101E7000E091EE0BE4300CF0E0E080EF95E09A8327
:101E800089838CEE95E09C838B8387EE95E09E831F
:101E90008D8382EE95E098878F83EE0FFF0B21E014
:101EA00030E02C0F3D1FE20FF31F608171818091A4
:101EB0008513909186130E949A480E9402576EE201
:101EC00076E080918513909186130E949A480E9433
:101ED000025762E276E080918513909186130E940A
:101EE0007648E091BC10F091BD1081819281883ECE
:101EF000934014F40E94F256E091BC10F091BD1092
:101F00006181728180918513909186130E944A6C41
:101F100084E00E94CF94E091BC10F091BD106581E7
:101F2000768180918513909186130E944A6C85E09A
:101F30000E94CF94E091BC10F091BD106381748138
:101F400080918513909186130E944A6C84E00E94D0
:101F5000CF94E091BC10F091BD1067818091851302
:101F6000909186130E949A6A88E00E94CF94E09133
:101F7000BC10F091BD1080850E94D85666E176E0D5
:101F800080918513909186130E947648E091C61047
:101F9000F091C71081819281883E934014F40E9491
:101FA000F256E091C610F091C71061817281809164
:101FB0008513909186130E944A6C84E00E94CF940E
:101FC000E091C610F091C7106581768180918513EC
:101FD000909186130E944A6C85E00E94CF94E09114
:101FE000C610F091C7106381748180918513909120
:101FF00086130E944A6C84E00E94CF94E091C61040
:10200000F091C710678180918513909186130E948B
:102010009A6A88E00E94CF94E091C610F091C710B0
:1020200080850E94D8566AE076E080918513909171
:1020300086130E947648E091D010F091D1108181F2
:102040009281883E934014F40E94F256E091D010A1
:10205000F091D110618172818091851390918613E6
:102060000E944A6C84E00E94CF94E091D010F091DD
:10207000D1106581768180918513909186130E949D
:102080004A6C85E00E94CF94E091D010F091D1107D
:102090006381748180918513909186130E944A6CAC
:1020A00084E00E94CF94E091D010F091D11067812C
:1020B00080918513909186130E949A6A88E00E940D
:1020C000CF94E091D010F091D11080850E94D85625
:1020D0006EEF75E080918513909186130E9476488B
:1020E000E091DA10F091DB1081819281883E93407B
:1020F00014F40E94F256E091DA10F091DB10618145
:10210000728180918513909186130E944A6C84E0BD
:102110000E94CF94E091DA10F091DB106581768116
:1021200080918513909186130E944A6C85E00E94ED
:10213000CF94E091DA10F091DB106381748180918B
:102140008513909186130E944A6C84E00E94CF947C
:10215000E091DA10F091DB10678180918513909106
:1021600086130E949A6A88E00E94CF94E091DA1068
:10217000F091DB1080850E94D85680918513909154
:1021800086130E947E470E94EBA0C82E66E976E087
:1021900080918513909186130E949A480E9402575D
:1021A00000E610E1E12CF12CD12C5701BFEFAB1A66
:1021B000BB0AB50180918513909186130E944A6CE9
:1021C000E9E0EE16F10410F48BE001C08AE00E9411
:1021D000CF94D8012C91809185139091861322235E
:1021E000C9F11596ED91FC911697618172810E945B
:1021F0004A6CD8011596ED91FC91169781819281D8
:10220000883E934014F40E94F25684E00E94CF94DA
:10221000D8011596ED91FC91169763817481809198
:102220008513909186130E944A6C84E00E94CF949B
:10223000D8011596ED91FC91169727818091851311
:1022400090918613222319F06EE876E00BC067E8C0
:1022500076E008C0EC14FD041CF46FE776E002C0E1
:1022600062E776E00E949A48095F1F4F7501BCE063
:10227000AB16B10409F099CF0E9402576BEC76E0DF
:1022800080918513909186130E9476480E94EBA05E
:10229000682F80918513909186130E94836A67EB63
:1022A00076E080918513909186130E947648609124
:1022B000EB0B7091EC0B80918513909186130E942B
:1022C000806C0E94AD978091851390918613DC01FC
:1022D000ED91FC910680F781E02D19958091851391
:1022E000909186130E947E470E9402576BE977E027
:1022F00080918513909186130E949A480E940257FC
:1023000067E877E080918513909186130E94764864
:102310008091BB120E94C14DBC01809185139091A8
:1023200086130E9476488091BB128A30C1F465E71B
:1023300077E080918513909186130E947648609192
:10234000791380918513909186130E949A6A6EE6A4
:1023500077E080918513909186130E947648809152
:102360008513909186130E947E476AE577E08091FD
:102370008513909186130E9476488091BC120E942A
:10238000C14DBC0180918513909186130E947648BF
:102390002091BC1280918513909186132B303CF4D0
:1023A000293054F4283069F469E477E007C02B3011
:1023B00041F465E577E002C06FE477E00E949A4857
:1023C00002C00E947E4765E377E08091851390917B
:1023D00086130E9476488091BD120E94C14DBC01B7
:1023E00080918513909186130E9476482091BD12AA
:1023F00080918513909186132B303CF4293054F44E
:10240000283069F464E277E007C02B3041F460E3E0
:1024100077E002C06AE277E00E949A4802C00E9418
:102420007E4760E177E080918513909186130E944A
:1024300076482091CF1280918513909186132223A4
:1024400019F068E077E002C066EF76E00E94764817
:102450002091DB138091851390918613222319F02C
:102460006BEE76E002C06FED76E00E9476488091D8
:102470008513909186130E947E470E94AD978091AC
:10248000851390918613DC01ED91FC910680F78114
:10249000E02D199580910002823011F00C94C01C3F
:1024A000F090F6120091F91210E08091851390914E
:1024B00086130E947E470E9402576EE77AE0809161
:1024C0008513909186130E949A480E94025765E6F0
:1024D0007AE080918513909186130E947648E0916E
:1024E0000613E7300CF0E0E08AEF97E09A838983E7
:1024F00085EF97E09C838B838BEE97E09E838D83A3
:1025000087EE97E098878F8383ED97E09A87898796
:1025100081EC97E09C878B8787EA97E09E878D8781
:10252000EE0FFF0B21E030E02C0F3D1FE20FF31FF9
:102530006081718180918513909186130E949A48E1
:102540006CE47AE080918513909186130E9476481E
:102550006091000280918513909186130E94836A96
:1025600063E37AE080918513909186130E94764808
:102570008F2D0E94C356FF2009F44BC069E27AE018
:1025800080918513909186130E94764880918513DF
:1025900090918613112339F06091F1120E949A6A8A
:1025A0009091F11206C06091F7120E949A6A909180
:1025B000F7128091931498130C94C71C6DE07AE085
:1025C00080918513909186130E947648809185139F
:1025D00090918613112339F06091F21261110CC0B1
:1025E00068E07AE006C06091F812611105C063E00E
:1025F0007AE00E94764805C0062E000C770B0E94F8
:102600004A6C61E07AE080918513909186130E9474
:10261000764880918513909186130E947E4768EEDC
:1026200079E080918513909186130E947648802FDF
:102630000E94C356002309F44BC06EED79E08091EF
:102640008513909186130E9476488091851390910E
:102650008613112339F06091F4120E949A6A9091C6
:10266000F41206C06091FA120E949A6A9091FA12CE
:102670008091951498130C94E11C62EC79E08091A0
:102680008513909186130E947648809185139091CE
:102690008613112339F06091F51261110CC06DEBB6
:1026A00079E006C06091FB12611105C068EB79E02A
:1026B0000E94764805C0062E000C770B0E944A6CDB
:1026C00066EB79E080918513909186130E9476489D
:1026D00080918513909186130E947E476DE979E081
:1026E00080918513909186130E94764880910F13F4
:1026F000811103C00E94D15635C062E078E080911C
:102700008513909186130E9476486AE979E080915A
:102710008513909186130E94764860910F138091E3
:102720008513909186130E949A6A6AE879E08091F5
:102730008513909186130E94764840911013509112
:10274000111360E070E02AE0809185139091861368
:102750000E94364765E879E0809185139091861351
:102760000E949A486CE679E08091851390918613D7
:102770000E947648809107138436C8F465E679E0B4
:1027800080918513909186130E947648609107137B
:1027900080918513909186130E949A6A63E679E08E
:1027A00080918513909186130E949A4803C080E01F
:1027B0000E94D1566AE479E0809185139091861346
:1027C0000E947648809108138436C8F463E479E067
:1027D00080918513909186130E947648609108132A
:1027E00080918513909186130E949A6A61E479E042
:1027F00080918513909186130E949A4803C080E0CF
:102800000E94D15668E279E08091851390918613F9
:102810000E94764820919F0780918513909186139E
:10282000222319F061E279E002C067E179E00E94B9
:102830009A486EEF78E080918513909186130E94FC
:1028400076486091FD127091FE12072E000C880BE5
:10285000990B0E9435C120E030E04AE754E40E9421
:102860003AC3AB01BC0121E080918513909186139E
:102870000E94984769EF78E08091851390918613C4
:102880000E949A4860EE78E08091851390918613BB
:102890000E9476486091FF1270910013072E000C81
:1028A000880B990B0E9435C120E030E04AE754E4E0
:1028B0000E943AC3AB01BC0121E080918513909145
:1028C00086130E9498476BED78E080918513909174
:1028D00086130E949A4862EC78E08091851390916B
:1028E00086130E9476486091011370910213072E9F
:1028F000000C880B990B0E9435C120E030E04AE7BC
:1029000054E40E943AC3AB01BC0121E080918513DD
:10291000909186130E9498476DEB78E08091851323
:10292000909186130E949A4864EA78E0809185131A
:10293000909186130E94764890910613913011F081
:102940009430F9F4809103130E94C35680910313CD
:10295000882329F160EA78E08091851390918613AD
:102960000E9476486091041380918513909186139C
:102970000E949A6A6EE978E080918513909186139F
:102980000CC02091851330918613953019F461E9BC
:1029900078E002C06CE778E0C9010E947648809137
:1029A0008513909186130E947E4763E678E08091BC
:1029B0008513909186130E947648909106132FEF0D
:1029C000290F8091851390918613223028F460910D
:1029D0000A070E94836A04C06EE478E00E949A4865
:1029E00065E378E080918513909186130E94764884
:1029F000809113130E94C35680911313882341F1D1
:102A000063E278E080918513909186130E94764866
:102A10006091141380918513909186130E949A6A95
:102A20006BE078E080918513909186130E94764840
:102A30006091151380918513909186130E949A6A74
:102A400069E078E080918513909186130E94764822
:102A500080918513909186130E947E470E94AD97C6
:102A60008091851390918613DC01ED91FC91068095
:102A7000F781E02D199580918513909186130E941E
:102A80007E470E94025767E07BE08091851390911A
:102A900086130E949A480E94025766EE7AE080915F
:102AA0008513909186130E9476488091C4128436D3
:102AB000C8F46FED7AE080918513909186130E949F
:102AC00076486091C41280918513909186130E947C
:102AD0009A6A6DED7AE080918513909186130E9439
:102AE0009A4803C080E00E94D1566CEB7AE0809156
:102AF0008513909186130E9476488091C312843684
:102B0000C8F465EB7AE080918513909186130E945A
:102B100076486091C31280918513909186130E942C
:102B20009A6A63EB7AE080918513909186130E94F4
:102B30009A4803C080E00E94D15662E97AE0809111
:102B40008513909186130E9476486091D1127091FE
:102B5000D2121616170614F50091851310918613DC
:102B6000072E000C880B990B0E9435C120E030E045
:102B70004AE754E40E943AC3AB01BC0122E0C80119
:102B80000E949847C8010E947E476DE87AE08091D4
:102B90008513909186130E949A4803C080E00E949A
:102BA000D1560E94AD978091851390918613DC01D8
:102BB000ED91FC910680F781E02D199580918513A8
:102BC000909186130E947E470E9402576EE27CE03D
:102BD00080918513909186130E949A480E94025713
:102BE0002091DE128091851390918613211103C0EC
:102BF0006CE07CE0CBC165EF7BE00E947648E09121
:102C0000E712E3300CF0E3E080E49BE09A838983F1
:102C10008CE29BE09C838B838FE19BE09E838D8382
:102C200087E19BE098878F83EE0FFF0B21E030E078
:102C30002C0F3D1FE20FF31F60817181809185137E
:102C4000909186130E949A48FF24F3948091E71292
:102C5000811101C0F12C6EED7BE080918513909184
:102C600086130E9476486091E812809185139091B6
:102C70008613611105C06AED7BE00E949A481AC074
:102C80000E949A6A61ED7BE0809185139091861392
:102C90000E9476488091EC07811108C06BEB7BE0C5
:102CA00080918513909186130E9476488DEC99E06F
:102CB0000E947E476091DF127091E012072E000C97
:102CC000880B990B0E9435C120E030E04FE753E4B8
:102CD0000E943AC320E030E048EC52E40E9494C1E4
:102CE00020E030E040E05FE30E94D6C20E94A2C331
:102CF000E62E262F372F8901C090E912D090EA12D4
:102D000064EA7BE080918513909186130E94764857
:102D10008E2D0E94B456043611053CF40E94F256E2
:102D20000A30110514F40E94F25683E00E94CF94F9
:102D3000FF2001F10E943595B601DD0C880B990B3F
:102D40000E9435C120E030E04FE753E40E943AC3CF
:102D500020E030E048EC52E40E9494C120E030E0F2
:102D600040E05FE30E94D6C20E94A2C3862F0E9469
:102D7000B45604C00E942D950E9425950E94EC56E1
:102D80006091E1127091E212072E000C880B990BF2
:102D90000E9435C120E030E04FE753E40E943AC37F
:102DA00020E030E048EC52E40E9494C120E030E0A2
:102DB00040E05FE30E94D6C20E94A2C3E62E262F07
:102DC000372F8901C090EB12D090EC126DE87BE0B8
:102DD00080918513909186130E9476488E2D0E94D3
:102DE000B456043611053CF40E94F2560A3011051F
:102DF00014F40E94F25683E00E94CF94FF2001F168
:102E00000E943595B601DD0C880B990B0E9435C1E7
:102E100020E030E04FE753E40E943AC320E030E086
:102E200048EC52E40E9494C120E030E040E05FE3CF
:102E30000E94D6C20E94A2C3862F0E94B45604C02C
:102E40000E942D950E9425950E94EC566091E312F8
:102E50007091E412072E000C880B990B0E9435C16B
:102E600020E030E04FE753E40E943AC320E030E036
:102E700048EC52E40E9494C120E030E040E05FE37F
:102E80000E94D6C20E94A2C3E62E262F372F8901A8
:102E9000C090ED12D090EE1266E77BE08091851332
:102EA000909186130E9476488E2D0E94B456043667
:102EB00011053CF40E94F2560A30110514F40E94E8
:102EC000F25683E00E94CF94FF2001F10E943595D5
:102ED000B601DD0C880B990B0E9435C120E030E073
:102EE0004FE753E40E943AC320E030E048EC52E45C
:102EF0000E9494C120E030E040E05FE30E94D6C22F
:102F00000E94A2C3862F0E94B45604C00E942D9531
:102F10000E9425950E94EC566FE57BE08091851319
:102F2000909186130E9476486091E5127091E612A6
:102F300000918513109186136115710521F466E5E2
:102F40007BE0C80123C0072E000C880B990B0E9460
:102F500035C120E030E04FE753E40E943AC320E05F
:102F600030E048EC52E40E9494C120E030E040E0C0
:102F70005FE30E94D6C20E94A2C3C8010E944A6CAD
:102F800064E57BE080918513909186130E949A48B6
:102F90000E94AD978091851390918613DC01ED918D
:102FA000FC910680F781E02D199580918513909111
:102FB00086130E947E470E9402576AE97DE0809155
:102FC0008513909186130E949A480E94025720917F
:102FD0002A078091851390918613FE0131966F0127
:102FE000222309F4B7C16BE67DE00E9476480E9477
:102FF000117B0E94D1560E94117B20918513309144
:103000008613882389F068E57DE0C9010E9476482F
:1030100080912D070E94F898BC01809185139091B2
:1030200086130E949A484BC065E47DE0C9010E9466
:10303000764880912A070E94F898BC0180918513F8
:10304000909186130E94764880912B07882389F1FE
:103050006DE37DE080918513909186130E94764800
:10306000E0912B07E4300CF0E0E08EEA93E09A83E5
:1030700089838CEA93E09C838B838AEA93E09E8326
:103080008D8388EA93E098878F83EE0FFF0BEC0D1A
:10309000FD1D6081718180918513909186130E943E
:1030A00076486BE37DE080918513909186130E94B2
:1030B000764880918513909186130E947E4768E23E
:1030C0007DE080918513909186130E9476488091CF
:1030D0002C070091851310918613882321F00E94FC
:1030E000F898BC0102C064E27DE0C8010E949A48E1
:1030F00061E17DE080918513909186130E9476486E
:1031000080912D070091851310918613882321F05B
:103110000E94F898BC0102C06DE07DE0C8010E94E9
:103120009A486AEF7CE080918513909186130E9403
:10313000764880912F078823E1F064EF7CE080914E
:103140008513909186130E94764880912E070E94E5
:10315000F898BC0180918513909186130E9476485F
:103160006DEB76E080918513909186130E948147E4
:1031700003C080E00E94D15661EE7CE0809185130F
:10318000909186130E947648809130078823E1F061
:103190006BED7CE080918513909186130E947648B8
:1031A00080912E070E94F898BC0180918513909120
:1031B00086130E9476486DEB76E08091851390919E
:1031C00086130E94814703C080E00E94D15668ECBC
:1031D0007CE080918513909186130E947648E0915F
:1031E0003107E3300CF0E3E080E79CE09A838983C9
:1031F00084E69CE09C838B838FE59CE09E838D839B
:1032000087E59CE098878F83EE0FFF0BEC0DFD1D8B
:103210006081718180918513909186130E949A48F4
:1032200065EB7CE080918513909186130E9476482F
:10323000E0912307E4300CF0E4E080E59CE09A8321
:1032400089838AE49CE09C838B8383E49CE09E8357
:103250008D838DE39CE098878F8385E39CE09A873C
:103260008987EE0FFF0BEC0DFD1D60817181809150
:103270008513909186130E949A4863EB7CE08091BD
:103280008513909186130E9476486091280780915B
:103290008513909186130E949A6A64EA7CE080917B
:1032A0008513909186130E9476488091230781119F
:1032B00010C06091290780918513909186130E9418
:1032C0009A6A69E97CE080918513909186130E9447
:1032D00076486091240770912507072E000C880B13
:1032E000990B0E9435C120E030E04AE754E40E9487
:1032F0003AC3AB01BC0121E0809185139091861304
:103300000E9498476BE87CE080918513909186132A
:103310000E9476486091260770912707072E000CBF
:10332000880B990B0E9435C120E030E04AE754E455
:103330000E943AC3AB01BC0121E0809185139091BA
:1033400086130E9498476CE77CE0809185139091EA
:10335000861302C06EE77DE00E949A480E94AD97F6
:103360008091851390918613DC01ED91FC9106808C
:10337000F781E02D199580918513909186130E9415
:103380007E470E94025768E17EE08091851390910C
:1033900086130E949A480E9402576BE07EE080915B
:1033A0008513909186130E947648E0911C13E630B5
:1033B0000CF0E6E08EE0D6011D928A95E9F789EFE0
:1033C0009DE09A83898382EE9DE09C838B8380EDD0
:1033D0009DE09E838D8381EC9DE098878F838EEAAC
:1033E0009DE09A87898786EA9DE09C878B87EE0F10
:1033F000FF0BEC0DFD1D6081718180918513909113
:1034000086130E949A480E94AD97809185139091EF
:103410008613DC01ED91FC910680F781E02D199572
:1034200024E73EE841E055272BAB3CAB4DAB5EAB10
:1034300080918513909186130E947E470E940257C7
:103440006DE270E180918513909186130E949A48F5
:103450000E94025764E170E1809185139091861378
:103460000E9476482091E90B8091851390918613F4
:10347000222319F060E170E102C06BE070E10E946C
:103480009A488091E90B882349F162EF7FE08091AF
:103490008513909186130E94764860911A1370915B
:1034A0001B13072E000C880B990B0E9435C120E0DE
:1034B00030E04AE754E40E943AC3AB01BC0122E089
:1034C00080918513909186130E9498476DEE7FE05E
:1034D00080918513909186130E949A4895E4E92E75
:1034E00092E1F92E29E2622E3AE0232E312C44E6B5
:1034F000842E912CD7012C91222309F4FFC1F701CE
:103500003297008111810115110509F4F7C18EEC84
:103510009DE8A1E0BB27820F911DA11DB11DABBF8E
:10352000FC01879177247394811101C0712C209143
:10353000851330918613C8010197849790F56DEC3F
:103540007FE0C9010E94764809500C3148F4E02F11
:10355000F0E0EE0FFF1FE15EFD4F6081718102C060
:1035600063E27EE080918513909186130E947648F5
:103570000C3130F4E02FF0E0E95AFD4F808101C0BA
:1035800080E090E08D53904F092E000CAA0BBB0BEE
:10359000ABBFFC0187919EE0981B892F09F053C1B6
:1035A00054C1C801845691098438934008F03FC043
:1035B00063EB7FE0C9010E947648C801B4010E9414
:1035C0006DC46130710531F06230710559F46FEAF4
:1035D0007FE002C061EB7FE08091851390918613BC
:1035E0000E9476480E94FA56A0908513B0908613E8
:1035F0007720B1F0C8010E94B695811107C06BEA2F
:103600007FE0C5010E94764887E01DC1813009F046
:103610001CC168EA7FE0C5010E94764888E013C1BA
:103620006FE97FE0C5010E94764882E00CC1C801C5
:10363000885E93408035964408F05CC0C80168EE0F
:1036400073E00E946DC45B0162E97FE0C9010E94E2
:103650007648FAE0AF16B10410F40E94F256B501B4
:1036600080918513909186130E944A6C0E94FA56AD
:1036700040908513509086137720B1F1C8010E94C5
:10368000B695782E6DE87FE0C2010E947648672DDE
:1036900080918513909186130E949A6A67E87FE073
:1036A00080918513909186130E94764828E13CEF23
:1036B000A29EC001A39E900DB29E900D1124800F7A
:1036C000911FB1010E9481C4772780918513909149
:1036D00086130E944A6C65E87FE080918513909183
:1036E00086130E947648B1C06CE77FE0C2010E9459
:1036F000764861C0F801E853FA44E83E43E0F40735
:1037000008F046C0EC30F10508F09FC08827EE585D
:10371000FF4F8F4F0C9494C46DE67FE019C062E6B2
:103720007FE0C9010E94764883E18DC060E57FE0BB
:1037300027C060E47FE016C063E37FE055C067E226
:103740007FE0C9010E94764882E17DC068E17FE0A8
:10375000C9010E9476488FE076C069E07FE0F8CF2B
:1037600069EF7EE0C9010E9476488EE06CC066EE8B
:103770007EE0C9010E9476488BE065C064ED7EE082
:10378000C9010E9476488CE05EC067EC7EE02CC0E8
:10379000C80180529E44883E934078F4005260EB0A
:1037A0007EE0C9010E9476480A3010F40E94F25669
:1037B000802F0E94B45684E046C0C80188509245CC
:1037C000883E934020F4085069E97EE0EACF013F4B
:1037D000B5E51B0719F468E87EE01CC0023FE5E58B
:1037E0001E0739F46BE77EE0C9010E94764881E14B
:1037F0002AC0033FF5E51F0739F46DE67EE0C901F5
:103800000E94764880E11FC0043F45E5140739F463
:103810006CE57EE0C9010E9476488DE014C0053F4A
:1038200055E5150739F464E47EE0C9010E94764845
:1038300086E009C0063F154541F46BE27EE0C90110
:103840000E94764885E00E94CF9468EE7FE08091E8
:103850008513909186130E9476486DED7FE08091EC
:103860008513909186130E947648D7016C9170E081
:1038700080918513909186130E944A6CF701808194
:103880008A3020F482E00E94CF9404C0843610F481
:103890000E94F2560E94FA56D7014C91649EA001F4
:1038A0001124052E000C660B770B8BA99CA9ADA9E2
:1038B000BEA9480F591F6A1F7B1FD6018A019B01B1
:1038C0000F5F1F4F2F4F3F4F6BBFFA0187918D93B3
:1038D000B901A8018111F2CFB601809185139091B1
:1038E00086130E9481478091851390918613DC0195
:1038F000ED91FC910680F781E02D1995B3E0EB0E78
:10390000F11CEDEBEE16E2E1FE0609F0F3CD0E94AC
:10391000AD978091851390918613DC01ED91FC9118
:103920000680F781E02D199580918513909186137B
:103930000E947E470E9402576EE870E180918513D5
:10394000909186130E949A480E9402576BE770E19B
:1039500080918513909186130E9476480E948E7301
:1039600020E030E040E050E40E942FC12091851318
:103970003091861387FF3FC068E770E1C90159C0E5
:10398000F090F0120091F31211E00C9455126AE1DC
:103990007AE080918513909186130E947648609119
:1039A000931480918513909186130E949A6A68E11E
:1039B0007AE080918513909186130E9476480C944A
:1039C000DE126FEC79E080918513909186130E944E
:1039D00076486091951480918513909186130E948A
:1039E0009A6A6DEC79E080918513909186130E941C
:1039F00076480C943D1364E770E1C9010E949A482F
:103A000061E670E180918513909186130E9476485B
:103A10000E948E73AB01BC0122E0809185139091CE
:103A200086130E9498476FE570E18091851390910D
:103A300086130E949A486CE470E1809185139091FE
:103A400086130E947648809166130E94C356209187
:103A500066138091851390918613222379F069E48F
:103A600070E10E9476480E940E956FE370E18091AC
:103A70008513909186130E949A4802C00E947E4747
:103A80000E94AD978091851390918613DC01ED9192
:103A9000FC910680F781E02D199580918513909116
:103AA00086130E947E470E94025766EE70E1809165
:103AB0008513909186130E949A480E94025762EDE6
:103AC00070E180918513909186130E947648409111
:103AD0005613509157136091581370915913809158
:103AE0008513909186130E94376C6EEB70E1809184
:103AF0008513909186130E94764840915E135091F1
:103B00005F136091601370916113809185139091A0
:103B100086130E94376C6AEA70E180918513909158
:103B200086130E94764840915A1350915B1360911E
:103B30005C1370915D1380918513909186130E94A0
:103B4000376C66E970E180918513909186130E942D
:103B500076484091621350916313609164137091A1
:103B6000651380918513909186130E94376C0E9493
:103B7000AD978091851390918613DC01ED91FC91B6
:103B80000680F781E02D1995809185139091861319
:103B90000E947E470E940257E6960FB6F894DEBF59
:103BA0000FBECDBFDF91CF911F910F91FF90EF908E
:103BB000DF90CF90BF90AF909F908F907F906F904D
:103BC0005F904F903F902F9008952F923F924F9289
:103BD0005F926F927F928F929F92AF92BF92CF929D
:103BE000DF92EF92FF920F931F93CF93DF93CDB7A6
:103BF000DEB7AB970FB6F894DEBF0FBECDBF8DED2D
:103C000091E00E9460C2603F7F4B8105910519F0F1
:103C10000E942B8F08C041EE51E060E070E08EE919
:103C200091E10E9448C240E052EC61E070E08DEC0E
:103C300099E00E941E8140915A1350915B1360914C
:103C40005C1370915D1380E399E00E941E814091A6
:103C50005E1350915F13609160137091611383E95B
:103C600098E00E941E81409162135091631360910D
:103C700064137091651386EF97E00E941E8183EABA
:103C80009EE09093F0078093EF0784E69CE090938A
:103C9000EE078093ED0711E01093A50E8DEC99E0EF
:103CA0009093A3148093A2141092A4141092A90EBE
:103CB0001092A60E1092A80E1092A70E1093031445
:103CC0000E941C6080917A138093A607109287133C
:103CD0001092800082E0809381008FE286BB109278
:103CE0006F0010928500109284009BE29093A000D8
:103CF00099E09093A10089BB109272001092A500E8
:103D00001092A4001092A9001092A8001092AB008B
:103D10001092AA001092AD001092AC0099EA909314
:103D20002001109321018ABB10927300109225018B
:103D300010922401109229011092280110922B0157
:103D400010922A0110922D0110922C0180913B12A9
:103D500090913C1280933B0790933C07813001F592
:103D60008FE380930C0C10920D0C61E00E94D04AFE
:103D700082E09CE00E94E99210920E0C1092110CCD
:103D80001092100C80913C07882329F082E09CE07F
:103D90000E94BC9411C082E09CE00E9495940CC0EB
:103DA00080913C07882311F062E001C060E08FE35E
:103DB0000E94D04A0E94947480913D1290913E12CC
:103DC0008093410790934207813001F58EE3809301
:103DD0003D0C10923E0C61E00E94D04A83E39CE0CF
:103DE0000E94E99210923F0C1092420C1092410CEA
:103DF00080914207882329F083E39CE00E94BC94D1
:103E000011C083E39CE00E9495940CC0809142070E
:103E1000882311F062E001C060E08EE30E94D04A86
:103E20000E94617460E085E40E94D04A62E08CE305
:103E30000E94D04A62E08BE30E94D04A62E080E4B4
:103E40000E94D04A62E081E40E94D04A62E082E4AB
:103E50000E94D04A62E081E20E94D04A62E084E49B
:103E60000E94D04A61E089E30E94D04A61E08AE37F
:103E70000E94D04A0E9422720E94597261E085E33A
:103E80000E94D04A61E085E00E94D04A61E070E083
:103E900085E00E940C4B61E084E00E94D04A61E022
:103EA00087E00E94D04A61E089E20E94A14A61E075
:103EB00089E20E94D04A519A60E085E30E94A14ABB
:103EC00060E085E00E94A14A60E084E00E94A14A8F
:103ED00060E087E00E94A14A599861E088E00E9472
:103EE000D04A80E090E09C0122563E4EF901E9550F
:103EF000FF4F40814F3629F4329720813181232BA7
:103F000031F403968837910571F760E001C061E0F4
:103F100088E00E94A14A61E08DE20E94D04A61E0FF
:103F20008EE20E94D04A61E08CE20E94D04A61E0B9
:103F30008BE20E94D04A60E08BE20E94A14A0E947C
:103F400059720E94C86B8091F20B813009F058C001
:103F50008091F50B9091F60BA091F70BB091F80BB7
:103F60004091F90B5091FA0B6091FB0B7091FC0B97
:103F7000841B950BA60BB70B84379E40A105B1059A
:103F800000F30E942B8F0E94EC560E94EC560E9478
:103F9000025764EF70E180918513909186130E941F
:103FA000764801E010E00E9426720E9459726EEE7F
:103FB00072E080E090E00E94174C61EF70E1809128
:103FC0008513909186130E9476480E9422720E9467
:103FD00055720530110531F064EF71E080E090E03A
:103FE0000E94174C0F5F1F4F06301105E1F60E942B
:103FF000EC560E9402570E94EC560E94EC5602C0FA
:1040000081119FCF80916F00826080936F008091BB
:104010008400909185008056904F90938900809302
:1040200088000E94352C85E69CE09093B71480931D
:10403000B6141091151320911413809103139091CD
:104040000513309106133093F50790930A07809378
:104050000B0730E0AFEFB0E00E94C6C224E630E0CC
:1040600040E050E00E9478C220939714612F70E0E6
:1040700080E090E00E9433C120ED34E448E55BE34A
:104080000E9494C126E636E646E25FE30E94D6C26D
:104090006093F1077093F2078093F3079093F4070E
:1040A0001093961410929500109294001092900024
:1040B0008CE08093910084EF90E09093990080933E
:1040C000980081E088BB82E08093710080910002BB
:1040D0000E94B75F80911C13863040F010921C1331
:1040E00060E070E08EE791E00E945B6B10911C1322
:1040F000123009F444C008F5112309F466C01130E8
:1041000009F05BC08CE090E00E94A8C42BE433E08F
:10411000DC0111963C932E9323E938E01B963C93E7
:104120002E931A979093A3078093A20710931F0FC3
:104130001093220F1093250F67C0133009F45EC04F
:104140001430D9F586E090E00E94A8C48C0125EBDC
:1041500033E0DC012D933D93CD0141E065E67CE049
:104160000E94157E87E792E0F80191838083109387
:10417000A3070093A20781E080931F0F41C086E050
:1041800090E00E94A8C421EE32E0FC01318320833C
:104190009093A3078093A2078FB7F8942CED35E096
:1041A0003093DE102093DD101092E3108FBF81E07A
:1041B00080931F0F8093220F25C010921C1360E084
:1041C00070E08EE791E00E945B6B86E090E00E94D9
:1041D000A8C48C0125EB33E0DC012D933D93CD0188
:1041E00040E065E67CE00E94157E87E792E0F801FA
:1041F000918380831093A3070093A20710921F0F4F
:104200001092220F1092250F8091A2079091A30780
:10421000DC01ED91FC910190F081E02D19958091E8
:10422000130F81111FC08091160F81111BC0809147
:10423000190F811117C080911C0F811113C080913B
:104240001F0F81110FC08091220F81110BC080912F
:10425000250F811107C081E00E941860882309F4AE
:1042600019C311C3A12CB12C912C1DA2412C512C8E
:10427000612C712C812C03E616E0EE24EA94A3E075
:10428000FA2ECC24CA94DD24D39487E5282E86E028
:10429000382EC50182569E4EFC01E955FF4FE08144
:1042A000EE2309F4E7C2DC01AB55BF4F8D919C9121
:1042B000892B09F4DFC28E2F90E0FC01F797EB32D7
:1042C000F10508F0D7C28827E258FF4F8F4F0C94B2
:1042D00094C48091130F882309F4CCC28110CAC200
:1042E00089E190E00E94A8C49C01FC011183008335
:1042F00087E090E09383828315821482F782E682BE
:10430000D186C086108EC9012AA73BA70E94D6413C
:104310002AA53BA5E7E3F4E0D901ED93FC933093A4
:10432000040F2093030FC9010E94BF8B7DC18091B0
:10433000160F882309F49EC271109CC289E190E097
:104340000E94A8C49C01DC0111961C930E93E6E028
:10435000F0E01396FC93EE93129715961C921E9222
:1043600014971796FC92EE9216971996DC92CE92BD
:10437000189758961C922AA73BA70E94D6412AA5B7
:104380003BA5E7E3F4E0D901ED93FC933093060FEE
:104390002093050FC9010E94BF8B74C18091190F32
:1043A000882309F467C2611065C289E190E00E9428
:1043B000A8C49C01DC0111961C930E93E5E0F0E08B
:1043C0001396FC93EE93129715961C921E921497D7
:1043D0001796FC92EE9216971996DC92CE92189749
:1043E00058961C922AA73BA70E94D6412AA53BA516
:1043F000E7E3F4E0D901ED93FC933093080F2093A9
:10440000070FC9010E94BF8B6BC180911C0F8823CD
:1044100009F430C251102EC289E190E00E94A8C474
:104420009C01DC0111961C930E93E4E0F0E01396DE
:10443000FC93EE93129715961C921E921497179662
:10444000FC92EE9216971996DC92CE921897589697
:104450001C922AA73BA70E94D6412AA53BA5E7E3C9
:10446000F4E0D901ED93FC9330930A0F2093090FE8
:10447000C9010E94BF8B62C180911F0F882309F47C
:10448000F9C14110F7C189E190E00E94A8C49C01E4
:10449000DC0111961C930E93E2E0F0E01396FC937E
:1044A000EE93129715961C921E9214971796FC92F3
:1044B000EE9216971996DC92CE92189758961C9207
:1044C0002AA73BA70E94D6412AA53BA5E7E3F4E033
:1044D000D901ED93FC9330930C0F20930B0FC9017E
:1044E0000E94BF8B59C18091220F882309F4C2C159
:1044F0002DA12111BFC189E190E00E94A8C49C01B7
:10450000DC0111961C930E93E1E0F0E01396FC930E
:10451000EE93129715961C921E9214971796FC9282
:10452000EE9216971996DC92CE92189758961C9296
:104530002AA73BA70E94D6412AA53BA5E7E3F4E0C2
:10454000D901ED93FC9330930E0F20930D0FC90109
:104550000E94BF8B59C18091250F882309F48AC11D
:10456000911088C189E190E00E94A8C49C01DC01FF
:1045700011961C930E9313961C921E9212971596E9
:104580001C921E9214971796FC92EE92169719960B
:10459000DC92CE92189758961C922AA73BA70E94AD
:1045A000D6412AA53BA587E394E0F9019183808356
:1045B0003093100F20930F0FC9010E94BF8B58C179
:1045C0008091130F882309F455C1811053C18CE1E8
:1045D00090E00E94A8C49C01DC0111961C930E93EC
:1045E000E7E0F0E01396FC93EE93129715961C9279
:1045F0001E9214971796FC92EE9216971996DC92DB
:10460000CE92189758961C922AA73BA70E94D64193
:104610002AA53BA5D9012D923C923093120F2093ED
:10462000110FC9010E945F8C8824839423C180915B
:10463000160F882309F41EC171101CC18CE190E093
:104640000E94A8C49C01FC011183008386E090E0D5
:104650009383828315821482F782E682D186C08694
:10466000108EC9012AA73BA70E94D6412AA53BA5C7
:10467000D9012D923C923093150F2093140FC9014C
:104680000E945F8C77247394F5C08091190F882362
:1046900009F4F0C06110EEC08CE190E00E94A8C463
:1046A0009C01FC011183008385E090E09383828369
:1046B00015821482F782E682D186C086108EC901E7
:1046C0002AA73BA70E94D6412AA53BA5D9012D9236
:1046D0003C923093180F2093170FC9010E945F8CF2
:1046E00066246394C7C080911C0F882309F4C2C05C
:1046F0005110C0C08CE190E00E94A8C49C01FC0154
:104700001183008384E090E0938382831582148276
:10471000F782E682D186C086108EC9012AA73BA700
:104720000E94D6412AA53BA5D9012D923C923093F7
:104730001B0F20931A0FC9010E945F8C55245394BC
:1047400099C080911F0F882309F494C0411092C032
:104750008CE190E00E94A8C49C01FC0111830083BD
:1047600082E090E09383828315821482F782E6824E
:10477000D186C086108EC9012AA73BA70E94D641C8
:104780002AA53BA5D9012D923C9230931E0F209370
:104790001D0FC9010E945F8C442443946BC080911B
:1047A000220F882309F466C02DA1211163C08CE17A
:1047B00090E00E94A8C49C01DC0111961C930E930A
:1047C000E1E0F0E01396FC93EE93129715961C929D
:1047D0001E9214971796FC92EE9216971996DC92F9
:1047E000CE92189758961C922AA73BA70E94D641B2
:1047F0002AA53BA5D9012D923C923093210F2093FD
:10480000200FC9010E945F8C21E02DA333C080914D
:10481000250F882379F191102DC08CE190E00E9442
:10482000A8C49C01DC0111961C930E9313961C9254
:104830001E92129715961C921E9214971796FC9230
:10484000EE9216971996DC92CE92189758961C9273
:104850002AA73BA70E94D6412AA53BA5F901318290
:1048600020823093240F2093230FC9010E945F8C74
:1048700099249394F3E0AF0EB11C28E7A216B1047B
:1048800009F007CDE8CC82E00E941860882311F07F
:104890001FA216C081E00E941860882329F082E0E0
:1048A0000E94FC5F81119CC78CE30E94794A892B8E
:1048B00009F087C78CE30E94794A892B09F087C7E2
:1048C00086E0ECE4F3E1DE01549601900D928A95C6
:1048D000E1F78091451390915513B09046130091E4
:1048E0004713109148137091491360914A135091E6
:1048F0004B13409152132091531330915413E09174
:10490000A207F091A307FEA3EDA3A0913D0FB091E4
:104910003E0FB9A7A8A79090781360907313E0900A
:104920006C13F0906D138090761370907513C09097
:10493000D112D090D2125090D4124090CF12309019
:10494000D012BFA1BB8B8A8F9B8FBC8E0D8F1E8F09
:104950007F8F68A359A34AA33CA32BA3F2E1AF2EF8
:10496000FE017396DE01119601900D92AA94E1F773
:10497000E5E6FCE0F0931407E0931307EFA1E98369
:1049800088879987BA860B871C877D876E875F87A4
:10499000488B3A8B298B22E1FE013196A3E2B7E0E6
:1049A00001900D922A95E1F7992321F0863011F0BC
:1049B00010922B073092DB134092DC135092D213EB
:1049C000D092CB13C092CA1360923F0F7092CF1354
:1049D0008092CE13F092CD13E092CC139092DA1322
:1049E00088A599A59093D1138093D0138DA19EA1F2
:1049F000909316078093150787E08093EE0A109234
:104A0000EF0A61E00E94D04A84EE9AE00E94E992A7
:104A10001092F00A1092F30A1092F20A80912E0777
:104A2000811102C010922F0790912A07911105C0A1
:104A3000811103C01092D90B98C08091D40B909132
:104A4000D50B0E943D9581E08093D90B809123077F
:104A5000882359F1813071F08330C1F488E293E208
:104A6000909325078093240789E08093280780E1AD
:104A700097E217C088EB9BE090932507809324076B
:104A800083E08093280788E99AE30BC088E893E1E4
:104A9000909325078093240786E08093280780EE73
:104AA0009EE2909327078093260780912A07882308
:104AB000E9F180912E076091280770E08823C9F002
:104AC000809130078823A9F080E090E00E9433C1F4
:104AD0009B01AC0160E070E088EC92E40E943AC374
:104AE00060931707709318078093190790931A071C
:104AF00025C080E090E00E9433C19B01AC0160E0E2
:104B000070E088EC92E40E943AC3609317077093B8
:104B100018078093190790931A0710920E071092A6
:104B20000F0710921007109211071FC0109217075D
:104B3000109218071092190710921A07609129070E
:104B400070E080E090E00E9433C19B01AC0160E026
:104B500070E088EC92E40E943AC360930E07709371
:104B60000F07809310079093110710929D111092D8
:104B70001B071092120710921C0710921D0710922B
:104B80001E0710921F070E944E815098589AE8986D
:104B9000809169008C7F809369008091DC13882369
:104BA00021F080916900826003C080916900836078
:104BB00080936900E8980E94FA8380E090E040E0EA
:104BC0009C0122563E4EF901E955FF4F5081552375
:104BD00031F0329720813181232B09F04F5F03960A
:104BE0008837910569F740933607A3E4B7E020E0E2
:104BF00030E087E3282E86E5382E98E8492E9BE59D
:104C0000592E4DE5642E4BE5742E50E7852E5BE55D
:104C1000952E6AE3A62E66E5B62E47E554E50DE32C
:104C200014E57AE4E72E74E5F72EE7E8CE2EE3E507
:104C3000DE2EC90182569E4EFC01E955FF4F608170
:104C4000662309F4B0C38B559F4FFC01808191818D
:104C5000892B09F4A8C370E0FB013197E53AF1050F
:104C600008F0A1C38827E755FF4F8F4F0C9494C4D9
:104C700086E39BE511969C938E9395C385E39BE514
:104C800011969C938E938FC383E39BE511969C931F
:104C90008E9389C38DE29BE511969C938E9383C37B
:104CA0008BE29BE511969C938E937DC384EA9AE5F3
:104CB00011969C938E9377C385EA9AE511969C93FF
:104CC0008E9371C387E89AE511969C938E936BC37C
:104CD00083E79AE511969C938E9365C384E69AE5E3
:104CE00011969C938E935FC388E09AE511969C93EE
:104CF0008E9359C38EEA98E511969C938E9353C375
:104D00008BEF99E511969C938E934DC388E899E5B6
:104D100011969C938E9347C382EF99E511969C93CD
:104D20008E9341C38AEF99E511969C938E933BC372
:104D300084EF99E511969C938E9335C38BEB99E59F
:104D400011969C938E932FC383EE99E511969C93B5
:104D50008E9329C38CED99E511969C938E9323C372
:104D60008BEA99E511969C938E931DC389EA99E588
:104D700011969C938E9317C387EA99E511969C939D
:104D80008E9311C387E999E511969C938E930BC37B
:104D900085E999E511969C938E9305C386E899E57C
:104DA00011969C938E93FFC286E799E511969C938A
:104DB0008E93F9C284E799E511969C938E93F3C282
:104DC00082E799E511969C938E93EDC288E297E570
:104DD00011969C938E93E7C286E297E511969C9379
:104DE0008E93E1C284E297E511969C938E93DBC289
:104DF00086E890E711969C938E93D5C280E799E55B
:104E000011969C938E93CFC280E699E511969C9360
:104E10008E93C9C289ED97E511969C938E93C3C278
:104E20008AEB97E511969C938E93BDC28EE599E52A
:104E300011969C938E93B7C28FE299E511969C933D
:104E40008E93B1C288E299E511969C938E93ABC282
:104E500087EF98E511969C938E93A5C286E595E918
:104E600011969C938E939FC28CEA98E511969C9321
:104E70008E9399C28AEA98E511969C938E9393C279
:104E800087EA98E511969C938E938DC283E898E506
:104E900011969C938E9387C28FE598E511969C930B
:104EA0008E9381C284EA98E511969C938E937BC27F
:104EB00080E898E511969C938E9375C28CE598E5F1
:104EC00011969C938E936FC281EA98E511969C93FC
:104ED0008E9369C28DE798E511969C938E9363C279
:104EE00089E598E511969C938E935DC28EE998E5CD
:104EF00011969C938E9357C28AE798E511969C93DE
:104F00008E9351C286E598E511969C938E934BC281
:104F10008BE998E511969C938E9345C287E798E5B7
:104F200011969C938E933FC283E598E511969C93CE
:104F30008E9339C288E998E511969C938E9333C27B
:104F400084E798E511969C938E932DC280E598E5B1
:104F500011969C938E9327C285E998E511969C93B0
:104F60008E9321C281E798E511969C938E931BC284
:104F70008DE498E511969C938E9315C282E998E58D
:104F800011969C938E930FC28EE698E511969C9392
:104F90008E9309C28AE498E511969C938E9303C27E
:104FA0008FE898E511969C938E93FDC18BE698E56A
:104FB00011969C938E93F7C187E498E511969C9384
:104FC0008E93F1C18CE898E511969C938E93EBC17A
:104FD00088E698E511969C938E93E5C184E498E564
:104FE00011969C938E93DFC189E898E511969C9366
:104FF0008E93D9C185E698E511969C938E93D3C183
:1050000081E498E511969C938E93CDC186E898E54E
:1050100011969C938E93C7C182E698E511969C9356
:105020008E93C1C18EE398E511969C938E93BBC17C
:105030008EE497E511969C938E93B5C18AE398E52B
:1050400011969C938E93AFC186E398E511969C933D
:105050008E93A9C182E398E511969C938E93A3C188
:105060008EE298E511969C938E939DC18AE298E515
:1050700011969C938E9397C186E298E511969C9326
:105080008E9391C182E298E511969C938E938BC189
:105090008EE198E511969C938E9385C185E497E502
:1050A00011969C938E937FC182E297E511969C9313
:1050B0008E9379C180E297E511969C938E9373C18C
:1050C00088EF97E511969C938E936DC188E697E5DE
:1050D00011969C938E9367C18CE397E511969C93F0
:1050E0008E9361C18AE397E511969C938E935BC181
:1050F00088E397E511969C938E9355C18EE896E5CB
:1051000011969C938E934FC18CE396E511969C93D8
:105110008E9349C182E495E511969C938E9343C189
:1051200087EF94E511969C938E933DC18AEB9BE5A6
:1051300011969C938E9337C186EA9BE511969C93BA
:105140008E9331C182E99BE511969C938E932BC17E
:105150008FE995E911969C938E9325C187E096E59A
:1051600011969C938E931FC18AEF95E511969C939F
:105170008E9319C184EE95E511969C938E9313C17D
:1051800082EC95E511969C938E930DC182EE95E588
:1051900011969C938E9307C184EC95E511969C9390
:1051A0008E9301C185E793E511969C938E93FBC086
:1051B0008BE293E511969C938E93F5C08DE493E575
:1051C00011969C938E93EFC08DE393E511969C937B
:1051D0008E93E9C08FE593E511969C938E93E3C07F
:1051E00083E093E511969C938E93DDC083EF92E567
:1051F00011969C938E93D7C085E193E511969C936D
:105200008E93D1C08BEE94E511969C938E93CBC078
:105210008FED94E511969C938E93C5C083ED94E534
:1052200011969C938E93BFC087EC94E511969C9346
:105230008E93B9C08BEB94E511969C938E93B3C07B
:105240008FEA94E511969C938E93ADC083EA94E522
:1052500011969C938E93A7C083EF93E511969C9330
:105260008E93A1C081EE93E511969C938E939BC083
:105270008FEC93E511969C938E9395C08DEB93E5FF
:1052800011969C938E938FC08BEA93E511969C9315
:105290008E9389C089E993E511969C938E9383C080
:1052A0001196DC92CE927FC01196FC92EE927BC05A
:1052B00011961C930E9377C08DE794E511969C93FD
:1052C0008E9371C011965C934E936DC01196BC92F3
:1052D000AE9269C011969C928E9265C011967C9296
:1052E0006E9261C011965C924E925DC011963C9296
:1052F0002E9259C0E4E3F6E51196FC93EE9353C069
:105300008BE296E511969C938E934DC0E8E2F6E50C
:105310001196FC93EE9347C085E296E511969C9317
:105320008E9341C0E2E2F6E51196FC93EE933BC00A
:105330008FE196E511969C938E9335C0E4E1F6E5F6
:105340001196FC93EE932FC08DE196E511969C93F8
:105350008E9329C0E6E1F6E51196FC93EE9323C007
:105360008FE194E511969C938E931DC0E2E1F4E5E4
:105370001196FC93EE9317C085E094E511969C93EB
:105380008E9311C0EFE9F5E51196FC93EE930BC0F7
:105390008DE895E511969C938E9305C0E1EBF5E5BC
:1053A0001196FC93EE932D5F3F4F129628373105EF
:1053B00009F03FCC1092370780913B07811114C050
:1053C00080E090E0FC01ED5BFD4E208131812456B0
:1053D00031092436310528F003968837910591F775
:1053E00003C081E08093370710923D078091410709
:1053F000811114C080E090E0FC01ED5BFD4E208146
:105400003181285C31092436310528F0039688372C
:10541000910591F703C081E080933D078091A20739
:105420009091A307DC01ED91FC91EE5AFF4F209182
:105430001F133091201340911D1350911E130190A2
:10544000F081E02D61E019958091A2079091A3076A
:10545000DC01ED91FC91EE5AFF4F20912313309126
:10546000241340912113509122130190F081E02DDB
:1054700062E019958091A2079091A307DC01ED915C
:10548000FC91EE5AFF4F2091271330912813409141
:105490002513509126130190F081E02D63E01995BA
:1054A0008091A2079091A307DC01ED91FC91EE5A47
:1054B000FF4F2091321330913313409130135091AC
:1054C00031130190F081E02D64E019958091A207DD
:1054D0009091A307DC01ED91FC91EE5AFF4F2091D2
:1054E0003613309137134091341350913513019096
:1054F000F081E02D65E019958091A2079091A307B6
:10550000DC01ED91FC91EE5AFF4F20913A1330915E
:105510003B1340913813509139130190F081E02DE5
:1055200066E019958091A2079091A307DC01ED91A7
:10553000FC91EC5AFF4F0190F081E02D409129132E
:1055400061E019958091A2079091A307DC01ED918C
:10555000FC91EC5AFF4F0190F081E02D40912A130D
:1055600062E019958091A2079091A307DC01ED916B
:10557000FC91EC5AFF4F0190F081E02D40912B13EC
:1055800063E019958091A2079091A307DC01ED914A
:10559000FC91EC5AFF4F0190F081E02D40913C13BB
:1055A00064E019958091A2079091A307DC01ED9129
:1055B000FC91EC5AFF4F0190F081E02D40913D139A
:1055C00065E019958091A2079091A307DC01ED9108
:1055D000FC91EC5AFF4F0190F081E02D40913E1379
:1055E00066E019958091A2079091A307DC01ED91E7
:1055F000FC9102ACF3ADE02D60912D1319958091D3
:10560000A2079091A307DC01ED91FC9106ACF7ADE8
:10561000E02D6091421319958091A2079091A30704
:10562000DC01ED91FC9100A8F1A9E02D60912E1311
:1056300019958091A2079091A307DC01ED91FC914F
:1056400006A8F7A9E02D60912F1319958091A20764
:105650009091A307DC01ED91FC91E65BFF4F019077
:10566000F081E02D4091431360E019958091A207ED
:105670009091A307DC01ED91FC91E65BFF4F019057
:10568000F081E02D4091441361E0199580E090E0B5
:105690009C0122563E4EF901E955FF4F40814237A9
:1056A00031F4329720813181232B09F09FC003967A
:1056B0008837910569F70E94B1968091A207909171
:1056C000A307DC01ED91FC91EC59FF4F0190F081B3
:1056D000E02D40E060913F1319958091A2079091D1
:1056E000A307DC01ED91FC91EC59FF4F0190F08193
:1056F000E02D41E06091411319958091A2079091AE
:10570000A307DC01ED91FC91EC59FF4F0190F08172
:10571000E02D42E060914013199520916A1330E02A
:10572000AFEFB0E00E94C6C224E630E040E050E0B7
:105730000E9478C220938F138091691381110E9477
:10574000B2720E9459A20E9476846B017C0110E023
:1057500011110FC08091A607882359F02CE234E57F
:1057600040ED57E060E070E085E69CE00E941B3F62
:1057700011E00E94878E882351F00E94CC720E9413
:10578000355C0E9459720E94148E0E94E9710E9439
:1057900018A1029711F00E9468640E94AD970E94C0
:1057A00018A10297A9F60E947684DC01CB018C191E
:1057B0009D09AE09BF098C3B9240A105B10540F29D
:1057C00018C082E00E94186081110DC073C882E089
:1057D0000E94FC5F882309F473C8A3E0AFA370C8DC
:1057E00081E08FA36DC892E09FA36AC80E94A5962E
:1057F00064CF0E94927A0E9459728091ED0B8111C0
:1058000002C00E94CF6C0E94EBA086E30E94D34BA3
:10581000BC01990F880B990B6115710581059105E4
:1058200011F00E94B0C02EEE32E548EE53E060E089
:1058300070E085E69CE0AB960FB6F894DEBF0FBE35
:10584000CDBFDF91CF911F910F91FF90EF90DF902F
:10585000CF90BF90AF909F908F907F906F905F9010
:105860004F903F902F900C941B3F5F926F927F92CE
:105870008F929F92AF92BF92CF92DF92EF92FF9260
:105880000F931F93CF93DF9381E08093130F809347
:10589000160F8093190F80931C0F8093280F80930D
:1058A0002B0F909106139150963040F08093061381
:1058B00061E070E088E691E00E945B6B90910613D6
:1058C0002DEF290F8091BB12233008F011C28A30CE
:1058D00079F03CF4883009F463C0893009F4C0C120
:1058E000B6C18B3009F4A4C08C3009F4E6C0AFC156
:1058F00084E290E00E94A8C4FC018091791328E022
:1059000030E0338322838824839499249A94958267
:105910008482AA24AA94B12CB782A682118610860A
:10592000108ED3E87D2E718E93E9C92E98E0D92E82
:10593000D38EC28E27E6E22E24E0F22EF182E082A0
:10594000CEE5D3E1D1A3C0A312A283A3F09399071C
:10595000E0939807CF010E94ED4C84E290E00E9412
:10596000A8C4FC018091791329E030E033832283BD
:1059700095828482B782A68211861086108E718EDF
:10598000D38EC28EF182E082D1A3C0A312A283A3E0
:10599000F0939707E0939607CF010E94ED4C0EC35A
:1059A00080E290E00E94A8C4FC0188E090E093832C
:1059B00082838824839499249A9495828482AA2449
:1059C000AA94B12CB782A68211861086108E7AE036
:1059D000D72ED18EA3E9EA2EA8E0FA2EF38EE28E1E
:1059E000CFE4D4E0D183C083F0939907E093980784
:1059F000CF010E94564C80E290E00E94A8C4FC01B6
:105A000089E090E09383828395828482B782A68224
:105A100011861086108ED18EF38EE28ED183C083D4
:105A2000F0939707E0939607CF010E94564CC6C2A9
:105A300089E190E00E94A8C4FC0188E090E0938393
:105A40008283CC24C394DD24DA94D582C482EE24EC
:105A5000EA94F12CF782E68211861086108EC3E458
:105A6000D4E0D183C083F0939907E0939807CF01E6
:105A70000E94898C1092280F80910613843009F0BF
:105A80009DC289E190E00E94A8C4FC0189E090E0F9
:105A900093838283D582C482F782E6821186108640
:105AA000108ED183C083F0939707E0939607CF01C0
:105AB0000E94898C10922B0F81C2943009F04BC048
:105AC00089E190E00E94A8C4EC01B3E68B2EB6E019
:105AD0009B2E9982888287E090E09B838A83AA2408
:105AE000A394BB24BA94BD82AC82CC24CA94D12C9A
:105AF000DF82CE8219861886188ECE010E94D6418A
:105B000027E3E22E24E0F22EF982E882D09399076F
:105B1000C0939807CE010E94BF8B1092130F89E1AA
:105B200090E00E94A8C4EC019982888286E090E00F
:105B30009B838A83BD82AC82DF82CE8219861886DF
:105B4000188ECE010E94D641F982E882D093970741
:105B5000C09396074DC0953009F050C089E190E0A0
:105B60000E94A8C4EC0173E6872E76E0972E9982F6
:105B7000888287E090E09B838A83AA24A394BB2435
:105B8000BA94BD82AC82CC24CA94D12CDF82CE825E
:105B900019861886188ECE010E94D641A7E3EA2EF8
:105BA000A4E0FA2EF982E882D0939707C093960773
:105BB000CE010E94BF8B1092130F89E190E00E94EA
:105BC000A8C4EC019982888286E090E09B838A8356
:105BD000BD82AC82DF82CE8219861886188ECE01F5
:105BE0000E94D641F982E882D0939907C093980722
:105BF000CE010E94BF8B1092160FE0C189E190E0A8
:105C00000E94A8C4EC0183E696E09983888387E02C
:105C100090E09B838A8381E09FEF9D838C838FEF4D
:105C200090E09F838E8319861886188ECE010E947D
:105C3000D64187E394E099838883D0939907C093F2
:105C40009807CE010E94BF8B1092130FB7C189E055
:105C50008093BB1269E070E08DE191E00E945B6B84
:105C600080E290E00E94A8C4FC0188E090E0938369
:105C700082838824839499249A9495828482AA2486
:105C8000AA94B12CB782A68211861086108E50E895
:105C9000D52ED18E63E9E62E68E0F62EF38EE28EE5
:105CA000CBE5D4E0D183C083F0939907E0939807C4
:105CB000CF010E94984C80E290E00E94A8C4FC01B1
:105CC00089E090E09383828395828482B782A68262
:105CD00011861086108ED18EF38EE28ED183C08312
:105CE000F0939707E0939607CF010E94984C66C106
:105CF0008A3009F458C03CF4883009F4A2C08930D5
:105D000009F405C1FBC08B3009F4BEC08C3009F02A
:105D1000F5C089E190E00E94A8C4EC0183E6882EDA
:105D200086E0982E9982888287E090E09B838A8320
:105D3000AA24A394BB24BA94BD82AC82CC24CA9476
:105D4000D12CDF82CE8219861886188ECE010E9451
:105D5000D64137E3E32E34E0F32EF982E882D09384
:105D60009B07C0939A0789E190E00E94A8C4EC01C8
:105D70009982888286E090E09B838A83BD82AC8290
:105D8000DF82CE8219861886188ECE010E94D641F7
:105D9000F982E882D0939D07C0939C071092130F5D
:105DA0001092160FF5C084E290E00E94A8C4FC0196
:105DB000709079136090121388E090E0938382834F
:105DC0008824839499249A9495828482AA24AA94FC
:105DD000B12CB782A68211861086108E83E8582EC9
:105DE000518E93E9C92E98E0D92ED38EC28E27E624
:105DF000E22E24E0F22EF182E082CEE5D3E1D1A3BF
:105E0000C0A362A273A2F0939B07E0939A0784E277
:105E100090E00E94A8C4FC0189E090E09383828313
:105E200095828482B782A68211861086108E518E4A
:105E3000D38EC28EF182E082D1A3C0A362A273A2EC
:105E4000A3C080E290E00E94A8C4FC0188E090E03A
:105E5000938382838824839499249A94958284825C
:105E6000AA24AA94B12CB782A68211861086108E1D
:105E7000AAE0DA2ED18EB3E9EB2EB8E0FB2EF38E3A
:105E8000E28ECFE4D4E065C089E190E00E94A8C42E
:105E9000FC0188E090E093838283CC24C394DD24CA
:105EA000DA94D582C482EE24EA94F12CF782E68259
:105EB00011861086108EC3E4D4E0D183C083F093A2
:105EC0009B07E0939A0789E190E00E94A8C4FC0137
:105ED00089E090E093838283D582C482F782E68250
:105EE00011861086108ED183C083F0939D07E093B6
:105EF0009C071092280F10922B0F4AC089E08093C4
:105F0000BB1269E070E08DE191E00E945B6B80E282
:105F100090E00E94A8C4FC0188E090E09383828313
:105F20008824839499249A9495828482AA24AA949A
:105F3000B12CB782A68211861086108EA0E8DA2EC8
:105F4000D18EB3E9EB2EB8E0FB2EF38EE28ECBE5DB
:105F5000D4E0D183C083F0939B07E0939A0780E25B
:105F600090E00E94A8C4FC0189E090E093838283C2
:105F700095828482B782A68211861086108ED18E79
:105F8000F38EE28ED183C083F0939D07E0939C074C
:105F900080919C0790919D07DC01ED91FC9102801E
:105FA000F381E02D199580919A0790919B07DC0170
:105FB000ED91FC910280F381E02D199580910613FB
:105FC000833039F0823009F06CC08091BB128C3084
:105FD00051F189E190E00E94A8C4EC0183E696E0CB
:105FE0009983888386E090E09B838A8381E09FEF9A
:105FF0009D838C838FEF90E09F838E831986188614
:10600000188ECE010E94D64187E394E0998388835D
:10601000D0939407C0939307CE010E94BF8B109238
:10602000160FC6E029C089E190E00E94A8C4EC01E7
:1060300083E696E09983888384E090E09B838A835B
:1060400081E09FEF9D838C838FEF90E09F838E8311
:1060500019861886188ECE010E94D64187E394E0F7
:1060600099838883D0939407C0939307CE010E94AD
:10607000BF8B10921C0FC4E06091CA127091CB12BA
:106080008C2F0E94EF406091CC127091CD128C2F1A
:106090000E94EB408091CE12E0919307F09194071B
:1060A000808FE091BC128E2FEE0F990BAA0BBB0BC9
:1060B000FC013897E830F10508F0BBC08827E25BA7
:1060C000FE4F8F4F0C9494C484E290E00E94A8C4C9
:1060D000FC018091791328E030E03383228321E0B2
:1060E0003FEF358324832FEF30E0378326831186FB
:1060F0001086108E94E8918F23E938E0338F228F39
:1061000027E634E0318320832EE533E131A320A359
:1061100012A283A31EC080E290E00E94A8C4FC01EA
:1061200088E090E09383828381E09FEF958384836E
:106130008FEF90E09783868311861086108E87E814
:10614000818F83E998E0938F828F8BE594E0918330
:106150008083F093A107E093A00799C080E290E0CC
:106160000E94A8C4FC0188E090E09383828381E0D0
:106170009FEF958384838FEF90E0978386831186CA
:106180001086108E8DE0818F83E998E0938F828F47
:106190008FE494E0DCCF89E190E00E94A8C4FC0188
:1061A00088E090E09383828381E09FEF95838483EE
:1061B0008FEF90E09783868311861086108E83E49C
:1061C00094E091838083F093A107E093A00710925D
:1061D000280F5DC08CE190E00E94A8C4EC0183E62A
:1061E00096E09983888385E090E09B838A8381E0B1
:1061F0009FEF9D838C838FEF90E09F838E83198622
:106200001886188ECE010E94D64187E596E037C0E9
:1062100089E190E00E94A8C4FC01138212821582D9
:1062200014821782168211861086108E8FE194E0F8
:106230008ECF8CE08093BC126CE070E08EE191E038
:106240000E945B6B89E190E00E94A8C4EC0183E6A8
:1062500096E09983888385E090E09B838A8381E040
:106260009FEF9D838C838FEF90E09F838E831986B1
:106270001886188ECE010E94D64187E394E0998358
:106280008883D093A107C093A0071092190F809123
:10629000A0079091A107DC01ED91FC910280F381B0
:1062A000E02D19958091C412843658F4853608F093
:1062B00084E664E6681B8091A0079091A1070E9484
:1062C000954D8091BC128C508230A8F46091C5121B
:1062D0007091C61285E00E9421406091C7127091B2
:1062E000C81285E00E9406408091C912E091A00783
:1062F000F091A107808F2091BD12822F022E000CF9
:10630000990BAA0BBB0BFC013897E830F10508F09C
:1063100089C08827EA5AFE4F8F4F0C9494C484E2B8
:1063200090E00E94A8C4FC018091791329E030E03C
:106330003383228321E03FEF358324832FEF30E046
:106340003783268311861086108E94E8918F23E977
:1063500038E0338F228F27E634E0318320832EE527
:1063600033E131A320A312A283A357C080E290E0BF
:106370000E94A8C4FC0189E090E09383828381E0BD
:106380009FEF958384838FEF90E0978386831186B8
:106390001086108E87E8818F83E998E0938F828F33
:1063A0008BE594E038C080E290E00E94A8C4FC0134
:1063B00089E090E09383828381E09FEF95838483DB
:1063C0008FEF90E09783868311861086108E8DE084
:1063D000818F83E998E0938F828F8FE494E01BC0D4
:1063E00080910613823009F0C9C28091BB128C30B3
:1063F00009F0C4C21FC089E190E00E94A8C4FC015A
:1064000013821282158214821782168211861086D8
:10641000108E8FE194E091838083F093A507E09341
:10642000A4075EC080910613823061F58091BB1293
:106430008C3041F58BE08093BD126BE070E08FE112
:1064400091E00E945B6B89E190E00E94A8C4FC018E
:1064500089E090E09383828381E09FEF958384833A
:106460008FEF90E09783868311861086108E83E4E9
:1064700094E091838083F093A507E093A4071092A2
:106480002B0F2EC08CE08093BD126CE070E08FE18A
:1064900091E00E945B6B89E190E00E94A8C4EC014E
:1064A00083E696E09983888384E090E09B838A83E7
:1064B00081E09FEF9D838C838FEF90E09F838E839D
:1064C00019861886188ECE010E94D64187E394E083
:1064D00099838883D093A507C093A40710921C0FBB
:1064E0008091A4079091A507DC01ED91FC910280B9
:1064F000F381E02D19958091C312843658F48536C6
:1065000008F084E664E6681B8091A4079091A507D3
:106510000E94954D8091BD128C50823000F56091A3
:10652000BE127091BF1284E00E9421406091C0129F
:106530007091C11284E00E9406408091C212E091E5
:10654000A407F091A507808F8091BD128D3039F49A
:106550008091C212E091A613F091A713808F8EE173
:1065600090E00E94A8C4EC01D090D312A090D71262
:10657000B090D8128090D5129090D61283E696E013
:106580009983888383E090E09B838A8381E09FEFF7
:106590009D838C83EE24EA94F12CFF82EE8219868F
:1065A0001886188ECE010E94D6418BE294E0998322
:1065B00088839A8E898EBC8EAB8EDD8ED0933E0FF3
:1065C000C0933D0F6091D9127091DA1283E00E945E
:1065D00021406091DB127091DC1283E00E94064042
:1065E0008091D312E0913D0FF0913E0F808F80910A
:1065F000D3120E94266B80913D0F90913E0FDC01DB
:10660000ED91FC910280F381E02D19958091DE12CD
:106610008823A1F18BE390E00E94A8C4FC01809143
:10662000E8129091E7122091ED123091EE12409114
:10663000EB125091EC126091E9127091EA12A09164
:10664000E312B091E412C091E112D091E212C09035
:10665000DF12D090E01211821082F382E282158262
:106660001482D4A2C3A2D6A3C5A3B0A7A7A372A71E
:1066700061A754A743A736A725A72FC08BE390E0B7
:106680000E94A8C4FC018091E8129091E712209129
:10669000ED123091EE124091EB125091EC1260919C
:1066A000E9127091EA12A091E112B091E212C09148
:1066B000DF12D091E01211821082F382E282158201
:1066C0001482D4A3C3A3B6A3A5A370A767A352A79C
:1066D00041A734A723A7F6A6E5A623E938E030AB07
:1066E00027A72EE533E132AB21AB93AB84ABF0931C
:1066F0002207E0932107C0912107D09122072FA103
:1067000038A54BA15CA18DA19EA1421753071CF493
:10671000821793077CF0281739071CF4481759078C
:1067200064F0241735075CF48417950744F4142F9C
:10673000052F05C0122F032F02C0182F092F1F820B
:106740001E82188709871B861A861D861C861E874F
:106750000F87198A188A2DA53EA549A55AA58BA58C
:106760009CA5421753071CF4821793077CF0281747
:1067700039071CF44817590764F0241735075CF4EF
:106780008417950744F4142F052F05C0122F032FEB
:1067900002C0182F092F1B8A1A8A1C8B0D8B1F8A87
:1067A0001E8A198E188E1A8F0B8F1D8E1C8E1AAE94
:1067B00019AE18A28BA9813069F08230E9F08111FD
:1067C00083C061E08CE20E94D04A10922D011092A9
:1067D0002C017AC061E08CE20E94D04A10922D0117
:1067E00010922C0161E088E00E94D04A60E070E0E5
:1067F00088E00E940C4B68C0E9A9FAA980819181C8
:10680000A281B38181159649A105B10509F457C04C
:1068100040E056E960E070E08FA598A90E941E81D3
:1068200064E170E080E090E00E94174CE9A9FAA9C9
:1068300080819181A281B38181152BE49207A1050A
:10684000B105E9F068F4803629E09207A105B105A9
:10685000A1F080389542A105B105C1F442E012C013
:10686000811521EE9207A105B10559F08115924CD1
:10687000A140B10559F445E005C041E003C043E043
:1068800001C046E06FE0CE010E94893C8FA598A927
:10689000DC01ED91FC910680F781E02D1995E9A9C5
:1068A000FAA940815181628173818FA598A90E94C4
:1068B0001E8164E170E080E090E00E94174C4AE0A5
:1068C0006EE0CE010E94893C8091E8128093EC0733
:1068D0008091280F8823F9F089E190E00E94A8C4F4
:1068E000FC0188E090E093838283158214828FEF0D
:1068F00093E0978386838FEF91E091878087108E56
:1069000083E494E091838083F093270FE093260F34
:10691000CF010E94898C80912B0F882309F478C0C5
:1069200089E190E00E94A8C4FC0189E090E0938393
:106930008283158214828FEF93E0978386838FEF93
:1069400091E091878087108E83E494E09183808327
:10695000F0932A0FE093290FCF01DF91CF911F9180
:106960000F91FF90EF90DF90CF90BF90AF909F90EE
:106970008F907F906F905F900C94898C2C3009F4ED
:106980008ACD8CE190E00E94A8C4EC0193E6692EC8
:1069900096E0792E7982688224E0822E912C9B8267
:1069A0008A82AA24A394BB24BA94BD82AC82CC244C
:1069B000CA94D12CDF82CE8219861886188ECE0119
:1069C0000E94D64157E5E52E56E0F52EF982E88281
:1069D000D093A507C093A4078CE190E00E94A8C4BF
:1069E000EC01798268829B828A82BD82AC82DF82DE
:1069F000CE8219861886188E0E94D641F982E882C6
:106A0000D093A713C093A613CE010E945F8C66CDCE
:106A1000DF91CF911F910F91FF90EF90DF90CF907A
:106A2000BF90AF909F908F907F906F905F900895F0
:106A30002F923F924F925F926F927F928F929F928E
:106A4000AF92BF92CF92DF92EF92FF920F931F937C
:106A5000CF93DF93CDB7DEB7CE5AD1090FB6F894F6
:106A6000DEBF0FBECDBFCDB6DEB6C455DF4F188238
:106A7000CC5AD040C555DF4F1882CB5AD0408091B8
:106A8000AA0E8B3709F4E8C180F4873709F4D7C21E
:106A900038F48F3109F440C5863709F4E0C102C6E5
:106AA0008937B9F008F4DAC234C0803809F472C406
:106AB00038F48C3709F4E1C28E3709F42DC3F2C5DE
:106AC000823809F408C508F418C5833809F4E6C407
:106AD000E9C50E94E9430E9476842B013C010E9493
:106AE00018A1029709F423C50E947684DC01CB012A
:106AF00084199509A609B70980329340A105B1050B
:106B000008F015C50E9468640E94E9430E94579FDF
:106B1000E6CF0E9418A1029729F060E084E80E9465
:106B20000BA08BC18091EE0B823031F0833039F4B1
:106B300082E08093720F03C081E08093DA0E81E0DF
:106B40008093B40E8E0104551F4F2FE0AE014057C5
:106B50005F4F68E871E90E94949F0E94EBA0893022
:106B600058F0015011092FE0AE014F575F4F68E810
:106B700072E981E00E94949F1092B30E772473947F
:106B80000E9401A1882309F43DC1198222961FAEFB
:106B900022971091B30E11110EC0BE0160577F4FA6
:106BA000CE018F5B9F4F0E94C6C6C455DF4F088140
:106BB000CC5AD04011C0113071F4BE016F577F4FD5
:106BC000CE018F5B9F4F0E94C6C6C555DF4F08811F
:106BD000CB5AD04001C000E0ADB6BEB68091EA0B02
:106BE000EDB7FEB722E0829FE019F10911240FB63C
:106BF000F894FEBF0FBEEDBF8DB79EB701967C0126
:106C000065E876E0CE018B559F4F0E94FE4680914D
:106C1000EE0B823089F0833061F1813009F0A1C040
:106C20004091EA0B50E0B7018091C1149091C214D9
:106C30000E944C9E10E039C02091EA0B30E05FB713
:106C4000F89440E0842F90E08217930774F4880F43
:106C5000991FF701E80FF91FDC01A754B14F8D917F
:106C60009C91918380834F5FEDCF5FBF1092D90ECF
:106C70001CC02091EA0B30E05FB7F89440E0842F0D
:106C800090E08217930774F4880F991FF701E80FBB
:106C9000F91FDC01A557B04F8D919C9191838083A2
:106CA0004F5FEDCF5FBF1092BE146DE270E0CE017A
:106CB0008B559F4F0E9401462091EA0B293048F0E6
:106CC000112321F0113021F418E004C028E001C0A4
:106CD00020E010E0121758F5F701E10FF11DE10F68
:106CE000F11D608171814AE0CE0181569F4FC355ED
:106CF000DF4F2883CD5AD0400E94A746BE0161567F
:106D00007F4FCE018B559F4F0E942846CE01815662
:106D10009F4F0E94A246CE018B559F4F0E948D6EC1
:106D20001F5FC355DF4F2881CD5AD040D3CF40E4F9
:106D300050E0BE016F5F7F4FCE018B559F4F0E9489
:106D4000856EC755DF4F1881C95AD040CE018B558B
:106D50009F4F0E94A2460FB6F894BEBE0FBEADBEB6
:106D60000BC0CE018B559F4F0E94A2460FB6F894E0
:106D7000BEBE0FBEADBE10E0BE016F5F7F4FCE0145
:106D80008F5B9F4F0E94C6C6010F10E0E1E4F0E068
:106D9000EC0FFD1FE00FF11F1082BE016F5B7F4FF4
:106DA0008091A2149091A3140E947548B801CE015D
:106DB0008F5B9F4F0E94749FBC018091A2149091A1
:106DC000A3140E944A6C6AE08091A2149091A314CB
:106DD0000E9491478091A2149091A314DC01ED913F
:106DE000FC910680F781E02D19950E94EBA0893077
:106DF00048F08091B30E811103C07092B30E02C0AF
:106E00001092B30E0E94E9430E94579F0E94158D75
:106E100081110EDE8091A90E81110FC08091B40EF8
:106E2000882359F08091A414811107C08091A70E86
:106E30009091A80E0A970CF4A3CE8091EE0B8230AD
:106E400039F0833009F02EC481E08093720F2AC498
:106E500081E08093DA0E26C41092B40E5AC31091CA
:106E6000AD0E8FEF810F853028F060E089E80E9439
:106E70000BA018C4133079F018F41230F9F004C0E4
:106E8000143079F0153099F040E6442E49E0542E44
:106E9000612C712C19C0412C3BE4532E612C712CB8
:106EA00013C0412C26E9522E612C712C0DC0412CAF
:106EB00092EC592E66246394712C06C080E8482E0B
:106EC00085E2582E612C712C00E0E12EF12C570147
:106ED000BFE8AB0EB11C1501E89427F83324E6E9AE
:106EE000EE0EF11CE894E7F8FF24023091F018F45C
:106EF000013051F004C0033089F00430A1F040E6C5
:106F000059E060E070E013C040E855E260E070E0F6
:106F10000EC040E05BE460E070E009C040E056E98C
:106F200060E070E004C040E052EC61E070E083E9B2
:106F300098E00E941E8183E998E00E9411450E941A
:106F400076844B015C01F2E38F0E911CA11CB11CF5
:106F50000E94179F0E947684681579058A059B0513
:106F6000B8F360E870E083E998E00E94068F6FE074
:106F700070E083E998E00E94068F612F83E998E032
:106F80000E94CB44B10183E998E00E94068F0E94E1
:106F900076844B015C012AE0820E911CA11CB11C7D
:106FA0000E94179F0E947684681579058A059B05C3
:106FB000B8F367E870E083E998E00E94068F6FE01D
:106FC00070E083E998E00E94068F612F83E998E0E2
:106FD0000E94CB44B70183E998E00E94068F83E9C1
:106FE00098E00E9411450E9476844B015C013EE5C9
:106FF000830E31E0931EA11CB11C0E94179F0E94BA
:107000007684681579058A059B05B8F30F5F05300E
:1070100009F06BCFB301A20183E998E00E941E81C1
:1070200040925E1350925F136092601370926113EE
:10703000B301A20180EC91E00E94C06E6AC283E0BD
:1070400090E00E94A8C42AE0DC012C9323E938E0F8
:1070500012963C932E9311976AE00CC083E090E067
:107060000E94A8C42DE0FC01208323E938E032838C
:1070700021836DE00E9492664CC24091AD0E50910A
:10708000AE0E0091AF0E1091B00E6091AB0E7091EC
:10709000AC0ECE010196C355DF4F4883CD5AD04088
:1070A000C255DF4F5883CE5AD0400E94CF91C3556E
:1070B000DF4F4881CD5AD040C255DF4F5881CE5A5C
:1070C000D040892BE9F08D81873050F4853080F4F1
:1070D0008130B0F0642F8B819C810E94B56C0DC013
:1070E000893070F4B8018B819C810E94C06E05C00C
:1070F000BA018B819C810E945B6B0E9486A004C0B8
:1071000061E085E80E940BA08091A60E8111CAC2A1
:1071100081E08093A60EC6C2B090AB0EE090AC0E9C
:10712000C156DF4F1882CF59D04065E876E0CE01D6
:107130008F579F4F0E94FE466B2D7E2DCE018057AC
:107140009F4F0E94CF91892B09F4BEC0CC56DF4FD0
:10715000E881C459D0404E2F50E0FA013197E83011
:10716000F10508F0B1C08827E25AFE4F8F4F0C940A
:1071700094C4CE56DF4F88819981C259D0400E9475
:1071800058C24AE0682FCE0101960E94D2461BC029
:10719000CE56DF4F88819981C259D0400E9458C293
:1071A000682F880F770B4AE00AC0CE56DF4F8881E0
:1071B0009981C259D0400E9465C24AE0BC01CE010B
:1071C00001960E94A746BE016F5F7F4FCE018F5789
:1071D0009F4F0E94C845CE01019663C0CE56DF4F37
:1071E00088819981C259D0400E9465C223961FAE02
:1071F0001EAE239725961FAE1EAE259727961FAE6F
:107200001EAE27974AE0BE016F5F7F4F0E9406C106
:1072100035C0CE56DF4F88819981C259D0400E9437
:1072200060C223961FAE1EAE239725961FAE1EAEDC
:10723000259727961FAE1EAE27972AE0AE014F5F17
:107240005F4F0E94CDC01AC0CE56DF4F8881998112
:10725000C259D0400E9460C223961FAE1EAE239733
:1072600025961FAE1EAE259727961FAE1EAE2797FA
:107270002AE0AE014F5F5F4F0E94DBC0BE016F5F2F
:107280007F4FCE018F5B9F4F0E948246BE016F5B96
:107290007F4FCE018F579F4F0E94C845CE018F5B15
:1072A0009F4F0E94A2464FE050E0BE016F5B7F4FB0
:1072B000CE018F579F4F0E94856ECB57DF4FF880CE
:1072C000C558D04011E002C0F12C10E0CE018F571C
:1072D0009F4F0E94A246112309F4C7CD8E0101568B
:1072E0001F4F20E4AE014F5F5F4F68E87B2D8E2D6E
:1072F0000E94949FBE016F5B7F4FCE0101960E945A
:10730000C6C6C156DF4F8881CF59D040F80E81E004
:107310008F0DC156DF4F8883CF59D040E1E0F0E0B8
:10732000EC0FFD1FEF0DF11D9CE79083E1E0F0E015
:10733000EC0FFD1FE80FF11D1082BE016F5F7F4F44
:107340008091A2149091A3140E947548C156DF4FFA
:107350006881CF59D04070E0CE0101960E94749FA1
:10736000BC018091A2149091A3140E944A6C6AE01F
:107370008091A2149091A3140E9491478091A2142D
:107380009091A314DC01ED91FC910680F781E02D32
:10739000199588C18091AB0E9091AC0E8038910503
:1073A00009F080C18E0100571F4F20E4AE014F5FEE
:1073B0005F4F68E870E880E00E94949F6BE676E09B
:1073C000CE018F579F4F0E94FE46CE018F579F4F91
:1073D0000E948D6EC057DF4F2881C059D040CB57D7
:1073E000DF4F88819981C558D040820F911DC057C9
:1073F000DF4F8883C059D04022961FAE22974FE0BE
:1074000050E0BE016F5B7F4FCE018F579F4F0E94B0
:10741000626EBE016F5B7F4FCE0101960E94C6C6B1
:10742000C057DF4F8881C059D040E1E0F0E0EC0F59
:10743000FD1FE80FF11D1082BE016F5F7F4F80912D
:10744000A2149091A3140E947548C057DF4F688121
:10745000C059D04070E0CE0101960E94749FBC01DB
:107460008091A2149091A3140E944A6C6AE08091CA
:10747000A2149091A3140E9491478091A21490911C
:10748000A314DC01ED91FC910680F781E02D1995A4
:10749000CE018F579F4F0E94A24604C18091AB0E30
:1074A0009091AC0E8338910509F0FCC08E01005715
:1074B0001F4F20E4AE014F5F5F4F68E873E880E044
:1074C0000E94949F4AE06091A50ECE018F579F4F76
:1074D0000E94D2467ACF8091AB0E9091AC0E82384A
:1074E000910509F0DFC08E0100571F4F20E4AE0167
:1074F0004F5F5F4F68E872E85ECF8091AB0E90916E
:10750000AC0E8138910509F0CDC08091B40E811187
:10751000C9C00E9486A0C6C08091AB0E9091AC0EEF
:107520004F9709F0BFC081E08093A90EBBC00E94B5
:1075300018A1029719F060E084E899CC8091ED0BD6
:10754000811102C00E94CF6C0E94EBA0F82E65E86A
:1075500076E0CE0180579F4F0E94FE46C156DF4F16
:107560001882CF59D0408E0101561F4F20E4AE0142
:107570004F5F5F4F68E879E780E00E94949FCF57A4
:10758000DF4F19821882C158D040CD57DF4F198282
:107590001882C358D040CB57DF4F19821882C55884
:1075A000D0406F2D70E080E090E02AE0AE014F5BAC
:1075B0005F4F0E94CDC0BE016F5B7F4FCE018F57E2
:1075C0009F4F0E948246BE016F577F4FCE0180576A
:1075D0009F4F0E94C845CE018F579F4F0E94A246E1
:1075E0004FE050E0BE016F5B7F4FCE0180579F4F51
:1075F0000E94626ECC56DF4F1881C459D040BE0144
:107600006F5B7F4FCE0101960E94C6C6C156DF4F09
:107610008881CF59D040810F91E0980FC156DF4F3C
:107620009883CF59D040E1E0F0E0EC0FFD1FE80F68
:10763000F11D8CE78083E1E0F0E0EC0FFD1FE90F26
:10764000F11D1082BE016F5F7F4F8091A214909157
:10765000A3140E947548C156DF4F6881CF59D040AE
:1076600070E0CE0101960E94749FBC018091A2142B
:107670009091A3140E944A6C6AE08091A2149091A8
:10768000A3140E9491478091A2149091A314DC014D
:10769000ED91FC910680F781E02D1995CE01805780
:1076A0009F4FF9CE0FB6F894DEBE0FBECDBEC255C9
:1076B000DF4F0FB6F894DEBF0FBECDBFDF91CF9185
:1076C0001F910F91FF90EF90DF90CF90BF90AF9000
:1076D0009F908F907F906F905F904F903F902F90F2
:1076E0000895FC0182810895482F50E095E1899F1B
:1076F000F0011124E452FF4E218132818085918571
:10770000280F391F838194818217930728F0858180
:10771000968128173907E8F485E1849FF001859F59
:10772000F00D1124E452FF4E858196812817390708
:1077300028F52581368185E1849FF001859FF00D34
:107740001124E452FF4E8285823019F4118610868E
:10775000128685E1849FF001859FF00D1124E4528B
:10776000FF4E328321838091840090918500280F01
:10777000391F309389002093880008958381948174
:1077800082179307C0F623813481D5CF62E30C942E
:10779000E68961E30C94E68960E30C94E68964E58C
:1077A0000C94E6896FE20C94E6896DE20C94E6890C
:1077B0006CE20C94E68977FF03C0719561957109BD
:1077C00020E0462F6EE20C94A089462F20E06DE465
:1077D0000C94A089FC016283611105C020E040E0A7
:1077E0006BE40C94A089089577FF03C071956195AF
:1077F000710920E0462F6BE40C94A0894F925F92B0
:107800006F927F928F929F92AF92BF92CF92DF92B0
:10781000EF92FF920F931F93CF93DF936C01A4EC31
:10782000CA1AADEFDA0AD601ED91FC917E970CF001
:107830005DC0FC01E858FF4F812C912CA191B191C2
:10784000AB2B21F42115310549F450C0BFEF8B1A41
:107850009B0AAEE18A16910489F748C0EC015401F5
:10786000AA0CBB1CAA0CBB1CAC0EBD1EF501EC5433
:10787000FF4F40835183628373837401EE0CFF1CBE
:10788000EC0EFD1EF701E858FF4F31832083EC54C6
:10789000FF4F11830083BE01680D791DFB01EC557C
:1078A000FE4F81E080830E947684F50160837183BE
:1078B00082839383C65CDD4F88819981F701E25012
:1078C000FE4F91838083D6012D913C9111972F5FBC
:1078D0003F4F2D933C939C012F5F3F4F1216130691
:1078E00014F021E030E03983288302C08FEF9FEF4E
:1078F000DF91CF911F910F91FF90EF90DF90CF908C
:10790000BF90AF909F908F907F906F905F904F90BF
:1079100008950F931F93CF93DF938C01C62FD42F1D
:1079200065E870E0DC019F968D919C91D0970E9454
:10793000068FF80187A590A9DC01ED91FC910190DB
:10794000F081E02D6C2F1995F80187A590A9DC0135
:10795000ED91FC910190F081E02D6D2F19952C2F68
:1079600030E0B9016B577F4F6D0F711D6F7777272F
:10797000F80187A590A9DF91CF911F910F910C94E9
:10798000068F262F2B7FA1F49A014F3F510519F046
:1079900014F02FEF30E0A90141302FEF520714F41B
:1079A00041E05FEF57FF03C0519541955109B1CFB9
:1079B0000895CF93DF93EC0189AD9AAD892B11F037
:1079C0001AAE19AECE010E94F6808BA9813029F043
:1079D000823069F0811117C005C060E070E088E076
:1079E0000E940C4B10922D0110922C0108C040E017
:1079F00064E0CE018EDF40E060E0CE018ADF1AA2B3
:107A000019A21F8E1E8E0E9476846DAB7EAB8FAB4B
:107A100098AFDF91CF9108958F929F92AF92BF92CE
:107A2000CF92DF92EF92FF920F931F93DC01149697
:107A30008D919C9115975696CD90DC90579768172D
:107A4000790709F455C09096FC9090974C01092E47
:107A5000000CAA08BB088B01072E000C220B330B6D
:107A6000861797073CF41296ED91FC911397FF202F
:107A700031F014C0ED91FC911197FF2079F00D2C9D
:107A8000000CEE08FF08A9019801281939094A09D4
:107A90005B0954966D917C9155970EC00D2C000C8E
:107AA000EE08FF08A9019801281939094A095B095C
:107AB00052966D917C915397CB01770FAA0BBB0B1C
:107AC000BC01CD016C197D098E099F090E945EC41D
:107AD0008F01FF0F220B330BA901980128193909D7
:107AE0004A095B090E9478C2C20ED31EE41EF51E2D
:107AF000C6011F910F91FF90EF90DF90CF90BF9044
:107B0000AF909F908F9008958F929F92AF92BF9267
:107B1000CF92DF92EF92FF920F931F93DC011496A6
:107B20008D919C9115971A96CD90DC901B976817B4
:107B3000790709F455C09096FC9090974C01092E56
:107B4000000CAA08BB088B01072E000C220B330B7C
:107B5000861797073CF41296ED91FC911397FF203E
:107B600031F014C0ED91FC911197FF2079F00D2CAC
:107B7000000CEE08FF08A9019801281939094A09E3
:107B80005B0918966D917C9119970EC00D2C000C15
:107B9000EE08FF08A9019801281939094A095B096B
:107BA00016966D917C911797CB01770FAA0BBB0BA3
:107BB000BC01CD016C197D098E099F090E945EC42C
:107BC0008F01FF0F220B330BA901980128193909E6
:107BD0004A095B090E9478C2C20ED31EE41EF51E3C
:107BE000C6011F910F91FF90EF90DF90CF90BF9053
:107BF000AF909F908F900895EF92FF920F931F93F5
:107C0000CF93DF93EC0189AD9AAD892B11F01AAEB9
:107C100019AE8BA98130B1F0823059F1811143C086
:107C2000CB0177FF03C0919581959109BC01CE01ED
:107C30006BDF90932D0180932C019AA389A39F8FD2
:107C40008E8F31C08B0177FF03C01195019511090B
:107C5000B801CE0159DF7C01B801CE01DDDE8C0117
:107C6000B70188E00E940C4B10932D0100932C016A
:107C700016C08B0177FF03C0119501951109B8015A
:107C8000CE0142DF7C01B801CE01C6DE8C01A70126
:107C900064E0CE0176DEA80160E0CE0172DEFAA2D9
:107CA000E9A21F8F0E8F0E9476846DAB7EAB8FABE7
:107CB00098AFDF91CF911F910F91FF90EF900895B2
:107CC000CF93DF93EC0189AD9AAD892B11F01AAEF9
:107CD00019AE2FA138A58DA19EA19F838E833987D0
:107CE00028879B878A872DA53EA58BA59CA59B8B66
:107CF0008A8B3D8B2C8B9F8B8E8B60E070E0CE014E
:107D00007BDF0E9476846DAB7EAB8FAB98AFDF914B
:107D1000CF910895CF93DF93EC0189AD9AAD892B74
:107D200011F01AAE19AE2FA138A58BA19CA19F838B
:107D30008E83398728879B878A872DA53EA589A5AD
:107D40009AA59B8B8A8B3D8B2C8B9F8B8E8B60E0B7
:107D500070E0CE0151DF0E9476846DAB7EAB8FABBD
:107D600098AFDF91CF910895DC01A250BE4F20E083
:107D700030E04D915D914617570739F4280F391FB0
:107D8000F901EC55FE4F808108952F5F3F4F2E3152
:107D9000310579F780E00895CF93DF93EC01C45C5F
:107DA000DD4FA881B981109709F442C0FC01E2506F
:107DB000FE4F20E030E0419151914617570799F569
:107DC000A901440F551F480F591FFA01E858FF4FEA
:107DD00060817181672B61F111821082FC01E20FD9
:107DE000F31FEC55FE4F1082FA01EE53FE4F118245
:107DF0001082235D3F4F220F331F220F331FFC01E0
:107E0000E20FF31F1082118212821382FA01E859E5
:107E1000FE4F11821082EA56FF4F11821082119795
:107E2000B983A88305C02F5F3F4F2E31310519F666
:107E3000DF91CF9108950F931F9301E010E0DEDCF6
:107E40001F910F9108950F931F9300E010E0D6DC6F
:107E50001F910F9108952F923F924F925F926F92D0
:107E60007F928F929F92AF92BF92CF92DF92EF92CA
:107E7000FF920F931F93CF93DF9300D000D0CDB725
:107E8000DEB78C010E94768498012E533E4F3C83CE
:107E90002B831E830D83D801AC55BE4FBA83A983B3
:107EA0001801B2E02B1ABEEF3B0AF901AA24A394F1
:107EB000B12C32E0832E912C118210829F012A5422
:107EC0003140D9012D913C91232B09F44DC0AD8156
:107ED000BE812D913D914D915C9113977D01B4EB45
:107EE000EB0EF11CD701CD90DD90ED90FC902B01B5
:107EF0003C01421A530A640A750A4C145D046E046C
:107F00007F0490F1C20ED31EE41EF51EAD81BE812A
:107F1000CD92DD92ED92FC921397A981BA812C91BA
:107F2000222311F19F0126593109D9012D913C914C
:107F30002115310519F4B182A08216C07F01BAE57E
:107F4000EB1AF108D7014D915C9111974217530735
:107F50005CF4B182A0824F5F5F4F4D935C934217F8
:107F6000530714F09182808232962D813E812C5FDE
:107F70003F4F3E832D83A981BA811196BA83A9838D
:107F8000E215F30509F098CFEB81FC818191919185
:107F9000FC83EB838130910599F00297C9F4EB8162
:107FA000FC81EC54F1400190F081E02D1995AB81FA
:107FB000BC81DA966D917C91DB97C801EDDE08C03B
:107FC000EB81FC81EC54F1400190F081E02D19959A
:107FD0002B813C8122153305B9F626960FB6F8940D
:107FE000DEBF0FBECDBFDF91CF911F910F91FF90EC
:107FF000EF90DF90CF90BF90AF909F908F907F9049
:108000006F905F904F903F902F9008956E3E22E0CA
:10801000720738F06B3C98E0790728F06AEC78E05A
:1080200002C06EEE72E0660F771F9FB7F89425E1ED
:10803000829FF0011124E452FF4E748363839FBF3B
:1080400008956E3E22E0720738F06B3C98E07907A5
:1080500028F06AEC78E002C06EEE72E0660F771FDF
:108060009FB7F89425E1829FF0011124E452FF4E5E
:10807000768365839FBF0895660F771F282F30E0B2
:1080800095E1899FF0011124E452FF4E858196818C
:108090006817790718F46581768107C08381948118
:1080A0008617970710F4638174818FB7F89495E170
:1080B000929FF001939FF00D1124E452FF4E7283C2
:1080C00061838FBF0895982F8FB7F89425E1929F11
:1080D000F0011124E452FF4E21E027838FBF41B10C
:1080E00021E030E0B90102C0660F771F9A95E2F7F0
:1080F000CB01842B81B908958A3058F49FB7F89446
:1081000025E1829FF0011124E452FF4E1186108672
:108110009FBF08951F93CF93DF9325E1829FC001F6
:108120001124EC01C452DF4E8A8581110FC01FB7A4
:10813000F89481E08A8789899A899A8389830E9441
:1081400076846B877C878D879E871FBFDF91CF9159
:108150001F910895CF93DF938A30D0F56233710574
:1081600038F061369DE6790728F060E67DE602C0CA
:1081700062E370E0D42FC82F80E090E00E9433C10A
:1081800020E030E04AE754E40E943AC320E030E0C7
:108190004CE852E40E9494C19B01AC0160E070E0A5
:1081A0008AEF94E40E943AC30E94A2C39B01DD239C
:1081B00021F022273327261B370B8FB7F89495E140
:1081C000C99FF0011124E452FF4E318720878FBFF1
:1081D000DF91CF9108958A3008F418CF08958A303E
:1081E00008F42FCF08958A3058F495E1899FF00163
:1081F0001124E452FF4E81819281969587950895CE
:1082000080E090E008958A3008F436CF08951F92F8
:108210000F920FB60F9211240BB60F920F931F936C
:108220002F933F934F935F936F937F938F939F937E
:10823000AF93BF93CF93EF93FF938091FC0E893060
:1082400048F01092FC0E80918B11882399F0809158
:1082500084110DC0E091FC0EE15025E1E29FF00198
:108260001124E452FF4E8781882321F0808192B14E
:10827000892782B9E091FC0E85E1E89FF001112485
:10828000E452FF4E8781882321F0808192B1892BAF
:1082900082B9E091FC0EC5E1CE9FF0011124E452B9
:1082A000FF4E80859185892B09F04DC0E091FC0E31
:1082B000CE9FF0011124E452FF4E8285813009F0F7
:1082C00060C00E947684E091FC0ECE9FF0011124E4
:1082D000E452FF4E0385148525853685E091FC0E1A
:1082E000CE9FF0011124E452FF4E0784F089E02D67
:1082F000AB01BC01401B510B620B730BCF01A0E023
:10830000B0E084179507A607B707D8F5E091FC0EF3
:10831000A091FC0ECA9FD0011124A452BF4E5396C7
:108320008D919C915497CE9FF0011124E452FF4E01
:1083300091878087E091FC0ECE9FF0011124E452DA
:10834000FF4E82E082878091FC0ECED98091FC0E98
:108350008F5F8093FC0EFF91EF91CF91BF91AF9112
:108360009F918F917F916F915F914F913F912F914D
:108370001F910F910F900BBE0F900FBE0F901F908B
:108380001895E091FC0E809184009091850025E184
:10839000E29FF0011124E452FF4E21813281820FCD
:1083A000931F9093890080938800D0CF1F93CF9321
:1083B000DF938091FB0E811173C01092FC0E9FB76A
:1083C000F89485E128EB3BE04CED55E064E971E180
:1083D000A1E0B0E0E091FC0EE93008F052C0E0917D
:1083E000FC0E8E9FF0011124E452FF4E3283218354
:1083F000E091FC0E8E9FF0011124E452FF4E568353
:108400004583E091FC0E8E9FF0011124E452FF4E53
:1084100074836383E091FC0EF091FC0EED0101C0CA
:10842000CC0FFA95EAF78E9FF0011124E452FF4E2B
:10843000C083E091FC0E8E9FF0011124E452FF4EA8
:108440001782E091FC0E8E9FF0011124E452FF4E42
:1084500011861086E091FC0E8E9FF0011124E452EB
:10846000FF4E1286E091FC0E8E9FF0011124E45223
:10847000FF4E148A138AE091FC0EEF5FE093FC0E2E
:10848000A9CF9FBF8FB7F89420EA3FE030938611C1
:1084900020938511109284118FBF81E08093FB0E91
:1084A000DF91CF911F9108950F931F93CF93DF9387
:1084B0008C01C62FD42FDC0111968D919C911297BF
:1084C000DC01ED91FC910190F081E02DD8016C91DF
:1084D0001995F80181819281DC01ED91FC91019067
:1084E000F081E02D6C2F1995F80181819281DC01DA
:1084F000ED91FC910190F081E02D6D2F1995F8011F
:1085000080816C2F70E0680F711D6D0F711D6F778A
:10851000772781819281DF91CF911F910F910C94E8
:10852000068F0F931F93CF93DF938C01C62FD42F09
:10853000DC0111968D919C911297DC01ED91FC91DB
:108540000190F081E02DD8016C911995F80181819D
:108550009281DC01ED91FC910190F081E02D6C2F76
:108560001995F80181819281DC01ED91FC910190D6
:10857000F081E02D6D2F1995F80180816C2F70E04E
:10858000680F711D6D0F711D6F7777278181928143
:10859000DF91CF911F910F910C94068F4F925F92B4
:1085A0006F927F92AF92BF92CF92DF92EF92FF9243
:1085B0001F93CF93DF93DD24D39445E0C42EC2E014
:1085C000D0E053E0E52EF12CAA24A394B12C8091A5
:1085D000DF0E9091E00EDC01ED91FC910084F185BD
:1085E000E02D1995892B09F4D1C0109130018091AB
:1085F000DF0E9091E00EDC01ED91FC910284F38599
:10860000E02D199596B3B39A20918400309185009E
:108610002059384E30938D0020938C00212F2C71DF
:1086200019F01092FA0E2AC093FB992790F9E09165
:10863000FA0EE11116C0992351F28F3041F6D09213
:10864000FA0E8093E10E8091DD0E9091DE0E892B63
:1086500009F0BDCFB092DE0EA092DD0E1092DC0EBE
:10866000B6CF992381F01092FA0E1092DC0E809111
:10867000DD0E9091DE0E029709F0A9CFF092DE0E8A
:10868000E092DD0EA4CF91E09E0F9093FA0EF0E001
:10869000EF51F14F8083993109F099CF811173C067
:1086A0008091F80E82FF05C0F092DE0EE092DD0EA2
:1086B0006AC083FDF9CF8091DD0E9091DE0E0197A7
:1086C00061F48091DC0E8F5F8093DC0E843058F073
:1086D000D093DE0EC093DD0E06C0D093DE0EC093A5
:1086E000DD0E1092DC0E8091DB0E8F5F8093DB0E2F
:1086F0009091DA0E981708F044C0D092D90EA9EBE9
:10870000BEE0E2EEFEE040E050E0BA0110E0CF0152
:10871000FC011B3098F401964080512C612C712C87
:10872000012E04C0440C551C661C771C0A94D2F719
:108730004429552966297729185FEACF9A013770AD
:10874000205E3340C29EC001C39E900D112497FD50
:10875000079623E0959587952A95E1F784529A4FDD
:108760008D939D931B503BE0769567955795479564
:108770003A95D1F78EE0A93DB80749F61092DB0E85
:1087800002C01092D90E1092FA0E21CFDF91CF9134
:108790001F91FF90EF90DF90CF90BF90AF907F90B0
:1087A0006F905F904F9008958091EE0B833031F47D
:1087B0008091B70E9091B80E0C94559908958091C0
:1087C000EE0B823029F48091B50E9091B60EE6CE74
:1087D0000895F5DFE9CF1092B5101092BF101092F6
:1087E000C9101092D31010925D1080E090E0FC014F
:1087F000E05AFF4E1182079684359105C1F708951E
:108800000895CF92DF92EF92FF920F931F93CF9331
:10881000DF936C017A018B01C0E0D0E0CE15DF055B
:1088200089F0D8016D918D01D601ED91FC910190F7
:10883000F081E02DC6011995892B11F47E0102C04B
:108840002196ECCFC701DF91CF911F910F91FF903F
:10885000EF90DF90CF900895FC01A089B1898C91B1
:10886000A689B78982FD0FC09C91818D8F5F8F7320
:10887000228D821749F0218DDF01A20FB11D5D9677
:108880009C93818F08958C910895089580E090E0E5
:108890000895FC01538D448D252F30E0842F90E006
:1088A000821B930B541710F0CF96089501970895EB
:1088B000FC01918D828D981761F0828DDF01A80FE8
:1088C000B11D5D968C91928D9F5F9F73928F90E00A
:1088D00008958FEF9FEF0895FC01918D828D981779
:1088E00031F0828DE80FF11D858D90E008958FEFB6
:1088F0009FEF0895FC01918D228D892F90E0805C7F
:108900009F4F821B91098F739927089586EF97E0F7
:10891000F1DF21E0892B09F420E0822F089583E91B
:1089200098E0E8DF21E0892B09F420E0822F089508
:1089300080E399E0DFDF21E0892B09F420E0822F3A
:1089400008958DEC99E0D6DF21E0892B09F420E031
:10895000822F0895FC01848DDF01A80FB11DA35A59
:10896000BF4F2C91848D90E001968F739927848F4F
:10897000A689B7892C93A089B1898C9180648C9346
:10898000938D848D981306C00288F389E02D808131
:108990008F7D80830895EF92FF920F931F93CF9363
:1089A000DF93EC0181E0888F9B8D8C8D981305C03F
:1089B000E889F989808185FD23C0F62E0B8D10E0B2
:1089C0000F5F1F4F0F731127E02E8C8DE8120BC025
:1089D0000FB607FCFACFE889F989808185FFF5CFCA
:1089E000CE01B8DFF2CF8B8DFE01E80FF11DE35A07
:1089F000FF4FF0820B8FEA89FB898081806207C07C
:108A0000EE89FF896083E889F989808180648083A9
:108A100081E090E0DF91CF911F910F91FF90EF9057
:108A20000895CF93DF93EC01888D8823C1F0EA8904
:108A3000FB89808185FD05C0A889B9898C9186FD57
:108A40000EC00FB607FCF5CF808185FFF2CFA88955
:108A5000B9898C9185FFEDCFCE017CDFE8CFDF9126
:108A6000CF91089580E090E0892B19F06ADF8111A1
:108A700016C080E090E0892B19F05ADF811112C0F6
:108A800080E090E0892B19F04ADF81110EC080E070
:108A900090E0892B79F03ADF81110AC008950E9495
:108AA0000000E7CF0E940000EBCF0E940000EFCF54
:108AB0000C940000089590E0FC013197E231F1053B
:108AC00008F04EC08827EA59FE4F8F4F0C9494C48B
:108AD000809180008F7703C0809180008F7D80938C
:108AE0008000089580918000877FF9CF84B58F77CB
:108AF00002C084B58F7D84BD08958091B0008F77CA
:108B000003C08091B0008F7D8093B0000895809164
:108B100090008F7707C0809190008F7D03C0809177
:108B20009000877F8093900008958091A0008F77B8
:108B300007C08091A0008F7D03C08091A000877F37
:108B40008093A0000895809120018F7707C08091C5
:108B500020018F7D03C080912001877F80932001B9
:108B600008950E94B9C66115710579F0FB01019065
:108B70000020E9F73197AF01461B570BDC01ED915F
:108B8000FC910280F381E02D199480E090E008953B
:108B90000F931F93CF93DF938C01EB01FC01808136
:108BA00091810097B1F0688179816115710579F043
:108BB000428153812C813D814217530740F00E942E
:108BC000D1C68C819D81F8019583848313C00E9456
:108BD0003DC588819981F801918380838A819B8139
:108BE000938382838C819D819583848319821882EB
:108BF0001B821A821D821C82DF91CF911F910F91DF
:108C000008950F931F93CF93DF93EC01888199818F
:108C1000009729F02A813B812617370788F48B01BA
:108C20006F5F7F4F0E94D5C5009761F0998388835D
:108C30001B830A832C813D81232B11F4FC011082BC
:108C400081E001C080E0DF91CF911F910F910895E5
:108C5000EF92FF920F931F93CF93DF93FB01248139
:108C60003581E080F180FC0104811581E114F1047B
:108C700011F480E016C02115310591F0EC01020FCE
:108C8000131FB801BEDF8823A1F3288139818C81AD
:108C90009D81B701820F931F0E94D1C61D830C8353
:108CA00081E0DF91CF911F910F91FF90EF90089598
:108CB000EF92FF920F931F93CF93DF93EC017B0111
:108CC0008A01BA019EDF2881398181110DC02115E9
:108CD000310519F0C9010E943DC5198218821D8213
:108CE0001C821B821A8206C01D830C83B701C90136
:108CF0000E94D1C6CE01DF91CF911F910F91FF90BD
:108D0000EF900895CF93DF93EC016115710551F059
:108D1000FB0101900020E9F73197AF01461B570B8B
:108D2000C7DF0CC088819981009711F00E943DC572
:108D3000198218821D821C821B821A82CE01DF9149
:108D4000CF910895FC01808191810C943DC50F93D2
:108D50001F93CF93DF93CDB7DEB762970FB6F8942A
:108D6000DEBF0FBECDBF8C01CB01F8011182108296
:108D7000138212821582148250E0BE016F5F7F4F12
:108D80000E94B9C0BE016F5F7F4FC801BBDF629612
:108D90000FB6F894DEBF0FBECDBFDF91CF911F910C
:108DA0000F9108950F931F93CF93DF93CDB7DEB745
:108DB00029970FB6F894DEBF0FBECDBF8C01862F6A
:108DC000F80111821082138212821582148250E0FF
:108DD000BE016F5F7F4F90E00E94FCC0BE016F5FDD
:108DE0007F4FC8018FDF29960FB6F894DEBF0FBE04
:108DF000CDBFDF91CF911F910F910895FC0111829A
:108E0000108213821282158214826115710549F055
:108E1000FB0101900020E9F73197AF01461B570B8A
:108E200047CF0895CF93DF9300D01F92CDB7DEB721
:108E3000611571058105910579F09B01AC0169838C
:108E40003A834B835C830E94ADC029813A814B8178
:108E50005C810E9478C203C060E070E0CB010F909B
:108E60000F900F900F90DF91CF9108954F925F92E6
:108E70006F927F92EF92FF920F931F93CF93DF93A6
:108E8000CDB7DEB7A1970FB6F894DEBF0FBECDBF4A
:108E90007C01FA01CB0119A2223008F42AE08E01EC
:108EA0000F5D1F4F422E512C612C712CBF01A3016D
:108EB00092010E94A4C2F901CA01015011096A304D
:108EC00014F4605D01C0695CD8016C93232B242BE2
:108ED000252B61F7B801C70146DEA1960FB6F894BD
:108EE000DEBF0FBECDBFDF91CF911F910F91FF90DD
:108EF000EF907F906F905F904F90089563E876E0D9
:108F000032CE0F931F93CF93DF93EC012CDE8C01B5
:108F1000CE01F4DF800F911FDF91CF911F910F9150
:108F20000895DC01ED91FC910190F081E02D199400
:108F30004F925F926F927F928F929F92AF92BF9269
:108F4000CF92DF92EF92FF92CF93DF93EC016A0111
:108F50007B01B22E9A01AB01C701B6010E94DDC3AD
:108F6000882319F066E876E027C026013701E894E7
:108F700077F82FEF3FEF4FE75FE7C301B2010E94A1
:108F8000DDC381110DC02FEF3FEF4FE75FE7C30156
:108F9000B2010E942FC118161CF46AE876E00CC0DA
:108FA0002FEF3FEF4FE75FE4C701B6010E94D3C345
:108FB000181694F46EE876E0CE01DF91CF91FF9021
:108FC000EF90DF90CF90BF90AF909F908F907F9069
:108FD0006F905F904F90C7CD2FEF3FEF4FE75FEC63
:108FE000C701B6010E942FC187FDE4CF20E030E029
:108FF000A901C701B6010E942FC187FF09C06DE218
:10900000CE018FDF4C01F7FAF094F7F8F09402C02C
:10901000812C912CA12C60E070E080E09FE3AB14E8
:1090200041F020E030E040E251E40E943AC3A394D2
:10903000F6CF9B01AC01C701B6010E94D6C22B013D
:109040003C010E94A7C36B017C010E9433C19B01BC
:10905000AC01C301B2010E94D5C22B013C012AE040
:10906000B701A601CE0102DF7C01E80CF91CBB2090
:1090700029F06EE2CE0155DFE80EF91EDB2CDD2073
:1090800021F120E030E040E251E4C301B2010E944E
:1090900094C12B013C010E94A7C34B01A12CB12C10
:1090A0002AE0B501A401CE01E1DEE80EF91EC501FA
:1090B000B4010E9433C19B01AC01C301B2010E9403
:1090C000D5C22B013C01DA94DACFC701DF91CF91F1
:1090D000FF90EF90DF90CF90BF90AF909F908F90D8
:1090E0007F906F905F904F9008953DCDEF92FF92EB
:1090F0000F931F93CF93DF938C017B01C0E0D0E0EF
:10910000F701EC0FFD1F6491662361F0D801ED912A
:10911000FC910190F081E02DC8011995892B11F087
:109120002196EECFCE01DF91CF911F910F91FF904D
:10913000EF9008950F931F93CF93DF93EC01D6DF49
:109140008C01CE01DBDE800F911FDF91CF911F914B
:109150000F9108951F920F920FB60F9211240BB624
:109160000F922F933F934F935F936F937F938F93C0
:109170009F93AF93BF93EF93FF9386EF97E0EADB64
:10918000FF91EF91BF91AF919F918F917F916F91DF
:109190005F914F913F912F910F900BBE0F900FBE9B
:1091A0000F901F9018951F920F920FB60F921124D7
:1091B0000BB60F922F933F934F935F936F937F93D1
:1091C0008F939F93AF93BF93EF93FF9386EF97E0B7
:1091D00043DBFF91EF91BF91AF919F918F917F9171
:1091E0006F915F914F913F912F910F900BBE0F9018
:1091F0000FBE0F901F9018951F920F920FB60F92EF
:1092000011240BB60F922F933F934F935F936F935D
:109210007F938F939F93AF93BF93EF93FF9383E9D4
:1092200098E098DBFF91EF91BF91AF919F918F9163
:109230007F916F915F914F913F912F910F900BBE56
:109240000F900FBE0F901F9018951F920F920FB6A0
:109250000F9211240BB60F922F933F934F935F936E
:109260006F937F938F939F93AF93BF93EF93FF93EE
:1092700083E998E0F1DAFF91EF91BF91AF919F916F
:109280008F917F916F915F914F913F912F910F90AF
:109290000BBE0F900FBE0F901F9018951F920F924C
:1092A0000FB60F9211240BB60F922F933F934F934B
:1092B0005F936F937F938F939F93AF93BF93EF933E
:1092C000FF9380E399E046DBFF91EF91BF91AF916F
:1092D0009F918F917F916F915F914F913F912F91CE
:1092E0000F900BBE0F900FBE0F901F9018951F92FE
:1092F0000F920FB60F9211240BB60F922F933F933C
:109300004F935F936F937F938F939F93AF93BF938D
:10931000EF93FF9380E399E09FDAFF91EF91BF9184
:10932000AF919F918F917F916F915F914F913F91FD
:109330002F910F900BBE0F900FBE0F901F9018959E
:109340001F920F920FB60F9211240BB60F922F930C
:109350003F934F935F936F937F938F939F93AF93BD
:10936000BF93EF93FF938DEC99E0F4DAFF91EF91C7
:10937000BF91AF919F918F917F916F915F914F912D
:109380003F912F910F900BBE0F900FBE0F901F902B
:1093900018951F920F920FB60F9211240BB60F92D1
:1093A0002F933F934F935F936F937F938F939F93ED
:1093B000AF93BF93EF93FF938DEC99E04DDAFF915C
:1093C000EF91BF91AF919F918F917F916F915F913D
:1093D0004F913F912F910F900BBE0F900FBE0F90AA
:1093E0001F901895CF93DF93EC01E881F9810680F7
:1093F000F781E02D1995EA89FB8980818F7E808332
:10940000EA89FB898081877F8083EA89FB89808163
:109410008F778083EA89FB8980818F7D80838A8D25
:10942000898FDF91CF910895CF92DF92EF92FF92D3
:109430001F93CF93DF93EC016A017B01122FE88920
:10944000F98982E080834115514E61057105B1F0C3
:1094500060E079E08DE390E0A70196010E94A4C24C
:10946000DA01C9010197A109B109B695A7959795A8
:109470008795AC01411580E15807A8F0E889F98982
:10948000108260E874E88EE190E0A70196010E94E6
:10949000A4C2BA01A9014150510961097109769527
:1094A000679557954795EC85FD855083EE85FF853B
:1094B0004083188EEC89FD891083EA89FB898081BD
:1094C00080618083EA89FB89808188608083EA8962
:1094D000FB89808180688083EA89FB8980818F7D18
:1094E0008083DF91CF911F91FF90EF90DF90CF901D
:1094F0000895CF93DF93282F30E0F901E252FE4E1A
:109500008491F901E856FE4ED491F901EE5AFE4ECF
:10951000C491CC2389F08111CEDAEC2FF0E0EE0F6C
:10952000FF1FE85CFE4EA591B491EC91ED2381E024
:1095300090E021F480E002C080E090E0DF91CF91E4
:1095400008951F93CF93DF93282F30E0F901E25263
:10955000FE4E8491F901E856FE4ED491F901EE5A7F
:10956000FE4EC491CC23C1F0162F8111A4DAEC2F4A
:10957000F0E0EE0FFF1FE25EFE4EA591B4918FB7B3
:10958000F894111105C09C91ED2FE095E92302C0DC
:10959000EC91ED2BEC938FBFDF91CF911F9108954C
:1095A000CF93DF9390E0FC01E856FE4E2491FC013E
:1095B000EE5AFE4E8491882361F190E0880F991F46
:1095C000FC01EC5FFE4EC591D491FC01E25EFE4EC3
:1095D000A591B491611109C09FB7F8948881209535
:1095E00082238883EC912E230BC0623061F49FB7F5
:1095F000F8943881822F809583238883EC912E2BD9
:109600002C939FBF06C08FB7F894E8812E2B288338
:109610008FBFDF91CF9108951F93CF93DF93182FC2
:10962000EB0161E0BDDF209711F460E004C0CF3FA3
:10963000D10531F461E0812FDF91CF911F9181CF6E
:10964000E12FF0E0E252FE4EE4914E2F50E0FA019D
:109650003197E231F10508F09DC08827E858FE4FA8
:109660008F4F0C9494C484B5806884BDC7BD97C0E7
:1096700084B5806284BDC8BD92C08091800080683E
:1096800080938000D0938900C093880088C0809127
:109690008000806280938000D0938B00C0938A000A
:1096A0007EC080918000886080938000D0938D0080
:1096B000C0938C0074C08091B00080688093B0002B
:1096C000C093B3006CC08091B00080628093B00002
:1096D000C093B40064C08091900080688093900033
:1096E000D0939900C09398005AC0809190008062F6
:1096F00080939000D0939B00C0939A0050C08091BB
:109700009000886080939000D0939D00C0939C004F
:1097100046C08091A00080688093A0008091A00046
:109720008F7B8093A000D093A900C093A80037C07E
:109730008091A00080628093A000D093AB00C09382
:10974000AA002DC08091A00088608093A000D093D3
:10975000AD00C093AC0023C080912001806880934D
:109760002001D0932901C093280119C080912001C4
:10977000806280932001D0932B01C0932A010FC0F7
:1097800080912001886080932001D0932D01C093A7
:109790002C0105C0C038D1050CF04CCF46CFDF916D
:1097A000CF911F910895863308F0865390917B00E6
:1097B000282F2870977F922B90937B00877080646E
:1097C00080937C0080917A00806480937A008091FD
:1097D0007A0086FDFCCF809178002091790090E09E
:1097E000922B08953FB7F8948091FD0E9091FE0E54
:1097F000A091FF0EB091000F26B5A89B05C02F3F8A
:1098000019F00196A11DB11D3FBFBA2FA92F982FA6
:109810008827820F911DA11DB11DBC01CD0142E021
:10982000660F771F881F991F4A95D1F708958F9269
:109830009F92AF92BF92CF92DF92EF92FF926B0115
:109840007C01D0DF4B015C01C114D104E104F104BF
:10985000E9F0C8DFDC01CB0188199909AA09BB0925
:10986000883E9340A105B10578F321E0C21AD108E2
:10987000E108F10888EE880E83E0981EA11CB11C57
:10988000C114D104E104F10421F7DECFFF90EF9081
:10989000DF90CF90BF90AF909F908F9008950895E4
:1098A0000895089508951092D20B0895CF93DF93F1
:1098B000EC018091020F811109C06A8D7B8DCE0170
:1098C00049960E94996B81E08093020F21E83FEF57
:1098D0003B872A878FE790E09D878C871F861E86AF
:1098E000398B288B9B8B8A8B1D8A1C8ADF91CF91A9
:1098F00008950F931F93CF93DF93EC011F8A1E8A65
:109900008C01075E1F4F40E060E0C8010E94914259
:1099100040E064E0C8010E9491420E9476846C8F0E
:109920007D8F8E8F9F8FDF91CF911F910F91089523
:109930000F931F93CF93DF93EC018091010F81115F
:1099400012C00A8D1B8D6AEA70E0C8010E94068F62
:10995000D801ED91FC910680F781E02DC8011995A1
:1099600081E08093010F4AE06EE0CE0149960E94AB
:10997000914221E83FEF3B872A878FE790E09D8760
:109980008C871F861E86398B288B9B8B8A8B1D8A22
:109990001C8ADF91CF911F910F9108950F931F9310
:1099A000CF93DF93EC011F8A1E8A8C01075E1F4F45
:1099B00040E060E0C8010E94544240E064E0C80119
:1099C0000E9454420E9476846C8F7D8F8E8F9F8F71
:1099D000DF91CF911F910F9108950F931F93CF9314
:1099E000DF93EC01E8A1F9A180819181A281B3818B
:1099F0008E01075E1F4F81159649A105B10509F437
:109A000050C040E056E960E070E083E998E00E94D1
:109A10001E8164E170E080E090E009DFE8A1F9A137
:109A200080819181A281B38181152BE49207A105E8
:109A3000B105E9F068F4803629E09207A105B10587
:109A4000A1F080389542A105B105C1F442E012C0F1
:109A5000811521EE9207A105B10559F08115924CAF
:109A6000A140B10559F445E005C041E003C043E021
:109A700001C046E06FE0C8010E94544283E998E0CB
:109A80000E941145E8A1F9A1408151816281738151
:109A900083E998E00E941E8164E170E080E090E03C
:109AA000C6DE4AE06EE0C8010E94544241E067E130
:109AB000C8010E9454424AA168E1C8010E94544270
:109AC0004BA18FEF840F8E3108F04CE066E1C801A6
:109AD0000E94544221E83FEF3B872A878FE790E0BE
:109AE0009D878C871F861E86398B288B9B8B8A8B44
:109AF0001D8A1C8ADF91CF911F910F9108950C94BC
:109B00000D8FCF93DF93C4E6DBE081E090E09A8392
:109B100089831092D20B66DE6C837D838E839F8354
:109B2000E49AEC9ADF91CF910895EF92FF920F9310
:109B30001F93CF93DF93EC016623E1F0262F653668
:109B400008F024E60A891B89E888F988D801AE194B
:109B5000BF0930E00E94A2C428EC30E040E050E0B1
:109B60000E94A4C2E20EF31EFB86EA86021B130BC0
:109B70001D870C87DF91CF911F910F91FF90EF9080
:109B80000895CF93DF93CDB7DEB7A2970FB6F894C1
:109B9000DEBF0FBECDBF80310CF080E123EE32E19D
:109BA0003A8329832BED32E13C832B8323ED32E191
:109BB0003E832D832BEC32E138872F8323EC32E177
:109BC0003A8729872BEB32E13C872B8723EB32E165
:109BD0003E872D872BEA32E1388B2F872DE932E142
:109BE0003A8B298B2BE832E13C8B2B8B2EE632E132
:109BF0003E8B2D8B29E532E1388F2F8B2FE432E11C
:109C00003A8F298F25E432E13C8F2B8F28E332E114
:109C10003E8F2D8F2CE232E138A32F8F24E232E1E8
:109C20003AA329A3E82FEE0FFF0BEC0FFD1F818154
:109C30009281A2960FB6F894DEBF0FBECDBFDF9122
:109C4000CF9108958F929F92AF92BF92CF92DF9261
:109C5000EF92FF920F931F93DC0118968D919C91C8
:109C600019971E96CD90DC901F976817790709F415
:109C700056C05896FC9058974C01092E000CAA0823
:109C8000BB088B01072E000C220B330B861797079E
:109C90003CF41696ED91FC911797FF2039F015C012
:109CA0001496ED91FC911597FF2079F00D2C000C86
:109CB000EE08FF08A9019801281939094A095B092A
:109CC0001C966D917C911D970EC00D2C000CEE081A
:109CD000FF08A9019801281939094A095B091A9650
:109CE0006D917C911B97CB01770FAA0BBB0BBC012D
:109CF000CD016C197D098E099F090E945EC48F01F8
:109D0000FF0F220B330BA9019801281939094A09C1
:109D10005B090E9478C2C20ED31EE41EF51EC60166
:109D20001F910F91FF90EF90DF90CF90BF90AF9079
:109D30009F908F900895EF92FF920F931F93CF9370
:109D4000DF938C01FC01778B668B7CDFEC01F801E3
:109D5000828193818830910531F57801F9E1EF0E28
:109D6000F11CD7FF06C06AE0C1388FEFD80754F066
:109D700001C068E02C2F9D2FC038D1052CF02FE7B3
:109D800090E002C021E89FEF422F592F57FF03C0F8
:109D9000519541955109C7010E94319ECD2B69F51E
:109DA0004FE766E027C0099741F57801E9E1EE0E3B
:109DB000F11CD7FF06C06EE0C138FFEFDF0754F09B
:109DC00001C06CE02C2F9D2FC038D1052CF02FE75F
:109DD00090E002C021E89FEF422F592F57FF03C0A8
:109DE000519541955109C7010E94319ECD2B29F40F
:109DF0004FE767E0C7010E94319E0E947684F80118
:109E0000648F758F868F978FDF91CF911F910F9100
:109E1000FF90EF900895CF93DF93EC017F8B6E8BD3
:109E200011DF9C018A819B8188309105C1F437FF45
:109E300006C061E021388FEF38074CF001C060E0C8
:109E4000A901203831052CF04FE750E002C041E86D
:109E50005FEF57FF1FC05195419551091BC00997EE
:109E6000E9F4922F832F2038310514F09FE780E02A
:109E7000492F582F41388FEF580714F441E85FEF0E
:109E800057FF03C0519541955109632F661F6627FF
:109E9000661F6C5FCE0149960E9491420E947684B3
:109EA0006C8F7D8F8E8F9F8FDF91CF9108950F9351
:109EB0001F93CF93DF93EC010E9476840C8D1D8D50
:109EC0002E8D3F8DDC01CB01801B910BA20BB30BC0
:109ED000853F9140A105B10540F06E897F89CE0193
:109EE000DF91CF911F910F9196CFDF91CF911F916D
:109EF0000F910895CF93DF93EC017F8B6E8BA2DEE1
:109F00009C018A819B8188309105C1F437FF06C08E
:109F100061E021388FEF38074CF001C060E0A90103
:109F2000203831052CF04FE750E002C041E85FEFE8
:109F300057FF1FC05195419551091BC00997E9F47E
:109F4000922F832F2038310514F09FE780E0492FAE
:109F5000582F41388FEF580714F441E85FEF57FF4F
:109F600003C0519541955109632F661F6627661FEF
:109F70006C5FCE0149960E9454420E9476846C8F99
:109F80007D8F8E8F9F8FDF91CF9108950F931F93B9
:109F9000CF93DF93EC010E9476840C8D1D8D2E8D66
:109FA0003F8DDC01CB01801B910BA20BB30B853FD6
:109FB0009140A105B10540F06E897F89CE01DF9106
:109FC000CF911F910F9196CFDF91CF911F910F915C
:109FD0000895CF93DF93EC0161E089E0E1DA60E07E
:109FE00089E0AFDA1092D70A83E395E099838883FA
:109FF000DF91CF910895CF92DF92EF92FF928091FF
:10A00000D80A833009F061C08091D90A8130D1F437
:10A0100088EE93E0A0E0B0E080936A0A90936B0A28
:10A02000A0936C0AB0936D0A80E797E1A0E0B0E0DE
:10A0300080936E0A90936F0AA093700AB093710A8E
:10A0400032E001C030E0E091D90AF0E0E652F54F8D
:10A050002081A0E1A30F48EE53E060E070E088EBC0
:10A06000C82E8BE0D82EE12CF12C832F90E0FC0140
:10A07000EE0FFF1FEE0FFF1FE659F54F27FF10C031
:10A08000C082D182E282F382880F991F880F991FC4
:10A09000FC01E259F54F40835183628373830FC003
:10A0A0004083518362837383880F991F880F991FA0
:10A0B000FC01E259F54FC082D182E282F3823E5F19
:10A0C000220F3A13D2CF3093D30AFF90EF90DF9054
:10A0D000CF900895CF93DF938091D70A811151C01B
:10A0E0001092D50A1092D20AC1E0C093D70AD0913B
:10A0F000D60A61E089E054DA60E089E022DA2D2FA7
:10A1000030E040E050E060E47FE180E090E00E94D9
:10A1100078C2C093B00089E08093B1002093B3006F
:10A120008BEA289F212D112426952093B40080913D
:10A130006F008B7F80936F008091B000806280936E
:10A14000B0002091840030918500E091D20A81E036
:10A150008E0F8093D20A84E0E89FF0011124E65923
:10A16000F54F80819181A281B381820F931F9093DB
:10A170008B0080938A00B29A80916F0084608093F4
:10A180006F00DF91CF9108954F925F926F927F920F
:10A190008F929F92AF92BF92CF92DF92EF92FF92F7
:10A1A0008AE18093D30A2093D40A88E28093D60A66
:10A1B00081E08093D90A8093DA0A8EE08093D80AEE
:10A1C00080EC92E1A0E0B0E080936A0A90936B0A81
:10A1D000A0936C0AB0936D0A80EB94E0A0E0B0E02D
:10A1E00080936E0A90936F0AA093700AB093710ADD
:10A1F000A4E1440F551F661F771FAA95D1F722E0EF
:10A2000030E0B0EBCB2EB4E0DB2EE12CF12C80E67D
:10A21000482E89E0582E612C712C90E4892E9CE9FF
:10A22000992EA12CB12CC901880F991F880F991F55
:10A23000FC01E659F54F77FF05C0408251826282EA
:10A24000738204C0C082D182E282F382C901019686
:10A25000880F991F880F991FFC01E659F54F283187
:10A2600029F0C082D182E282F38204C0808291828E
:10A27000A282B382440F551F661F771F2E5F3F4F88
:10A280002A31310581F6FF90EF90DF90CF90BF909B
:10A29000AF909F908F907F906F905F904F901ACF6C
:10A2A0008F929F92AF92BF92CF92DF92EF92FF92E6
:10A2B00082E18093D30A86E08093D40A96E2909359
:10A2C000D60A91E09093D90A9093DA0A8093D80A3B
:10A2D00088ED90E4A0E0B0E080936A0A90936B0A66
:10A2E000A0936C0AB0936D0A8CE19CE0A0E0B0E012
:10A2F00080936E0A90936F0AA093700AB093710ACC
:10A30000742F66275527442722E030E0ACE1CA2E9F
:10A31000ACE0DA2EE12CF12CB8E38B2EB8E19B2EC9
:10A32000A12CB12CC901880F991F880F991FFC011E
:10A33000E659F54F77FF05C080829182A282B382F1
:10A3400004C0C082D182E282F382F901EE0FFF1FC6
:10A35000EE0FFF1FE259F54FC082D182E282F382F5
:10A36000440F551F661F771F2E5F3F4F2231310567
:10A37000C9F68CE199E8A0E0B0E08093AE0A909332
:10A38000AF0AA093B00AB093B10AFF90EF90DF90AC
:10A39000CF90BF90AF909F908F909CCE1F920F92C6
:10A3A0000FB60F9211240BB60F922F933F934F933A
:10A3B0005F936F937F938F939F93AF93BF93EF932D
:10A3C000FF939091D20A8091D30A981316C01092ED
:10A3D000D20A8091D90A8F5F8093D90A9091D90AC5
:10A3E0008091DA0A891740F481E08093D90A80913C
:10A3F000D50A8F5F8093D50AFEDD9091D50A8091B2
:10A40000D40A98130DC08091B0008F7D8093B00066
:10A4100080916F008B7F80936F001092D70A27C0C6
:10A420008091B00085FF04C08091B0008F7D03C093
:10A430008091B00080628093B000209184003091C0
:10A440008500E091D20A81E08E0F8093D20A84E0E9
:10A45000E89FF0011124E659F54F80819181A28196
:10A46000B381820F931F90938B0080938A00FF919A
:10A47000EF91BF91AF919F918F917F916F915F917C
:10A480004F913F912F910F900BBE0F900FBE0F90E9
:10A490001F9018951F920F920FB60F9211240BB6B2
:10A4A0000F921F932F933F934F935F936F937F93DD
:10A4B0008F939F93AF93BF93EF93FF93CF93DF93CC
:10A4C00000D01F92CDB7DEB78091640B12D811E097
:10A4D000892B09F010E086D969837A838B839C836A
:10A4E00089819A81AB81BC814091680B5091690B45
:10A4F00060916A0B70916B0B841B950BA60BB70BCD
:10A500002091650B3091660B2430310509F44CC065
:10A510002530310521F021303105E9F414C02091B6
:10A52000670B222339F02091D20B20FF02C0289A1A
:10A5300001C02898112379F0813E2EE29207A105EF
:10A54000B10548F02BC0112379F125E030E03093BC
:10A55000660B2093650B2091650B3091660B2530BF
:10A56000310511F5E091D20BF0E0EE0FFF1FE45939
:10A57000F44F9183808389819A81AB81BC818093E0
:10A58000680B9093690BA0936A0BB0936B0B80914F
:10A59000D20B8F5F8093D20B833330F084E090E056
:10A5A0009093660B8093650B0F900F900F900F9018
:10A5B000DF91CF91FF91EF91BF91AF919F918F91DB
:10A5C0007F916F915F914F913F912F911F910F90CC
:10A5D0000BBE0F900FBE0F901F9018958091A6078D
:10A5E00080938713089580912B0F882359F08091D1
:10A5F000290F90912A0FDC01ED91FC910480F581E7
:10A60000E02D1994089580912B0F882369F0809193
:10A61000290F90912A0FDC01ED91FC910190F081BE
:10A62000E02D6FEF73E01994089580912B0F88232C
:10A6300089F08091360F882321F080E090E0D3DF0D
:10A6400003C080E090E0DFDF9091360F81E0892742
:10A650008093360F089520912B0F222369F0A0914B
:10A66000290FB0912A0FED91FC9111970190F08183
:10A67000E02DBC01CD01199408958091280F882305
:10A6800059F08091260F9091270FDC01ED91FC91FC
:10A690000480F581E02D199408958091280F882376
:10A6A00069F08091260F9091270FDC01ED91FC91CC
:10A6B0000190F081E02D6FEF73E01994089580917F
:10A6C000280F882389F08091350F882321F080E0BE
:10A6D00090E0D3DF03C080E090E0DFDF9091350FA2
:10A6E00081E089278093350F08952091280F222338
:10A6F00069F0A091260FB091270FED91FC91119771
:10A700000190F081E02DBC01CD01199408952091B4
:10A71000250F222369F0A091230FB091240FED9112
:10A72000FC9111970190F081E02DBC01CD011994AD
:10A7300008952091220F222369F0A091200FB0915B
:10A74000210FED91FC9111970190F081E02DBC015A
:10A75000CD011994089520911F0F222369F0A09133
:10A760001D0FB0911E0FED91FC9111970190F0819A
:10A77000E02DBC01CD011994089520911C0F2223D6
:10A7800069F0A0911A0FB0911B0FED91FC911197F8
:10A790000190F081E02DBC01CD0119940895209124
:10A7A000190F222369F0A091170FB091180FED91A6
:10A7B000FC9111970190F081E02DBC01CD0119941D
:10A7C00008952091160F222369F0A091140FB091E3
:10A7D000150FED91FC9111970190F081E02DBC01D6
:10A7E000CD01199408952091130F222369F0A091AF
:10A7F000110FB091120FED91FC9111970190F08122
:10A80000E02DBC01CD01199408958091A20790918B
:10A81000A307DC01ED91FC91EE59FF4F0190F0810F
:10A82000E02D19948091A2079091A307DC01ED918E
:10A83000FC91E05AFF4F0190F081E02D1994809136
:10A84000A2079091A307DC01ED91FC91E25AFF4F22
:10A850000190F081E02D19948091A607882361F082
:10A860000E9418A1029741F067ED73E18091851372
:10A87000909186130C949A480895809187138823A9
:10A8800041F069E273E180918513909186130C94F5
:10A890009A48089580918713882341F069E173E114
:10A8A00080918513909186130C949A480895CF93C4
:10A8B000DF932091390F30913A0F28173907D1F0E3
:10A8C00090933A0F8093390F20918713222391F0B0
:10A8D000EC0168EA73E180918513909186130E94E0
:10A8E0007648BE018091851390918613DF91CF91B8
:10A8F0000C94DD67DF91CF910895CF93DF93209182
:10A90000370F3091380F28173907D1F09093380F4F
:10A910008093370F20918713222391F0EC016EE88A
:10A9200073E180918513909186130E947648BE0151
:10A930008091851390918613DF91CF910C94DD6700
:10A94000DF91CF9108952091250F222339F0BC018A
:10A9500080910F0F9091100F0C940D8F08952091FE
:10A96000220F222339F0BC0180910D0F90910E0F20
:10A970000C940D8F089520911F0F222339F0BC01F4
:10A9800080910B0F90910C0F0C940D8F08952091D6
:10A990001C0F222339F0BC018091090F90910A0FFE
:10A9A0000C940D8F08952091190F222339F0BC01CA
:10A9B0008091070F9091080F0C940D8F08952091AE
:10A9C000160F222339F0BC018091050F9091060FDC
:10A9D0000C940D8F08952091130F222339F0BC01A0
:10A9E0008091030F9091040F0C940D8F0895CF92D6
:10A9F000DF92EF92FF9220910002213019F4209112
:10AA0000F31204C02230C9F52091F9122223A9F1D2
:10AA10009C01211584E0380710F02FEF33E0ADE002
:10AA2000B0E00E94C6C22FEF33E040E050E00E9449
:10AA300078C269017A018FEFC81AD80AE80AF80AC1
:10AA4000809195148C15C9F0C0929514809187134C
:10AA5000882399F067E773E18091851390918613BD
:10AA60000E9476486C2D8091851390918613FF90FB
:10AA7000EF90DF90CF900C94836AFF90EF90DF907F
:10AA8000CF900895CF92DF92EF92FF922091000233
:10AA9000213019F42091F01204C02230C9F5209120
:10AAA000F6122223A9F19C01211584E0380710F049
:10AAB0002FEF33E0ADE0B0E00E94C6C22FEF33E0ED
:10AAC00040E050E00E9478C269017A018FEFC81A15
:10AAD000D80AE80AF80A809193148C15C9F0C0923C
:10AAE000931480918713882399F060E673E1809135
:10AAF0008513909186130E9476486C2D8091851362
:10AB000090918613FF90EF90DF90CF900C94836A22
:10AB1000FF90EF90DF90CF90089583E080939F07A0
:10AB200081E0FAD680918713882341F063E573E1D1
:10AB300080918513909186130C949A48089582E031
:10AB400080939F0781E0E8D680918713882341F0A6
:10AB500069E373E180918513909186130C949A4870
:10AB6000089581E080939F07A9D680918713882359
:10AB700041F066E473E180918513909186130C9403
:10AB80009A4808950C94D09680912D0F81110BC096
:10AB900081E09091E812911101C080E080932C0F28
:10ABA00081E080932D0F80912C0F882329F00E9443
:10ABB000BD9610922C0F08950E94D09681E080934C
:10ABC0002C0F08950C94BD968091DE12811111C056
:10ABD0008091210790912207FC0121A132A1121638
:10ABE00013061CF460E070E002C06FEF70E00C949C
:10ABF000FC3D08958091DE12811108C060E070E094
:10AC000080912107909122070C94FC3D089580913A
:10AC1000DE12811108C06FEF70E0809121079091E2
:10AC200022070C94FC3D08950C94909780910102AA
:10AC300081110C9476970C9490970C94769784E6F7
:10AC40000C94145F89E10C94145F82E30C94145FFC
:10AC50008BE40C94145F80910002813011F482E047
:10AC600001C081E00C94B75F82E00C94B75F81E093
:10AC70000C94B75F0C94BD0ECF93DF93CDB7DEB7C6
:10AC800065970FB6F894DEBF0FBECDBF809141121D
:10AC90009091421220913F12309140123A832983C1
:10ACA0009C838B8381E08D8B82E08F938DB79EB7E1
:10ACB00045970FB6F8949EBF0FBE8DBFADB7BEB718
:10ACC000119685E1FE01319601900D928A95E1F78A
:10ACD00083E39CE00E94FD920FB6F894DEBF0FBEA6
:10ACE000CDBF80918713882381F06EEF72E1809150
:10ACF00085139091861365960FB6F894DEBF0FBE4C
:10AD0000CDBFDF91CF910C949A4865960FB6F89419
:10AD1000DEBF0FBECDBFDF91CF9108958091420776
:10AD2000882339F083E39CE00E94959421EB31E77E
:10AD300006C083E39CE00E94BC9421E731E74CE22B
:10AD400051E060E070E085E69CE00E941B3F80914E
:10AD50008713882341F06BEE72E180918513909107
:10AD600086130C949A480895682F809185139091CA
:10AD700086130E949A6A65ED73E180918513909124
:10AD800086130C947648209185133091861388237E
:10AD900019F062E078E002C066E078E0C9010C9446
:10ADA0007648F1DF80918513909186130C947E474D
:10ADB0002091851330918613882319F06AEC73E192
:10ADC00002C06FEC73E1C9010E947648809185133F
:10ADD000909186130C947E478091851390918613F1
:10ADE0000C947E4768EC73E18091851390918613F3
:10ADF0000C94764864EC73E18091851390918613EE
:10AE00000C947648CF93CDE262EC73E18091851388
:10AE1000909186130E947648C150B1F780918513B6
:10AE2000909186130E947E4780918513909186139E
:10AE3000DC01ED91FC910680F781E02DCF91199412
:10AE40000C9491710C94CD710C94B5700C94F070BD
:10AE50008091470F882319F00E94B57002C00E94AC
:10AE6000F0709091470F81E089278093470F0895F4
:10AE70000C9471710C94B17183E39CE00E94A894CE
:10AE800081110C9471710C94B17182E09CE00E946C
:10AE9000A89481110C9491710C94CD718091A207AA
:10AEA0009091A307DC01ED91FC91EA5BFF4F0190CB
:10AEB000F081E02D199580918713882341F063E696
:10AEC00075E180918513909186130C949A480895AA
:10AED000CF93DF93CDB7DEB765970FB6F894DEBF9B
:10AEE0000FBECDBF809141129091421220913F122E
:10AEF000309140123A8329839C838B8381E08D8B30
:10AF000082E08F938DB79EB745970FB6F8949EBF9A
:10AF10000FBE8DBFADB7BEB7119685E1FE0131966C
:10AF200001900D928A95E1F782E09CE00E94FD92EB
:10AF30000FB6F894DEBF0FBECDBF80918713882374
:10AF400081F06BE875E18091851390918613659689
:10AF50000FB6F894DEBF0FBECDBFDF91CF910C943A
:10AF60009A4865960FB6F894DEBF0FBECDBFDF914D
:10AF7000CF9108950E94B57040916C1350916D135C
:10AF800060E070E020EF30E785E69CE00E941B3F28
:10AF9000909368148093671480918713882341F0FD
:10AFA00066E175E180918513909186130C949A481F
:10AFB00008950E94F07040916C1350916D1360E001
:10AFC00070E025EB30E785E69CE00E941B3F909304
:10AFD00068148093671480918713882341F063E09D
:10AFE00075E180918513909186130C949A48089589
:10AFF00080913C07882339F082E09CE00E94959480
:10B000002DEC31E706C082E09CE00E94BC9421E96F
:10B0100031E74CE251E060E070E085E69CE00E94A0
:10B020001B3F80918713882341F068E775E1809189
:10B030008513909186130C949A48089569E081E0F5
:10B040000C94EB9568E081E00C94EB9567E081E06F
:10B050000C94EB9561E081E00C94EB9569E080E065
:10B060000C94EB9568E080E00C94EB9567E080E051
:10B070000C94EB9561E080E00C94EB958CE00C94E3
:10B0800038968BE00C9438968AE00C94389689E0D8
:10B090000C94389688E00C94389687E00C94389697
:10B0A00086E00C94389685E00C94389684E00C94F5
:10B0B000389683E00C94389682E00C94389681E0C0
:10B0C0000C9438968CE00C945F968BE00C945F9611
:10B0D0008AE00C945F9689E00C945F9688E00C946B
:10B0E0005F9687E00C945F9686E00C945F9685E00F
:10B0F0000C945F9684E00C945F9683E00C945F96CA
:10B1000082E00C945F9681E00C945F968CE00C9446
:10B1100086968BE00C9486968AE00C94869689E05D
:10B120000C94869688E00C94869687E00C9486961C
:10B1300086E00C94869685E00C94869684E00C94C8
:10B14000869683E00C94869682E00C94869681E045
:10B150000C9486960C94A5960C94B1960F931F931D
:10B16000CF93DF930091420F1091430FC0911307CB
:10B17000D0911407B801CE010E94B43E882379F023
:10B18000B801CE010E94CC3E809115079091160720
:10B19000DC01ED91FC9102A0F3A1E02D1995009145
:10B1A000400F1091410FC0911307D0911407B801BF
:10B1B000CE010E94B43E882321F0B801CE010E9446
:10B1C000CC3E599880918713882361F065EA74E139
:10B1D0008091851390918613DF91CF911F910F91EC
:10B1E0000C949A48DF91CF911F910F910895CF93BE
:10B1F000DF9380916614882321F11092661460E039
:10B2000088E00E94A14AC0916714D0916814BE01E1
:10B2100085E69CE00E94B43E882329F0BE0185E6C5
:10B220009CE00E94CC3E80918713882371F06AE4F1
:10B2300075E18091851390918613DF91CF910C94E5
:10B240009A48DF91CF910C94E394DF91CF910895C8
:10B2500080916614811102C00C94E3940895CF93F9
:10B26000DF9380916914882311F10E94B5701092C8
:10B270006914C0916714D0916814BE0185E69CE002
:10B280000E94B43E882329F0BE0185E69CE00E941E
:10B29000CC3E80918713882371F061E375E1809142
:10B2A000851390918613DF91CF910C949A48DF918A
:10B2B000CF910C940571DF91CF9108950C94057195
:10B2C0008091480F882319F00E94B57002C00E9437
:10B2D00088729091480F81E089278093480F0895E4
:10B2E0000C9488720C949B720C94B2728091460FED
:10B2F000882319F00E949B7202C00E94B272909142
:10B30000460F81E089278093460F08950C94FD72C3
:10B310000E94FD728091A2079091A307DC01ED913C
:10B32000FC9106A0F7A1E02D19940C943A7380913A
:10B33000450F882319F00E94FD7202C00E943A73E3
:10B340009091450F81E089278093450F08950C94D3
:10B3500056730C9472738091440F882319F00E94E5
:10B36000567302C00E9472739091440F81E0892746
:10B370008093440F08950E946A86809187138823E2
:10B38000D1F020914513809185139091861321115E
:10B3900007C020914813211103C06DEA74E109C070
:10B3A0002091D90B222319F06CEE74E102C068EDF4
:10B3B00074E10C949A4808958091D90B81110C94F2
:10B3C00062860C946A860E94628680918713882325
:10B3D00041F067EF74E180918513909186130C948E
:10B3E0009A4808950C9442A28091DB138111BAC649
:10B3F0000C9442A2B7C60E9441718091A20790911D
:10B40000A307DC01ED91FC9104A0F5A1E02D1994B6
:10B41000CF93DF93C0911307D09114076091420F2F
:10B420007091430FCE010E94B43E811129C040911A
:10B430003F0F50E060E070E021E231E8CE010E9471
:10B44000233F9093430F8093420F80911507909173
:10B450001607DC01ED91FC9100A0F1A1E02D1995FA
:10B4600080912F07882361F06091400F7091410F08
:10B4700080911307909114070E94B43E882371F0C5
:10B48000809187138823E9F06CE974E1809185133A
:10B4900090918613DF91CF910C949A480E941D845D
:10B4A0002DE134E844E650E060E070E0809113075D
:10B4B000909114070E94233F9093410F8093400F77
:10B4C000DFCFDF91CF9108950E948086809187130E
:10B4D000882341F061E774E1809185139091861390
:10B4E0000C949A480895E0913D0FF0913E0F8281AF
:10B4F0000E948A4080918713882341F063E574E1BC
:10B5000080918513909186130C949A4808958091A8
:10B51000DC13882319F00E94EA8602C00E94D486B8
:10B5200080918713882379F02091CF128091851321
:10B5300090918613222319F067E174E102C060E361
:10B5400074E10C949A480895B9C1CF938091DA0BB5
:10B55000882309F47EC00E94117B9091D80B882328
:10B5600041F0911176C080913507882309F45AC0C3
:10B5700070C091116EC0809187138823D1F068EF5D
:10B5800073E180918513909186130E947648809193
:10B59000D90B882341F06DEE73E180918513909172
:10B5A00086130E94764880918513909186130E949D
:10B5B0007E470E94BA7B81E080932007809113131D
:10B5C000882309F446C08091DB13882349F18091D8
:10B5D000CF12882379F02DE032EA42E350E060E0B8
:10B5E00070E085E69CE00E94233F90933C0F80939F
:10B5F0003B0F2FC080910702813059F54091D11245
:10B600005091D212141615065CF4052E000C660B30
:10B61000770B22E53BE585E69CE0CF910C941B3F40
:10B62000CF9140C082E080933507809187138823B3
:10B6300041F064E074E180918513909186130E943B
:10B640009A48C1E0C0937F1339D10E94BA7BC0935E
:10B650002007CF91089581E05FC18091801381110F
:10B660002DC181E059C10C94A16A53C28091891304
:10B6700081110C94A16A4DC28091A2079091A307F9
:10B68000DC01ED91FC910084F185E02D199580910C
:10B69000A2079091A307DC01ED91FC910480F58154
:10B6A000E02D199480910702813019F485E0809390
:10B6B0000702089510929E07089580910B07882332
:10B6C00071F010920B0780918713882341F060E995
:10B6D00077E180918513909186130C949A48089590
:10B6E00080910613833099F080910B0781110FC070
:10B6F00081E080930B0780918713882341F06BE7EB
:10B7000077E180918513909186130C949A4808955F
:10B7100080910B07882319F080E090E0CECF80E085
:10B7200090E0DECF80910A07833079F083E0809348
:10B730000A0780918713882341F06AE677E18091B8
:10B740008513909186130C949A48089580910A0766
:10B75000823079F082E080930A07809187138823F2
:10B7600041F069E577E180918513909186130C94FF
:10B770009A48089580910A07813079F081E080939A
:10B780000A0780918713882341F068E477E180916C
:10B790008513909186130C949A480895809189138B
:10B7A000882371F00E94A16A80918713882341F059
:10B7B00068E077E180918513909186130C949A4804
:10B7C000089580910613833059F02CF48130E9F00C
:10B7D0008230D9F030C0863044F08630B1F02BC0D2
:10B7E00080919807909199071FC080919807909138
:10B7F0009907DC01ED91FC910480F581E02D19950C
:10B8000080919607909197070FC080919C07909127
:10B810009D07DC01ED91FC910480F581E02D1995E7
:10B8200080919A0790919B07DC01ED91FC91048037
:10B83000F581E02D19958091A2079091A307DC0175
:10B84000ED91FC91E25BFF4F0190F081E02D1995A5
:10B850008091A2079091A307DC01ED91FC910484F3
:10B86000F585E02D60E070E01994ABDF0E943C8626
:10B870008091891381110E94A16A8091A4079091FF
:10B88000A507DC01ED91FC910480F581E02D19956F
:10B890008091A0079091A107DC01ED91FC910480BB
:10B8A000F581E02D19958091DE12882331F0809189
:10B8B0002107909122070C94D93C08958091891317
:10B8C000882339F180918013882319F11092801315
:10B8D0000E94F79680917F13882319F010927F13AE
:10B8E0000CC08091A2079091A307DC01ED91FC911F
:10B8F0000288F389E02D60E01995809187138823F1
:10B9000041F061E377E180918513909186130E9465
:10B910009A48109280130895CF9390918913992398
:10B92000D1F19091D80B911136C090918013911163
:10B9300032C0C82F81E08093801380916F0F8823DD
:10B9400031F081E00E94469710926F0F02C00E9472
:10B95000069780917F13882319F010927F130CC0F3
:10B960008091A2079091A307DC01ED91FC910288E0
:10B97000F389E02D61E0199580918713882359F0B0
:10B98000CC2349F06DE177E1809185139091861386
:10B99000CF910C949A48CF91089581E0BDCFCF9379
:10B9A000DF93C0916D0FD0916E0FBE0185E69CE0D4
:10B9B0000E94B43E882329F0BE0185E69CE00E94E7
:10B9C000CC3E10926E0F10926D0FDF91CF910895C3
:10B9D000CF92DF92EF92FF920F931F93CF93DF935B
:10B9E000C0900B13D0900C13E0900D13F0900E1339
:10B9F0001C141D041E041F040CF040C08091891308
:10BA0000882399F100916D0F10916E0FB80185E6B2
:10BA10009CE00E94B43E8823D9F0E3E6FEE0C0E05B
:10BA2000D0E0819191918017910769F40E9476840A
:10BA3000CC0FDD1FCC0FDD1FCB59D34F688379832B
:10BA40008A839B831BC02196CE31D10551F716C046
:10BA50002EEC3BE5B701A60185E69CE00E941B3F6A
:10BA600090936E0F80936D0F09C0DF91CF911F915E
:10BA70000F91FF90EF90DF90CF9091CFDF91CF911A
:10BA80001F910F91FF90EF90DF90CF9008950F934B
:10BA90001F9380910C0281111EC00E947684009138
:10BAA000690F10916A0F20916B0F30916C0FAB01F1
:10BAB000BC01401B510B620B730B8091FF129091E4
:10BAC0000013A0E0B0E0481759076A077B0718F099
:10BAD00081E080930C021F910F9108958091FF12D5
:10BAE00090910013892B89F080910C02882381F0BA
:10BAF0000E9476846093690F70936A0F80936B0F36
:10BB000090936C0F10920C02089581E080930C02C8
:10BB10000895CF92DF92EF92FF92CF93DF938091BF
:10BB2000D80B81117AC180919F07823040F08091BB
:10BB30008713882309F471C166EC76E191C0809186
:10BB4000E712882309F498C08091EC07882309F450
:10BB500093C08091881381118FC08091EF12882348
:10BB600059F18091991190919A11A0919B11B091E6
:10BB70009C11892B8A2B8B2BF9F00E947684C09024
:10BB80009911D0909A11E0909B11F0909C119B011B
:10BB9000AC012C193D094E095F0969017A01209118
:10BBA000EF1230E0A8EEB3E00E94C6C2C616D70678
:10BBB000E806F90608F460C0C0912107D091220779
:10BBC00089AD9AAD892B11F01AAE19AE8BA98130CF
:10BBD00009F06FC08FEF90E090932D0180932C01BE
:10BBE0009F8F8E8F0E9476846DAB7EAB8FAB98AFAC
:10BBF0008091A2079091A307DC01ED91FC91028452
:10BC0000F385E02D199581E0809388132091EC074E
:10BC100030E0A8EEB3E00E94C6C2AB01BC0129E847
:10BC20003DE585E69CE00E941B3F90938413809342
:10BC3000831380918713882309F4EFC064E976E1C8
:10BC400080918513909186130E9476486091EC074D
:10BC500080918513909186130E949A6A6BE876E131
:10BC60008091851390918613DF91CF91FF90EF9093
:10BC7000DF90CF900C949A480ADF80910C028823C1
:10BC800009F4CBC0809189138111C7C081E08093F2
:10BC9000891380930C0222DF809187138823A1F0FF
:10BCA00061E476E180918513909186130E949A4811
:10BCB0000BC0823009F096CF4FEF60E0CE010E94BA
:10BCC000893C8FEF90E08CCF80918813811136C032
:10BCD0008091E712882391F18091EC07882371F11C
:10BCE0008091EF12882351F18091991190919A11CE
:10BCF000A0919B11B0919C11892B8A2B8B2BF1F079
:10BD00000E947684C0909911D0909A11E0909B1176
:10BD1000F0909C119B01AC012C193D094E095F0963
:10BD200069017A012091EF1230E0A8EEB3E00E94A1
:10BD3000C6C2C616D706E806F906D8F110928813CF
:10BD400080918113909182138061909382138093EC
:10BD500081138091A2079091A307DC01ED91FC91E2
:10BD60000280F381E02D199580919F0781111AC0FF
:10BD7000409101135091021381E080937F1341158C
:10BD8000510561F060E070E02DEC3CE585E69CE05B
:10BD90000E941B3F80E00E94469704C080936F0F73
:10BDA00080E0BADDDF91CF91FF90EF90DF90CF90F0
:10BDB0000FCE66E776E180918513909186130E94FD
:10BDC00076480E947684C0909911D0909A11E090A4
:10BDD0009B11F0909C116C197D098E099F0928EE2A
:10BDE00033E040E050E00E94A4C2BA01A90121E082
:10BDF00080918513909186130E94364760E576E125
:10BE000080918513909186130E94764880918513C6
:10BE1000909186130E947E4791CFDF91CF91FF9042
:10BE2000EF90DF90CF900895AF92BF92CF92DF92C4
:10BE3000EF92FF920F931F93CF93DF939091610F37
:10BE400091110BC02091AB073091AC073093600F7C
:10BE500020935F0F91E09093610F9091570F911194
:10BE60000BC02091A9073091AA073093560F209359
:10BE7000550F91E09093570FA0905F0FB090600F17
:10BE80000091550F1091560FD0918713843608F00A
:10BE900047C0C82F682F70E080E090E00E9433C157
:10BEA00020E030E048EC52E40E943AC36B017C0190
:10BEB000B501BB0C880B990B0E9435C19B01AC01ED
:10BEC000C701B6010E9494C10E94A2C37093AC073F
:10BED0006093AB07B801110F880B990B0E9435C115
:10BEE0009B01AC01C701B6010E9494C10E94A2C38C
:10BEF0007093AA076093A907DD2371F160E276E1F0
:10BF000080918513909186130E9476486C2F8091C2
:10BF10008513909186130E949A6A6EE176E10CC0B7
:10BF2000B092AC07A092AB071093AA070093A907A1
:10BF3000DD2391F062E376E1809185139091861381
:10BF4000DF91CF911F910F91FF90EF90DF90CF90F5
:10BF5000BF90AF900C949A48DF91CF911F910F91B1
:10BF6000FF90EF90DF90CF90BF90AF900895CF9368
:10BF7000823069F49091FA122091F7123091FB12FD
:10BF80004091F8125091F9126091F6120CC0909104
:10BF9000F4122091F1123091F5124091F212509169
:10BFA000F3126091F01260939414509391144093A3
:10BFB000921430939014209393149093951490912D
:10BFC00000028917B9F0809300029091871399239A
:10BFD00089F0C82F65E076E18091851390918613F2
:10BFE0000E9476486C2F8091851390918613CF9193
:10BFF0000C94836ACF910895833079F030F48130C6
:10C0000051F0823091F48BE30BC0843041F08530E5
:10C0100061F482E405C08CE303C080E401C081E4E4
:10C020000E94794A21E0892B09F420E0822F0895AB
:10C03000E3DF91E0892708950F931F9380914D0FBF
:10C0400081110DC00E9476846093490F70934A0F4E
:10C0500080934B0F90934C0F81E080934D0F809114
:10C060000A028A3AF1F485E0C7DF882371F080E3A1
:10C0700099E09093A3148093A214909386138093D5
:10C0800085138FEF80930A020CC08DEC99E090939A
:10C09000A3148093A2149093861380938513109217
:10C0A0000A020E9476840091490F10914A0F209154
:10C0B0004B0F30914C0FDC01CB01801B910BA20B7D
:10C0C000B30BC397A105B10508F449C00E9476845B
:10C0D0006093490F70934A0F80934B0F90934C0FCE
:10C0E00085E08ADF882321F080910A02882349F0C5
:10C0F00085E082DF811133C080910A028F3F79F59C
:10C1000018C080E399E09093A3148093A2149093B5
:10C1100086138093851380918713882331F06BEE0B
:10C1200075E180E399E00E949A488FEF80930A02BC
:10C1300016C08DEC99E09093A3148093A214909371
:10C1400086138093851380918713882331F066EDE1
:10C1500075E18DEC99E00E949A4810920A021F91B5
:10C160000F9108951092DB1380918713882379F043
:10C170002091CF128091851390918613222319F07C
:10C1800066EA75E102C069EB75E10C949A4808957E
:10C1900081E08093E50B089581E08093E60B08959C
:10C1A00081E08093E70B08952F923F924F925F9228
:10C1B0006F927F928F929F92AF92BF92CF92DF92B7
:10C1C000EF92FF920F931F93CF93DF9300D000D095
:10C1D000CDB7DEB74DB65EB60E94DF430E94D443B2
:10C1E0000E9418A1029709F0EFC20E9401A18823C2
:10C1F00009F4E4C2C090B814D090B914E090B61419
:10C20000F090B714B601C7010E94B43E8823F1F044
:10C21000F701E250FE4F00E010E0819191918C1502
:10C220009D0571F40E947684000F111F000F111FED
:10C23000F701E00FF11F608371838283938308C04D
:10C240000F5F1F4F0E31110541F702C00E94EEA192
:10C250001092E80BEDB6FEB64091EB0B5091EC0B53
:10C26000CA01880F991FADB6BEB6A81AB90A0FB693
:10C27000F894BEBE0FBEADBE0DB71EB70F5F1F4F09
:10C280008091EE0B823069F0833029F1813009F022
:10C2900071C0B8018091C1149091C2140E944C9E4B
:10C2A00033C03FB7F89420E0822F90E084179507C1
:10C2B00074F4880F991FF801E80FF91FDC01A754E7
:10C2C000B14F8D919C91918380832F5FEDCF3FBFC4
:10C2D0001092D90E19C03FB7F89420E0822F90E059
:10C2E0008417950774F4880F991FF801E80FF91F58
:10C2F000DC01A557B04F8D919C91918380832F5F76
:10C30000EDCF3FBF1092BE1420E06AE071E0822FB3
:10C3100090E04091EB0B5091EC0B8417950754F58E
:10C32000689FF001699FF00D1124E554F04FA0853E
:10C33000B1858C918823E1F0A081B1813C91C80145
:10C34000830F911D830F911DDC0112978D919C919C
:10C35000A281B3814D915C9111970480F581E02D0C
:10C360004817590711F4108203C070838D939C9372
:10C370002F5FCDCF0FB6F894FEBE0FBEEDBE8091FD
:10C38000B510882321F084EB90E10E9436A18091C2
:10C39000BF10882321F08EEB90E10E9436A180919E
:10C3A000C910882321F088EC90E10E9436A1809189
:10C3B000D310882321F082ED90E10E9436A1809174
:10C3C000E90B882309F465C08091C910811105C06B
:10C3D0008091D310882309F450C08091CC109091A3
:10C3E000CD10E091D010F091D11023813481281725
:10C3F000390724F48085811109C00EC02181328162
:10C400008217930734F48085811106C088E090E09C
:10C4100005C080E190E002C080E290E02091D6105B
:10C420003091D710E091DA10F091DB104381548104
:10C430004217530724F42085222349F00AC0418182
:10C440005281241735073CF42085222311F08160A6
:10C4500003C0846001C0826020915B1030915C1049
:10C460002817390719F410925D1007C090935C10DB
:10C4700080935B1081E080935D1080915B109091C0
:10C480005C10429709F4A4C181E08093D510809399
:10C49000CB10A1E6B0E164E670E188EE682E83E09F
:10C4A000782E22242394FD0131978081882309F47A
:10C4B0007CC11496CD90DC901597DE82CD82F6017A
:10C4C0008781882309F471C18C91882309F46DC197
:10C4D00011964D915C91129730847301E41AF50A1C
:10C4E0001E141F042CF07A01F8EEEF1AF3E0FF0A95
:10C4F00020E030E001E010E0EFE0F7E290E0832C94
:10C50000912CA32CB12CC12CD12CA982BA82CB8224
:10C51000DC82650182E0C81AD108081519050CF003
:10C520004AC08BE0C816D104E0F5F6018827E6572B
:10C53000FE4F8F4F0C9494C4F901E15BF94F27C073
:10C54000F901E75BF94F23C0F901EF5BF94F1FC019
:10C55000F901E95CF94F1BC0F901E55DF94F17C01E
:10C56000F901E35EF94F13C0F901E35FF94F0FC022
:10C57000F901E550FA4F0BC0F901E951FA4F07C034
:10C58000F901EF52FA4F03C0F901E754FA4F028064
:10C59000F381E02DE41BF50BF7FF03C0F195E19566
:10C5A000F109EE15FF0514F4902F7F010F5F1F4F67
:10C5B0002E5F3F4FB2CF9F5FED81FE818185882343
:10C5C00009F4EAC0032D10E0F8013297EB30F105D1
:10C5D00008F0E2C08827EB56FE4F8F4F0C9494C4AE
:10C5E000913009F0ACC0C3C0913009F4D4C093308D
:10C5F00009F0D2C0A4C0913009F4CBC0923009F444
:10C60000CAC0933009F4B3C0943009F0C5C097C0D4
:10C61000913009F4BCC0923009F4BBC0943009F4E5
:10C62000A6C0953009F0B8C08AC0913009F4ADC0F9
:10C63000923009F4ACC0933009F4ABC0943009F4E3
:10C64000AAC0953009F493C0963009F0A5C077C010
:10C65000913009F498C0923009F497C0933009F4EE
:10C6600096C0953009F497C0963009F480C0973091
:10C6700009F092C064C0913009F483C0923009F48B
:10C6800082C0933009F481C0943009F480C09530A1
:10C6900009F47FC0963009F47EC0973009F467C072
:10C6A000983009F079C04BC0913009F468C09230DD
:10C6B00009F467C0933009F466C0943009F465C08A
:10C6C000963009F466C0973009F465C0983009F4D3
:10C6D0004EC0993009F060C032C0913009F44DC0AD
:10C6E000923009F44CC0933009F44BC0943009F4F3
:10C6F0004AC0953009F449C0963009F448C09730D3
:10C7000009F447C0983009F446C0993081F19A3055
:10C7100009F042C014C0913071F1923071F1933040
:10C7200071F1943071F1953071F1973081F1983059
:10C7300081F1993081F19A30D1F09B3069F591E027
:10C740002BC09130B1F09230B1F09330B1F0943011
:10C75000B1F09530B1F09630B1F09730B1F098303B
:10C76000B1F09930B1F09A30B1F09B30A9F492E079
:10C7700013C09CE011C09BE00FC09AE00DC099E08F
:10C780000BC098E009C097E007C096E005C095E0AF
:10C7900003C094E001C093E0FB018081891302C0D3
:10C7A0001C9203C02C92FB0190831796695F7F4F08
:10C7B000F0E1A53BBF0709F076CE04C00E94EB4331
:10C7C0000E94EEA181E066C00E94EB4380E062C05F
:10C7D000E0905E10F0905F101E141F040CF055C026
:10C7E0008091CA100091B6141091B7146091AA0FED
:10C7F0007091AB0F8823B1F081E08093CB10C8011A
:10C800000E94B43E811115C0A701FF0C660B770B87
:10C8100028EE30EAC8010E941B3F9093AB0F809333
:10C82000AA0F07C0C8010E94B43E811102C0109235
:10C83000CB108091D4100091B6141091B714609170
:10C84000A80F7091A90F8823D1F081E08093D510B3
:10C85000C8010E94B43E81111CCE40915E105091DF
:10C860005F10052E000C660B770B25EE30EAC80131
:10C870000E941B3F9093A90F8093A80F0ACEC80176
:10C880000E94B43E811105CE02C01092CB101092CE
:10C89000D510FFCD0FB6F8945EBE0FBE4DBE2696E6
:10C8A0000FB6F894DEBF0FBECDBFDF91CF911F91C1
:10C8B0000F91FF90EF90DF90CF90BF90AF909F903F
:10C8C0008F907F906F905F904F903F902F90089542
:10C8D000CF938091A70FC0910B02811101C1C2308B
:10C8E00009F450C0C33009F49DC0C13009F028C11B
:10C8F0008091E70B811124C181E090E00E94A8C4DF
:10C900009093C2148093C11462E083E00E94D04AE5
:10C910001092880F1092BB141092BA141092BF1488
:10C9200080E090E0FC01EE0FFF1FEA58F04F11820B
:10C930001082019688309105A9F71092870F109206
:10C94000860F80916A008C6080936A00ED9A8FB7A1
:10C95000F89420918400309185003093710F2093DA
:10C96000700F8FBF20ED30E64AEF50E060E070E0DE
:10C970008091B6149091B7140E941B3F81E0809380
:10C98000A70FDEC08091E60B8111DAC081E090E054
:10C990000E94A8C49093B60E8093B50E80910401B6
:10C9A0008E7F809304018091050181608093050151
:10C9B00086EF97E09093E00E8093DF0E2EE240EA40
:10C9C00056E861E070E00E94144A809165008B7F18
:10C9D000809365001092350189E0809334018EE2E6
:10C9E000809332018CEF8093300180E98093310194
:10C9F0001092DE0E1092DD0E1092DC0E1092DB0E05
:10CA00001092D90EE9EBFEE08CED95E081939193C5
:10CA10002EE0E93DF207D1F7C1E0C093DA0E2CEC2D
:10CA200030E651C08091E50B81118AC081E090E031
:10CA30000E94A8C49093B80E8093B70E8091040111
:10CA40008E7F8093040180910501816080930501B0
:10CA500086EF97E090938A0F8093890F26E040E05D
:10CA600052EC61E070E00E94144A809165008B7F77
:10CA7000809365001092350180E18093340186E057
:10CA8000809332018EEF8093300180E980933101F1
:10CA90001092BD141092BC141092750F1092740F66
:10CAA0001092BE14EBE8FFE08CED95E0819391933A
:10CAB0002FE0E73AF207D1F71092730FC1E0C0936D
:10CAC000720F28EC30E64AEF50E060E070E08091B1
:10CAD000B6149091B7140E941B3FC093A70F30C0AB
:10CAE000C23069F0C330D1F0C13051F58091E70B0D
:10CAF000811126C08091BA149091BB141DC0809101
:10CB0000E60B81111DC08091B50E9091B60E0E946A
:10CB1000CE428091DD0E9091DE0E0EC08091E50B2D
:10CB200081110EC08091B70E9091B80E0E94559958
:10CB30008091BC149091BD14029711F4C093EE0B38
:10CB400080910B028230A1F1833009F454C081300E
:10CB500009F074C08091E70B882309F46FC0ED9849
:10CB6000E59A1092880F1092C0141092BB14109284
:10CB7000BA141092BF1480E090E0FC01EE0FFF1F8A
:10CB8000EA58F04F11821082019688309105A9F77A
:10CB90001092870F1092860F8091C1149091C21449
:10CBA0000E943DC51092A70F1092E60B82E044C090
:10CBB0008091E60B882309F441C08091DF0E9091AB
:10CBC000E00E0E94F249809131018F77809331010C
:10CBD000809131018F7E80933101109230018091DC
:10CBE000B50E9091B60E0E943DC51092A70F1092FF
:10CBF000E50B83E021C08091E50B8823F9F080915B
:10CC0000890F90918A0F0E94F249809131018F77AC
:10CC100080933101809131018F7E80933101109298
:10CC200030018091B70E9091B80E0E943DC51092D0
:10CC3000A70F1092E70B81E080930B028091B6144E
:10CC40009091B714CF910C942B3FAF92BF92CF929B
:10CC5000DF92EF92FF920F931F93CF93DF937C01AC
:10CC60006B015A01D0E0C0E08D2F90E0F701A18167
:10CC7000B2818A159B05D0F4F601E80FF91F608197
:10CC80000AE019EA21E03327C6270C0F111D211DE8
:10CC9000311D2BBFF801C791ED91FC9111970190C7
:10CCA000F081E02DCD011995DF5FDECFED91FC9194
:10CCB00011970190F081E02D6C2FCD01DF91CF9184
:10CCC0001F910F91FF90EF90DF90CF90BF90AF90AA
:10CCD0001994CF93DF9300D01F921F92CDB7DEB788
:10CCE000FE01319625E0DF011D922A95E9F724E83F
:10CCF000298325E52C832AE22D836A834B8345E033
:10CD000050E0BF01A2DF65E070E080E090E00E94AB
:10CD1000174C80E00F900F900F900F900F90DF91C5
:10CD2000CF910895EF92FF921F93CF93DF931F92BD
:10CD3000CDB7DEB77C01162FFC0161817281F9D479
:10CD400065E070E080E090E00E94174C42E462E40D
:10CD5000C701BFDF412F60E0C701BBDF811163C0A6
:10CD600040E061E0C701B5DF81115DC040E062E0F5
:10CD7000C701AFDF811157C046E062E0C701A9DFFC
:10CD8000811151C040E063E0C701A3DF81114BC0B6
:10CD900040E064E0C7019DDF11E0811110E040E058
:10CDA00065E0C70196DF811101C01F5F40E066E0CA
:10CDB000C7018FDF811101C01F5F40E067E0C7013D
:10CDC00088DF811101C01F5F40E068E0C70181DF9B
:10CDD000811101C01F5F40E069E0C7017ADF811166
:10CDE00001C01F5F44E06AE0C70173DF811101C029
:10CDF0001F5F44E06AE0C7016CDF811101C01F5F63
:10CE000062E370E080E090E00E94174C82E8898342
:10CE100041E050E0BE016F5F7F4FC70116DF81E048
:10CE2000183011F0111180E00F90DF91CF911F9118
:10CE3000FF90EF900895CF93DF93EC010E947684EA
:10CE4000688379838A839B83CE01DF91CF91089594
:10CE5000EF92FF921F93CF93DF93CDB7DEB7659725
:10CE60000FB6F894DEBF0FBECDBF182F7B0184EE46
:10CE70009AE00E94D79281E08093120B84E690E0C2
:10CE80009093F50A8093F40A84E6E816F10418F406
:10CE900084E6E82EF12CC70164E670E00E946DC4C0
:10CEA0007093140B6093130B7093F70A6093F60A58
:10CEB0001093F10A8FEF810F823010F41230D1F00D
:10CEC00084EE9AE00E94E9928091EF0A882329F08B
:10CED00083EC95EFA8ECBFE304C084EB98ECA6E9E3
:10CEE000B0E480930E0B90930F0BA093100BB093B4
:10CEF000110B55C08091EF0A882329F084EB98EC40
:10CF0000A6E9B0E404C083EC95EFA8ECBFE38093FE
:10CF10000E0B90930F0BA093100BB093110B84EE9C
:10CF20009AE00E94F3928091120B8823C1F1109233
:10CF3000F10A8EE690E09A83898388E290E09C83F0
:10CF40008B838CE390E09E838D831D8A83E08F9397
:10CF50008DB79EB745970FB6F8949EBF0FBE8DBF95
:10CF6000ADB7BEB7119685E1FE01319601900D92E5
:10CF70008A95E1F784EE9AE00E94FD920FB6F8944C
:10CF8000DEBF0FBECDBF65960FB6F894DEBF0FBEF5
:10CF9000CDBFDF91CF911F91FF90EF90089584EE68
:10CFA0009AE065960FB6F894DEBF0FBECDBFDF9155
:10CFB000CF911F91FF90EF903ECF0F931F93CF9390
:10CFC000DF93EC01AB0160E070E02AE00E9436479D
:10CFD0008C01CE010E947E47800F911FDF91CF917F
:10CFE0001F910F9108958F929F92AF92BF92CF920F
:10CFF000DF92EF92FF920F931F93CF93DF931F92D5
:10D000001F92CDB7DEB7082E000C990BAA0BBB0BF5
:10D01000FC013197EF30F10508F066C28827E05631
:10D02000FE4F8F4F0C9494C484E08093D30A8AE01F
:10D030008093D40A86E28093D60A81E08093D90A4D
:10D040008093DA0A8093D80A42E158E120E030E088
:10D050008091D30A90E0281739070CF08CC1FA01AF
:10D0600085919491A0E0B0E0880F991FAA1FBB1F83
:10D07000F901EE0FFF1FEE0FFF1FE659F54F8083FA
:10D080009183A283B3832F5F3F4F4E5F5F4FE0CF0B
:10D0900084E08093D30A8AE08093D40A86E2809366
:10D0A000D60A81E08093D90A8093DA0A82E08093DD
:10D0B000D80A4AE058E120E030E08091D30A90E0BD
:10D0C000281739070CF057C1FA0185919491A0E017
:10D0D000B0E0880F991FAA1FBB1FF901EE0FFF1FB9
:10D0E000EE0FFF1FE659F54F80839183A283B38330
:10D0F0002F5F3F4F4E5F5F4FE0CF84E08093D40AB5
:10D1000085E28093D60A81E08093D90A88E08093F3
:10D11000DA0A83E08093D80A80E090E0FC01EE5FB9
:10D12000F74EE491DC01A552B54FEC93019688309F
:10D130009105A1F70E94FB4F1EC188E08093D30A9E
:10D1400086E08093D40A86E28093D60A81E08093B9
:10D15000D90A8093DA0A84E08093D80A42EF57E133
:10D1600020E030E08091D30A90E0281739070CF0D6
:10D1700002C1FA0185919491A0E0B0E0880F991F57
:10D18000AA1FBB1FF901EE0FFF1FEE0FFF1FE6598D
:10D19000F54F80839183A283B3832F5F3F4F4E5F10
:10D1A0005F4FE0CF88E08093D30A81E08093D40A78
:10D1B00097E29093D60A8093D90A8093DA0A85E0A1
:10D1C0008093D80A42EE57E120E030E08091D30A04
:10D1D00090E0281739070CF0CEC0FA0185919491A0
:10D1E000A0E0B0E0880F991FAA1FBB1FF901EE0F46
:10D1F000FF1FEE0FFF1FE659F54F80839183A28337
:10D20000B3832F5F3F4F4E5F5F4FE0CF82E180934C
:10D21000D30A81E08093D40A97E29093D60A809350
:10D22000D90A8093DA0A8FE08093D80A4EEB57E14F
:10D2300020E030E08091D30A90E0281739070CF005
:10D240009AC0FA0185919491A0E0B0E0880F991FEF
:10D25000AA1FBB1FF901EE0FFF1FEE0FFF1FE659BC
:10D26000F54F80839183A283B3832F5F3F4F4E5F3F
:10D270005F4FE0CFE0913E0BF0913F0B74978081C0
:10D28000918140E550E060E070E0825C944F0E9444
:10D2900050512AC182E18093D30A85E08093D40A59
:10D2A00082E28093D60A81E08093D90A8093DA0AD9
:10D2B00087E08093D80A80E993E3A0E0B0E0809310
:10D2C0006A0A90936B0AA0936C0AB0936D0AF2E01D
:10D2D0008F2E912C01E010E080E090E0A0E0BBE513
:10D2E0004CE454E060E070E024EEC22E2CE0D22E3C
:10D2F000E12CF12C9801220F331F220F331F540110
:10D30000AA0CBB1CAA0CBB1C2659354FF901B7FF50
:10D310000DC0C082D182E282F38295012659354F39
:10D32000F90140835183628373830CC0408351832E
:10D330006283738395012659354FF901C082D182EA
:10D34000E282F382880F991FAA1FBB1F0E5F1F4F37
:10D35000F2E08F0E911C22E18216910459F688E7C3
:10D360009FEFA0E0B0E08093AE0A9093AF0AA09345
:10D37000B00AB093B10A0E946A50B6C0CE010196BD
:10D380000E94E94F23E040E150E060E070E072C0AD
:10D3900084E08093D30A82E38093D40A86E2809368
:10D3A000D60A81E08093D90A8093DA0A8AE08093D2
:10D3B000D80A46EB57E120E030E08091D30A90E0B4
:10D3C00028173907C4F6FA0185919491A0E0B0E0DE
:10D3D000880F991FAA1FBB1FF901EE0FFF1FEE0F49
:10D3E000FF1FE659F54F80839183A283B3832F5F9C
:10D3F0003F4F4E5F5F4FE1CF84E08093D30A80E2DE
:10D400008093D40A86E28093D60A81E08093D90A79
:10D410008093DA0A8BE08093D80A4EEA57E120E045
:10D4200030E08091D30A90E0281739070CF0A3CFA1
:10D43000FA0185919491A0E0B0E0880F991FAA1F8E
:10D44000BB1FF901EE0FFF1FEE0FFF1FE659F54F4F
:10D4500080839183A283B3832F5F3F4F4E5F5F4FE3
:10D46000E0CFCE0101960E94E94F21E040E154E077
:10D4700060E070E0CE0101960E94C45035C084E0A7
:10D480008093D30A83E08093D40A86E28093D60AFD
:10D4900081E08093D90A8093DA0A8DE08093D80ADC
:10D4A00046EA57E120E030E08091D30A90E0281767
:10D4B00039070CF060CFFA0185919491A0E0B0E0BB
:10D4C000880F991FAA1FBB1FF901EE0FFF1FEE0F58
:10D4D000FF1FE659F54F80839183A283B3832F5FAB
:10D4E0003F4F4E5F5F4FE0CF0F900F90DF91CF9196
:10D4F0001F910F91FF90EF90DF90CF90BF90AF9072
:10D500009F908F9008950F931F93CF93DF93EC011B
:10D51000462F50E060E070E02AE00E9436478C0120
:10D52000CE010E947E47800F911FDF91CF911F9106
:10D530000F910895462F50E060E070E02AE00C94CF
:10D5400036478091D80B811180C00E94475D809141
:10D550000C02882321F080918913811105C08091EC
:10D560008813882309F471C01092891381E0809395
:10D570000C020E946E5D809187138823D1F062E9CE
:10D5800076E080918513909186130E947548809172
:10D590008813882341F062EA76E0809185139091A8
:10D5A00086130E94754880918513909186130E947E
:10D5B0007E4780918813882369F06091831370916E
:10D5C00084131616170624F485E69CE00E94CC3ED0
:10D5D00010928813809181139091821380629093AE
:10D5E00082138093811380918013882311F081E04E
:10D5F00001C080E00E94159781E080937F130E9414
:10D600005E5C80911C1381110FC080919D11882355
:10D6100059F02CE33BE544E650E060E070E085E63D
:10D620009CE00E941B3F02C00E943C5B0E94E15BA9
:10D630000E94E85C0E9476846093991170939A111D
:10D6400080939B1190939C11089508952FB7F8949F
:10D65000882381F080911E1190911F1190932D11BC
:10D6600080932C1180912E1190912F11181619066C
:10D67000ACF00FC0809120119091211190932D1149
:10D6800080932C1180912E1190912F11181619064C
:10D690002CF480912E1190912F1107C080912E11A2
:10D6A00090912F1191958195910990932F118093CD
:10D6B0002E112FBF0895AF92BF92CF92DF92EF92BB
:10D6C000FF920F931F93CF93DF931F921F92CDB7BB
:10D6D000DEB78C017A836983CE0101966C01580113
:10D6E00092E0A90EB11CE12CF12CC8010E9458C295
:10D6F000F60161916F01861731F0C8010E946AC27C
:10D70000FFEFEF1AFF0A0F5F1F4F0A151B0569F79E
:10D7100081E0EF2809F480E00F900F90DF91CF9126
:10D720001F910F91FF90EF90DF90CF90BF90AF903F
:10D730000895EF92FF920F931F93CF93DF931F9261
:10D740001F92CDB7DEB78C017B018AEA8A8341E064
:10D7500050E0BE016E5F7F4FC80177DAD701ED91CF
:10D76000FC910680F781E02DC701199582E8898335
:10D7700041E050E0BE016F5F7F4FC80166DA0F9055
:10D780000F90DF91CF911F910F91FF90EF9008952F
:10D79000CF92DF92EF92FF920F931F930E947684B5
:10D7A0006B017C0160938B1370938C1380938D13AA
:10D7B00090938E138091EF0B0E94794A80938A1385
:10D7C0009091F10B992329F091E0811190E09093D1
:10D7D0008A138091F90B9091FA0BA091FB0BB091F9
:10D7E000FC0B97018601081B190B2A0B3B0B409180
:10D7F000FD0B5091FE0B6091FF0B7091000C90910E
:10D80000F20B041715072607370760F4C092F50BD3
:10D81000D092F60BE092F70BF092F80B1092F40B0B
:10D82000892F1EC09093F30B80918A138093F20B83
:10D83000C092F50BD092F60BE092F70BF092F80B3A
:10D84000891761F0C092F90BD092FA0BE092FB0BB2
:10D85000F092FC0B91E09093F40B02C01092F40B49
:10D860001F910F91FF90EF90DF90CF9008950F934D
:10D870001F93CF93DF93EC012AE00E9436478C017F
:10D88000CE010E947E47800F911FDF91CF911F91A3
:10D890000F910895CF92DF92EF92FF920F931F9313
:10D8A000CF93DF936B01770FEE08FF08F7FE1BC0E5
:10D8B000EC016DE20E9491478C0144275527BA0183
:10D8C0004C195D096E097F092AE0CE010E94364796
:10D8D000800F911FDF91CF911F910F91FF90EF90DB
:10D8E000DF90CF9008952AE0B701A601DF91CF9194
:10D8F0001F910F91FF90EF90DF90CF900C943647DF
:10D90000CF92DF92EF92FF920F931F93CF93DF930B
:10D910008C016B01770FEE08FF08F7FE12C06DE275
:10D920000E949147EC0144275527BA014C195D0923
:10D930006E097F092AE0C8010E943647C80FD91F27
:10D9400006C02AE0B701A6010E943647EC01C801D3
:10D950000E947E478C0F9D1FDF91CF911F910F91E9
:10D96000FF90EF90DF90CF9008950F931F93CF9388
:10D97000DF931F92CDB7DEB78C0169830E9458C236
:10D980006981861729F0C8010E946AC281E001C03E
:10D9900080E00F90DF91CF911F910F910895CF9369
:10D9A0000E94EBA084E090E09093EC0B8093EB0B53
:10D9B0001092B4101092BE101092C8101092D21093
:10D9C000E0E6F0E1DF011C92179680E1A43BB80786
:10D9D000D1F78FE991E19093BD108093BC10109224
:10D9E000B7108091EA0B90919F11891718F091E080
:10D9F0009093B41028EA31E13093C7102093C610F9
:10DA00001092C1109091A811891718F091E090938D
:10DA1000BE1021EB31E13093D1102093D010109241
:10DA2000CB109091B111891718F091E09093C81024
:10DA30002AEB31E13093DB102093DA101092D510ED
:10DA40009091BA11891718F091E09093D21010922A
:10DA5000E90B20E030E0D901AD5BBD4E4D915C910A
:10DA6000415051094432510520F491E09093E90B63
:10DA700005C02D5F3F4F2837310569F79091E90BBD
:10DA8000992341F12091B2113091B3112D5D3F4F97
:10DA90003093B3112093B2112091B4113091B5118C
:10DAA000235231093093B5112093B4112091BB1149
:10DAB0003091BC112D5D3F4F3093BC112093BB11B1
:10DAC0002091BD113091BE11235231093093BE1106
:10DAD0002093BD119091BC129F3049F49091BD12DA
:10DAE0009F3029F410925F1010925E1008C02091B0
:10DAF0001A1330911B1330935F1020935E1022E1B4
:10DB000030E030935C1020935B102091EB0B309150
:10DB1000EC0BA3ECB1E141E0B683A5839C91992382
:10DB200029F0891718F040832F5F3F4F1A963796D8
:10DB300090E1E43BF90781F73093EC0B2093EB0B7A
:10DB40002131310534F080E190E09093EC0B80932B
:10DB5000EB0B0E94EB4388EB90E19093BE0F809318
:10DB6000BD0F8091BC109091BD109093BC0F80931D
:10DB7000BB0F85EB90E19093C00F8093BF0F86EBB6
:10DB800090E19093C20F8093C10F84EB90E190934A
:10DB9000C40F8093C30F82EC90E19093C80F8093E1
:10DBA000C70F8091C6109091C7109093C60F8093B5
:10DBB000C50F8FEB90E19093CA0F8093C90F80EC53
:10DBC00090E19093CC0F8093CB0F8EEB90E19093EC
:10DBD000CE0F8093CD0F8CEC90E19093D20F809379
:10DBE000D10F8091D0109091D1109093D00F80934D
:10DBF000CF0F89EC90E19093D40F8093D30F8AECF0
:10DC000090E19093D60F8093D50F88EC90E190939C
:10DC1000D80F8093D70F86ED90E19093DC0F80931F
:10DC2000DB0F8091DA109091DB109093DA0F8093E4
:10DC3000D90F83ED90E19093DE0F8093DD0F84ED9B
:10DC400090E19093E00F8093DF0F82ED90E190934D
:10DC5000E20F8093E10F2091EB0B3091EC0B2450FD
:10DC6000310960E07AE0C7E0462F50E042175307E1
:10DC700024F5CA010496789FF001799FF00D1124D4
:10DC8000E554F04FC49FC001C59F900D1124AC0115
:10DC90004E595F4E53834283DC01A05ABF4E159606
:10DCA0004D915C911697518340838F599F4E958378
:10DCB0008483B187A0876F5FD7CF81E08093ED0B1E
:10DCC000CF9108950F931F93CF93DF93FC0124818D
:10DCD00035812115310519F4FB01108211C0EA01CB
:10DCE00021972C173D0708F4E9018B01FC016081A5
:10DCF0007181AE01C8010E94D8C6C00FD11F188221
:10DD0000DF91CF911F910F9108954115510521F099
:10DD10006115710509F0D6CF0895EF92FF920F9328
:10DD20001F93CF93DF931F921F92CDB7DEB78C0165
:10DD30008CE789831A82F801E480F580FFEFEF1AFF
:10DD4000FF0AB701C8010E940146882381F0F8014B
:10DD50002081318184819581BE016F5F7F4F820F69
:10DD6000931F0E94D1C6F801F582E48281E00F90F2
:10DD70000F90DF91CF911F910F91FF90EF90089539
:10DD8000AF92BF92CF92DF92EF92FF920F931F93C9
:10DD9000CF93DF9300D01F92CDB7DEB78C014983BC
:10DDA0005A836B837C83CE0101966C01580194E009
:10DDB000A90EB11CE12CF12CC8010E9458C2F60139
:10DDC00061916F01861731F0C8010E946AC2FFEFAE
:10DDD000EF1AFF0A0F5F1F4F0A151B0569F781E055
:10DDE000EF2809F480E00F900F900F900F90DF91D3
:10DDF000CF911F910F91FF90EF90DF90CF90BF9048
:10DE0000AF900895CF92DF92EF92FF920F931F93FE
:10DE1000CF93DF93EC010091AC0FE0E0F0E020E065
:10DE200030E0A90110E0CE17DF071CF1309711F4A4
:10DE30000D32E1F0DF01A455B04FFC9080ED8F0D65
:10DE40008A30A8F4AAE0B0E00E9494C22F2DFF0C03
:10DE5000330B205331096901330FEE08FF089B0192
:10DE6000AC012C0D3D1D4E1D5F1D01C011E0319612
:10DE7000DACFCA01B901112339F0909580957095D8
:10DE800061957F4F8F4F9F4FDF91CF911F910F91E2
:10DE9000FF90EF90DF90CF9008958091F20B811169
:10DEA00005C081E09091F40B911101C080E00895CC
:10DEB00060E089E30E94A14A60E08AE30E94A14AEF
:10DEC00060E085E30E94A14A60E085E00E94A14AEB
:10DED00060E084E00E94A14A60E087E00E94A14ADD
:10DEE00059980895CF93C09111026C2F89E30E9435
:10DEF000A14A81E0C8276C2F8AE30E94A14AC093FF
:10DF00001102CF910895CF93DF93C09110026C2F2F
:10DF100089E30E94A14AD1E0DC276D2F8AE30E94A9
:10DF2000A14A6C2F85E30E94A14A6D2F85E00E94D3
:10DF3000A14A6D2F84E00E94A14A6C2F87E00E94C5
:10DF4000A14ACC2311F0599801C0599A909110021E
:10DF500081E0892780931002DF91CF910895CF93BC
:10DF6000DF938091A41381110DC01092A31310921E
:10DF7000A21381E090E09093A1138093A01380936B
:10DF8000A41336C08091A2139091A31386319105FA
:10DF90007CF18F38910534F48091A0139091A113F6
:10DFA000019609C08D3521E0920754F48091A013A9
:10DFB0009091A11302969093A1138093A01318C07F
:10DFC000863222E0920734F48091A0139091A1133D
:10DFD0000496F1CF883E93403CF48091A013909139
:10DFE000A1138A5B9F4FE7CF1092A1131092A01349
:10DFF0008ADFC091A213D091A313C93E83E0D80752
:10E0000054F01092A41354DF27E230E748EE53E0B7
:10E0100060E070E007C02FEA3FE6AE010D2E000C75
:10E02000660B770B85E69CE00E941B3F90939F1345
:10E0300080939E138091A0139091A1138C0F9D1F2C
:10E040009093A3138093A213DF91CF910895CF9360
:10E05000DF938091A807882319F0DF91CF917FCFBC
:10E06000C0919E13D0919F13BE0185E69CE00E9453
:10E07000B43E882329F0BE0185E69CE00E94CC3E98
:10E08000DF91CF9115CFCF93C0919B136C2F70E090
:10E0900088E00E940C4B89E180939A1390910F02C3
:10E0A000992311F0CD5F01C0C350C0939B138091A1
:10E0B0009B13873970F0992321F08FEF80939B1386
:10E0C00008C08D3D30F086E980939B1388E78093EC
:10E0D0009A1380919B138F3F19F410920F0205C081
:10E0E0008A3118F481E080930F0240919A1350E036
:10E0F00060E070E023E430E785E69CE00E941B3F8F
:10E100009093681480936714CF910895CF92DF9213
:10E11000EF92FF92CF93DF93EC019C01AFEFB0E061
:10E120000E94C6C2CC24CA9423E0D22EE12CF12C4A
:10E13000A70196010E9478C2B90188E00E940C4BA9
:10E140009E01A4E6B0E00E94C6C2A70196010E940B
:10E1500078C280917213821320937213DF91CF9152
:10E16000FF90EF90DF90CF900895CF93DF93C09111
:10E170006714D0916814BE0185E69CE00E94B43E0D
:10E18000882329F0BE0185E69CE00E94CC3E60E039
:10E1900088E00E94A14A809187138823D1F0809162
:10E1A0006914882319F06EE479E10DC0809166143A
:10E1B000882319F065E379E106C08091A5138111E8
:10E1C00008C066E279E180918513909186130E94E0
:10E1D0009A481092691410926614DF91CF910895B5
:10E1E00061E088E00E94A14A80918713882361F052
:10E1F00080916914811108C068E179E180918513EB
:10E20000909186130C949A48089580916914811115
:10E2100010C0ABDF81E0809369148091871388235D
:10E2200041F06DE779E180918513909186130E940A
:10E230009A4880919913882329F060E088E00E9431
:10E24000A14A01C0CDDF9091991381E08927809385
:10E250009913882329F040916E1350916F1304C0D5
:10E26000409170135091711360E070E025E031E748
:10E2700085E69CE00E941B3F90936814809367148E
:10E280000895CF938091971381110FC081E08093FF
:10E29000971380918713882341F066EE78E180918F
:10E2A0008513909186130E949A48C09196136C2F03
:10E2B00085E00E94A14A4091771350E060E070E051
:10E2C00021E431E785E69CE00E941B3F9093951383
:10E2D0008093941381E06C2F682760939613CF91FD
:10E2E00008958091070180FF1BC0809187138823C8
:10E2F00051F083E39CE00E94A894811108C08091B2
:10E300003F0C811104C083E39CE00C9495946DE56F
:10E3100078E180918513909186130E949A48F3CFFB
:10E3200008958091070181FF1BC080918713882386
:10E3300051F082E09CE00E94A894811108C0809175
:10E340000E0C811104C082E09CE00C94959460E373
:10E3500078E180918513909186130E949A48F3CFBB
:10E3600008958091070180FF17C08091871388234B
:10E3700031F083E39CE00E94A894882321F083E39A
:10E380009CE00C94BC9467E478E1809185139091B3
:10E3900086130E949A48F3CF08958091070181FF68
:10E3A00017C080918713882331F082E09CE00E949F
:10E3B000A894882321F082E09CE00C94BC946AE14C
:10E3C00078E180918513909186130E949A48F3CF4B
:10E3D000089560919C1370919D1385E69CE00E94C6
:10E3E000B43E81112EC060E089E30E94A14A60E042
:10E3F0008AE30E94A14A60E085E30E94A14A60E0AE
:10E4000085E00E94A14A60E084E00E94A14A60E0A9
:10E4100087E00E94A14A599880917413882319F0CB
:10E4200023E83FE602C022E73FE642E350E060E037
:10E4300070E085E69CE00E94233F90939D138093BB
:10E440009C13089560E08AE30C94A14A61E08AE39A
:10E450000C94A14A0F931F93CF93DF938C01C1E0DB
:10E46000D0E00C171D079CF0F1DF64E670E080E05F
:10E4700090E00E94174CE6DFC017D10734F46AE53C
:10E4800070E080E090E00E94174C2196EACFDF9187
:10E49000CF911F910F91089583E090E0DBCF82E050
:10E4A00090E0D8CF81E090E0D5CF60E089E30C9494
:10E4B000A14A61E089E30C94A14A0F931F93CF9383
:10E4C000DF938C01C1E0D0E00C171D079CF0F1DF59
:10E4D00064E670E080E090E00E94174CE6DFC01731
:10E4E000D10734F46AE570E080E090E00E94174CB8
:10E4F0002196EACFDF91CF911F910F91089583E08C
:10E5000090E0DBCF82E090E0D8CF81E090E0D5CF03
:10E510006091721370E088E00E940C4B8091871329
:10E52000882341F067E679E1809185139091861305
:10E530000C949A4808951092981380919507811130
:10E5400004C060E084E00E94A14A80918713882380
:10E5500041F065E079E180918513909186130C94E8
:10E560009A48089581E080939813809195078111CE
:10E5700006C060918F1370E084E00E940C4B809184
:10E580008713882341F063EF78E1809185139091A0
:10E5900086130C949A480895CF93DF93C0919C13EF
:10E5A000D0919D13BE0185E69CE00E94B43E882375
:10E5B00051F0BE0185E69CE00E94CC3E10929D1376
:10E5C00010929C1375DC80916913882319F0DF91F8
:10E5D000CF91C8CFDF91CF91089510929507809188
:10E5E0009813811104C060E084E00C94A14A60910A
:10E5F0008F1370E084E00C940C4BCF93DF9360E0BA
:10E6000085E00E94A14A8091971381110BC08091EF
:10E61000A2079091A307DC01ED91FC9104ACF5AD4C
:10E62000E02D1995C0919413D0919513BE0185E604
:10E630009CE00E94B43E882329F0BE0185E69CE060
:10E640000E94CC3E80918713882379F02091971304
:10E650008091851390918613222319F06AED78E159
:10E6600002C06EEC78E10E949A4810929713DF91F5
:10E67000CF91089561E085E00E94A14A8091A207B0
:10E680009091A307DC01ED91FC9104ACF5ADE02D78
:10E69000199580918713882341F063EC78E180918C
:10E6A0008513909186130C949A48089560E085E351
:10E6B0000E94A14A8091A2079091A307DC01ED91ED
:10E6C000FC9100ACF1ADE02D199580918713882362
:10E6D00041F067EB78E180918513909186130C945B
:10E6E0009A48089561E085E30E94A14A8091A207BB
:10E6F0009091A307DC01ED91FC9100ACF1ADE02D10
:10E70000199580918713882341F06CEA78E1809114
:10E710008513909186130C949A4808958F929F9236
:10E72000AF92BF92CF92DF92EF92FF9285E40E9468
:10E73000D34BBC01990F880B990B0E9435C120E087
:10E7400030E040E85AE30E9494C120E030E040EA23
:10E7500050E40E9494C16B017C0180910E028823D9
:10E7600051F0C0929013D0929113E0929213F092D4
:10E77000931310920E0226E636E646E65FE36091BA
:10E7800090137091911380919213909193130E9422
:10E7900094C14B015C0120ED3CEC4CEC5DE3C70106
:10E7A000B6010E9494C19B01AC01C501B4010E9455
:10E7B000D6C26093901370939113809392139093A9
:10E7C00093132DE33CE248E450E40E9494C12AE90B
:10E7D00039E949E95EE30E94D6C2FF90EF90DF90ED
:10E7E000CF90BF90AF909F908F90089580910D0231
:10E7F000882351F093DF20E030E040E050E40E94B5
:10E800002FC187FF39C0089589DF20E030E04AE753
:10E8100054E40E9494C10E94A7C3209167133091D1
:10E8200068134091A8076217730710F4442351F14D
:10E83000442309F445C072DF20E030E04AE754E4A5
:10E840000E9494C10E94A7C320916713309168135E
:10E8500062177307A8F11092A80781E08093A707B9
:10E8600080918713882361F164E778E180918513B3
:10E87000909186130C949A4810920D0281E0809337
:10E88000A707089581E08093A8071092A7078091B9
:10E890008713882391F063E978E180918513909143
:10E8A00086130E9476480E940E9560E978E1809177
:10E8B0008513909186130E949A480E94355CC7CBBD
:10E8C0000895CF93DF938091070180FD2AC0C09106
:10E8D0003E07D0913F0780914207882371F08EE375
:10E8E0000E94D34B813092402CF010923F0710923F
:10E8F0003E070AC081E090E003C08EE30E94D34B44
:10E9000090933F0780933E0780913E0790913F0789
:10E910008C179D0719F41092400703C081E0809383
:10E920004007DF91CF910895CF93DF938091070146
:10E9300081FD2AC0C0913807D091390780913C07EA
:10E94000882371F08FE30E94D34B813092402CF0EA
:10E9500010923907109238070AC081E090E003C096
:10E960008FE30E94D34B90933907809338078091AF
:10E970003807909139078C179D0719F410923A07C0
:10E9800003C081E080933A07DF91CF9108952F92E1
:10E990003F924F925F926F927F928F929F92AF922F
:10E9A000BF92CF92DF92EF92FF920F931F93CF937C
:10E9B000DF9300D01F92CDB7DEB75C010E94355CBB
:10E9C00041DD77DD80918513909186130E947E470B
:10E9D0000E94025724E0A216B10409F49CC00CF076
:10E9E0004FC0A3E0AA16B10409F03CC18CE190E04D
:10E9F0000E94A8C49C838B8383E696E0AB81BC8194
:10EA000011969C938E931396BC92AE92129781E0CE
:10EA10009FEF15969C938E9314978FEF90E0179627
:10EA20009C938E93169719961C921E92189758963F
:10EA30001C925897CD010E94D64187E596E0EB8164
:10EA4000FC8191838083E0913D0FF0913E0FD08C4B
:10EA5000009120111091211116950795E0901E113B
:10EA6000F0901F11F694E7946CEB7AE18091851396
:10EA7000909186130E949A48812C9924939412C1F4
:10EA8000B5E0AB16B10409F4A6C0E6E0AE16B104D9
:10EA900009F0E8C08CE190E00E94A8C49C838B83BD
:10EAA00083E696E0AB81BC8111969C938E9313967E
:10EAB000BC92AE92129781E09FEF15969C938E9335
:10EAC00014978FEF90E017969C938E931697199654
:10EAD0001C921E92189758961C925897CD010E942E
:10EAE000D64187E596E0EB81FC8191838083E091BC
:10EAF0009307F0919407D08C00915F1110916011F1
:10EB000016950795E0905D11F0905E11F694E794EC
:10EB10006FEE7AE1A0C08CE190E00E94A8C49C83D3
:10EB20008B8383E696E0AB81BC8111969C938E9398
:10EB30001396BC92AE92129781E09FEF15969C932C
:10EB40008E9314978FEF90E017969C938E93169761
:10EB500019961C921E92189758961C925897CD01A0
:10EB60000E94D64187E596E0EB81FC81918380830A
:10EB7000009135111091361116950795E0903311DB
:10EB8000F0903411F694E7948091BD128C5082304D
:10EB900040F4E091A407F091A507D08C6FE27BE1EF
:10EBA0005AC080910613823009F07AC08091BB125E
:10EBB0008C3009F075C0E0919307F0919407D08CE8
:10EBC0006FE07BE180918513909186130E949A48B3
:10EBD0008824839466C08CE190E00E94A8C49C8342
:10EBE0008B8383E696E0AB81BC8111969C938E93D8
:10EBF0001396BC92AE92129781E09FEF15969C936C
:10EC00008E9314978FEF90E017969C938E931697A0
:10EC100019961C921E92189758961C925897CD01DF
:10EC20000E94D64187E596E0EB81FC819183808349
:10EC3000E091A007F091A107D08C00914A111091AA
:10EC40004B1116950795E0904811F0904911F694F4
:10EC5000E7946FEC7AE180918513909186130E947E
:10EC60009A481EC063EA7AE18091851390918613D9
:10EC70000F900F900F900F90DF91CF911F910F91F8
:10EC8000FF90EF90DF90CF90BF90AF909F908F90CC
:10EC90007F906F905F904F903F902F900C949A4888
:10ECA000812C912C0E94025766E97AE180918513AC
:10ECB000909186130E949A486AE87AE180918513C0
:10ECC000909186130E947648B801809185139091A7
:10ECD00086130E94806C6EE77AE180918513909193
:10ECE00086130E947648B701809185139091861310
:10ECF0000E94806C62E77AE180918513909186137F
:10ED00000E9476488D2D0E94D8568091851390914F
:10ED100086130E947E47AB81BC81ED91FC911197D7
:10ED20000280F381E02DCD011995CA2C8A2D0E9415
:10ED3000F3408D3D9540A8F464E378E08A2D0E946D
:10ED4000EB40EB81FC81F78AE68AB70182810E9461
:10ED500003416CED75E08A2D0E94EF40DD20C1F08B
:10ED60001AC064E873E08A2D0E94EF40AB81BC8139
:10ED700057961C930E935697B80112968C910E9449
:10ED800003416CED75E08A2D0E94EB40DD2019F007
:10ED90003324339401C0312C21E02983212C2A8390
:10EDA0000E94D4608091C910882359F1AB81BC8145
:10EDB000ED91FC9111976091CE107091CF10019060
:10EDC000F081E02DCD0119958C2D0E94F3408D3DF1
:10EDD000B5E09B075CF48438E3E09E0784F08C0187
:10EDE0008D3D954074F00CED15E00BC07C01853332
:10EDF00098403CF064E3E62E68E0F62E02C004E89A
:10EE000013E02A8121111FC08091BF108823C9F10E
:10EE1000E091C610F091C710858196814091C21093
:10EE20005091C3109C0121533109421753074CF1F3
:10EE3000C196841795072CF10E9476846415750598
:10EE400086059705F0F08091BF108823C1F04091AE
:10EE5000C2105091C310E091C610F091C710858187
:10EE600096819C01285C3109421753072CF0885386
:10EE70009F4F841795071CF481E0382605C021E0D8
:10EE80002A83222009F47CC0332009F445C0DD2008
:10EE9000F9F064E873E08C2D0E94EF40992009F4AA
:10EEA00058C06091D7127091D81241E08C2D0E9409
:10EEB000AA400E94AD97AB81BC8112968C910E94B2
:10EEC000F34008171907ACF38C2D0E947C4041C019
:10EED00064E378E08C2D0E94EB409920B1F06091C2
:10EEE000D7127091D81240E08C2D0E94AA400E9447
:10EEF000AD97AB81BC8112968C910E94F3408E1528
:10EF00009F05ACF38C2D0E947C40EB81FC81F78A3D
:10EF1000E68AB701828110C0DD20B1F064E378E0B9
:10EF20008C2D0E94EB40AB81BC815796FC92EE92F7
:10EF30005697B70112968C910E9403416CED75E0D3
:10EF40008C2D0E94EF4012C064E873E08C2D0E946B
:10EF5000EF40EB81FC81178B068BB80182810E9408
:10EF600003416CED75E08C2D0E94EB400E9476848D
:10EF70002B013C01F8EC4F0E511C611C711C1A82D4
:10EF800029812223D1F18091B5108823A1F14091EC
:10EF9000B8105091B910E091BC10F091BD1085816E
:10EFA00096819C01285C3109421753072CF0885345
:10EFB0009F4F84179507FCF481E0D8268091851334
:10EFC00090918613DD2039F063E67AE10E949A4839
:10EFD00082E090E006C061E57AE10E949A4881E013
:10EFE00090E038DA0E947684AB81BC815896DC923E
:10EFF0002224239403C0212C1EC0212C8091B51003
:10F00000882309F48AC2E091BC10F091BD1085817B
:10F0100096814091B8105091B9109C01215331094B
:10F02000421753070CF479C2C19621E02983841753
:10F0300095070CF472C20E94E9430E94C86B85E6F2
:10F040009CE00E942B3F8091F20B882309F4A8CE0C
:10F050008091F40B882309F4A3CE0E94C86B0E9410
:10F060004D6F8823D1F384E0A816B104D9F134F4AC
:10F07000B3E0AB16B10409F438C1C4C1E5E0AE1683
:10F08000B10409F4CDC0F6E0AF16B10409F0BAC17D
:10F090001093CB120093CA12F092CD12E092CC12D0
:10F0A000D092CE12B8018CE291E00E945B6BB70166
:10F0B0008EE291E00E945B6B6D2D80E391E00E94F7
:10F0C000B56CB80186E00E942140B70186E00E943D
:10F0D0000640E0919307F0919407D08E6CED75E0B7
:10F0E00086E091C08820C1F01093CB120093CA1221
:10F0F000F092CD12E092CC12D092CE12B8018CE2F6
:10F1000091E00E945B6BB7018EE291E00E945B6B25
:10F110006D2D80E391E017C01093BF120093BE12D3
:10F12000F092C112E092C012D092C212B80180E2F5
:10F1300091E00E945B6BB70182E291E00E945B6B01
:10F140006D2D84E291E00E94B56CB80184E00E94CC
:10F150002140B70184E00E940640882049F0E091F8
:10F160009307F0919407D08E6CED75E084E04BC06E
:10F17000E091A407F091A507D08E8091BD128D304B
:10F1800029F4E091A613F091A713D08E6CED75E0F1
:10F1900084E00E94034166E970E080E090E00E9414
:10F1A000174C8091BD128D3011F584E00E94F34020
:10F1B000A091A407B091A5078D3D95404CF0ED912D
:10F1C000FC9111970190F081E02D6FEF7FEF08C067
:10F1D000ED91FC9111970190F081E02D61E070E0DC
:10F1E000CD0119958091A4079091A5076FC08091DA
:10F1F000A4079091A507DC01ED91FC910480F581B5
:10F20000E02D1995FFC00E94034166E970E080E09F
:10F2100090E00E94174C8091930790919407EBCF58
:10F220001093C6120093C512F092C812E092C71252
:10F23000D092C912B80187E291E00E945B6BB701DE
:10F2400089E291E00E945B6B6D2D8BE291E00E9460
:10F25000B56CB80185E00E942140B70185E00E94AD
:10F260000640E091A007F091A107D08E6CED75E00B
:10F2700085E00E94034166E970E080E090E00E9432
:10F28000174C8091BC128D3059F585E00E94F340F7
:10F29000A091A007B091A1078D3D95404CF0ED9154
:10F2A000FC9111970190F081E02D6FEF7FEF08C086
:10F2B000ED91FC9111970190F081E02D61E070E0FB
:10F2C000CD0119958091A0079091A107DC01ED91E6
:10F2D000FC910190F081E02D60E070E0199592C002
:10F2E0008091A0079091A10786CF1093DA12009326
:10F2F000D912F092DC12E092DB12D092D312B80154
:10F300008BE391E00E945B6BB7018DE391E00E947B
:10F310005B6B6D2D85E391E00E94B56CB80183E0D5
:10F320000E942140B70183E00E9406408091D312E1
:10F33000E0913D0FF0913E0F808F8091D3120E949B
:10F34000266B83E00E94F3402091D312222369F1BF
:10F35000B9E0BC1538F0209120113091211136957B
:10F36000279502C02EEE32E08217930709F44AC0B7
:10F370006091D7127091D81241E083E00E94AA40B8
:10F380000E94AD97EB81FC8182810E94F3400817B7
:10F390001907B4F383E00E947C40AB81BC8157968F
:10F3A0001C930E935697B80129C0A9E0AC1508F438
:10F3B000B6C020911E1130911F11369527958217E6
:10F3C000930701F16091D7127091D81240E083E069
:10F3D0000E94AA400E94AD97EB81FC8182810E942D
:10F3E000F3408E159F05B4F383E00E947C40AB810F
:10F3F000BC815796FC92EE925697B70112968C916B
:10F400000E94034180918513909186130E947E474C
:10F410000E940257B4E0AB16B10499F03CF4F3E05B
:10F42000AF16B10449F565ED79E120C025E0A216DB
:10F43000B104D1F086E0A816B104F1F465E07AE1F8
:10F4400015C08091BD128C50823018F467E37AE1C8
:10F450000DC080910613823079F48091BB128C30FC
:10F4600059F46EE17AE102C06CEE79E18091851386
:10F47000909186130E949A480E9402576AEC79E1A3
:10F4800080918513909186130E949A486EEB79E1E2
:10F4900080918513909186130E947648B8018091DF
:10F4A0008513909186130E94806C62EB79E18091C4
:10F4B0008513909186130E947648B7018091851339
:10F4C000909186130E94806C66EA79E180918513A1
:10F4D000909186130E9476488D2D0E94D856809177
:10F4E0008513909186130E947E470F900F900F9086
:10F4F0000F90DF91CF911F910F91FF90EF90DF90D0
:10F50000CF90BF90AF909F908F907F906F905F90C3
:10F510004F903F902F900C94557219828CCD2AEC0D
:10F5200038E04DCFCF93DF93CDB7DEB728970FB636
:10F53000F894DEBF0FBECDBF8091A5138823D9F10B
:10F540001092A51329D881E0809303028091A60729
:10F55000882389F167E979E1809185139091861379
:10F560000E947648E091EE0BE4300CF0E0E080EF92
:10F5700095E09A8389838CEE95E09C838B8387EE5C
:10F5800095E09E838D8382EE95E098878F83EE0FC2
:10F59000FF0BEC0FFD1F61817281809185139091AB
:10F5A000861328960FB6F894DEBF0FBECDBFDF914D
:10F5B000CF910C949A4828960FB6F894DEBF0FBEF0
:10F5C000CDBFDF91CF9108958091A8139091A91399
:10F5D00091609093A9138093A81308958091C91303
:10F5E000811112C08AE09AEAA1E0BB27ABBFFC01FF
:10F5F0006791769182E00E943C4081E08093D51330
:10F600001092D9131092D613089581E08093AE130F
:10F610006CED75E00C943C406CED75E080E00C9472
:10F620003C4081E20E94794A21E0892B09F420E0E4
:10F63000822F089580912A07882309F44BC0809176
:10F64000D90B882309F446C081E08093D60BE9DF0B
:10F65000882329F080912D078823D9F106C0809155
:10F660002B07811105C080912A070E94F36731C0E2
:10F6700090912A07963069F5823081F08330D1F07D
:10F68000813039F5E0913E0BF0913F0B749780810A
:10F69000918145E550E060E070E017C0E0913E0BDD
:10F6A000F0913F0B7497808191814AE550E060E0D2
:10F6B00070E00BC0E0913E0BF0913F0B749780819E
:10F6C00091814FE550E060E070E0825C944F0E94D1
:10F6D0005051E4C508958091DC13882339F080915E
:10F6E000DB13882319F081E08093D30B80911507F9
:10F6F00090911607DC01ED91FC91008CF18DE02DCD
:10F7000019958091CF1381110E9480868091CE132C
:10F71000882391F061E088E00E94A14A4091CC13D7
:10F720005091CD1360E070E022EF33E88091130731
:10F73000909114070E941B3F8091DC13882321F0D5
:10F740008091DB13811101C075DF8091DB13882369
:10F7500079F08091DC13882359F08091D2138823AB
:10F7600039F0E091D013F091D11382810E948A4048
:10F770000C9400878091D80B811158C052DF8823E8
:10F78000F1F081E08093D80B8091150790911607D6
:10F79000DC01ED91FC910488F589E02D19953ED6A8
:10F7A00022E332E848E95AE360E070E08091130711
:10F7B000909114070E941B3F0E9400870AC080910D
:10F7C000DB13882339F18091DC13882319F00E9420
:10F7D000EA8630CF0E94D4868091D213882339F0F4
:10F7E000E091D013F091D11382810E948A40409120
:10F7F000CA135091CB1314161506BCF4052E000C39
:10F80000660B770B2BE63BE780911307909114076B
:10F810000C941B3F8091D213882339F0E091D013D0
:10F82000F091D11382810E948A4055CF08950F93A1
:10F830001F932091C913211135C04AE05AEA61E0B3
:10F8400077279C01220F331F820F931F092E000C74
:10F85000AA0BBB0B0296A11DB11D840F951FA61FFD
:10F86000B71FABBFFC0187910AE01AEA21E03327FA
:10F870004091D91393E0499FA0011124052E000C5B
:10F88000660B770B4E5F5F4F6F4F7F4F040F151F57
:10F89000261F371F2BBFF8010791801718F01F9103
:10F8A0000F919CCE1F910F910895833091F028F411
:10F8B000813049F0823051F00895853081F060F058
:10F8C000863081F0089589E090E00EC08AE090E0F3
:10F8D0000BC08BE090E008C08CE090E005C08DE0AC
:10F8E00090E002C08EE090E0A2CF8F929F92AF9204
:10F8F000BF92CF92DF92EF92FF920F931F93CF931D
:10F90000DF93EC01A62E8091C91381116BC04AE0F0
:10F910005AEA61E077276E01CC0CDD1CCC0EDD1EAF
:10F920000D2C000CEE08FF08D701C6010296A11DA0
:10F93000B11D480F591F6A1F7B1F6BBFFA018791CA
:10F940004AE05AEA61E07727B090D91393E0B99E74
:10F9500080011124012E000C220B330B0E5F1F4F70
:10F960002F4F3F4F400F511F621F731F6BBFFA0194
:10F970004791481708F036C08090D7139090D8135D
:10F980000091C2131091C313B401C8010E94B43E88
:10F99000882321F0B401C8010E94CC3E8AE09AEA93
:10F9A000A1E0BB278C0D9D1DAE1DBF1DABBFFC0193
:10F9B0006791769182E00E943C40B092D613C0934A
:10F9C000D913AA2079F01092D5132EEE3AE742E32C
:10F9D00050E060E070E0C8010E941B3F9093D81394
:10F9E0008093D713DF91CF911F910F91FF90EF90EC
:10F9F000DF90CF90BF90AF909F908F900895CF925F
:10FA0000DF92EF92FF928091C913811134C08091EF
:10FA1000C813882381F161E08EE090E066DF609199
:10FA2000C6137091C713CB01A0E0B0E0C090C4131F
:10FA3000D090C513E12CF12CC816D906EA06FB06B6
:10FA400064F4BC01CD016C197D098E099F090E94E7
:10FA50001247C60ED71EE81EF91E2FEF3CE7B7016E
:10FA6000A6018091C2139091C3130E941B3F9093F3
:10FA7000C1138093C013FF90EF90DF90CF90089553
:10FA8000CF92DF92EF92FF928091C913811134C01F
:10FA90008091BF13882381F161E08DE090E025DF44
:10FAA0006091BD137091BE13CB01A0E0B0E0C09097
:10FAB000BB13D090BC13E12CF12CC816D906EA0672
:10FAC000FB0664F4BC01CD016C197D098E099F0908
:10FAD0000E941247C60ED71EE81EF91E20E43DE71D
:10FAE000B701A6018091C2139091C3130E941B3FDE
:10FAF0009093BA138093B913FF90EF90DF90CF905B
:10FB00000895CF92DF92EF92FF928091C9138111F5
:10FB100034C08091B813882381F161E08CE090E0DB
:10FB2000E4DE6091B6137091B713CB01A0E0B0E0B2
:10FB3000C090B413D090B513E12CF12CC816D9069F
:10FB4000EA06FB0664F4BC01CD016C197D098E093F
:10FB50009F090E941247C60ED71EE81EF91E21E813
:10FB60003DE7B701A6018091C2139091C3130E9493
:10FB70001B3F9093B3138093B213FF90EF90DF90ED
:10FB8000CF9008958091C91381112CC08091B11339
:10FB9000882341F08091B813811104C081E08093E3
:10FBA000B813AFDF8091B013882361F08091C9133F
:10FBB000811108C08091BF13811104C081E080933E
:10FBC000BF135EDF8091AF13882361F08091C9136A
:10FBD000811108C08091C813811104C081E0809315
:10FBE000C8130DCF08951092AE1325E03BE744EF04
:10FBF00051E060E070E08091C2139091C3130E94C5
:10FC00001B3F9093AD138093AC1308958091C9135B
:10FC100081110AC08091AE13882331F060ED77E046
:10FC200081E00E943C40DFCF08950F931F93CF9354
:10FC3000DF93EC017093C3136093C2134093C91315
:10FC400081E090E00E94A8C48C010E94D6411093EC
:10FC5000D4130093D31391E09093AE139093D513E4
:10FC60001092AD131092AC131092D8131092D713B8
:10FC70001092D9131092D6131092AB1324EF31E0E7
:10FC80003093B5132093B41328EB3BE03093B713B4
:10FC90002093B61320E233E03093BC132093BB13C0
:10FCA0002CEA3DE03093BE132093BD1328E037E0EB
:10FCB0003093C5132093C41324E931E13093C71363
:10FCC0002093C6131092B1131092B0131092AF1379
:10FCD0001092B8131092BF131092C8131092AA1367
:10FCE0001092B3131092B2131092BA131092B91368
:10FCF0001092C1131092C013988399839A83DF9155
:10FD0000CF911F910F910895089508950895089532
:10FD10000895623039F0633041F0613041F440932E
:10FD2000B11308954093B01308954093AF1308950D
:10FD3000623069F06330A1F06130D1F45093B513B3
:10FD40004093B4133093B7132093B6130895509390
:10FD5000BC134093BB133093BE132093BD1308957F
:10FD60005093C5134093C4133093C7132093C61305
:10FD70000895FC01858108950895089508950895D2
:10FD80002091C913211102C0FC01628308952091C2
:10FD9000C913211102C0FC01648308952091C91385
:10FDA000211102C0FC016383089508950895809194
:10FDB000C913811101C029CC0895089580E00895E8
:10FDC0000895089508950895089508958091C91398
:10FDD000811103C08FE090E02ACD08952091C913CE
:10FDE000211107C0FC018481882319F082E090E092
:10FDF0001ECD08952091C913211107C0FC018381F4
:10FE0000882319F081E090E012CD08958091C91304
:10FE1000811103C08BE090E00ACD08958091C91351
:10FE2000811104C060E080E190E05FCD0895809191
:10FE3000C913811104C060E08FE090E056CD0895B1
:10FE40008091C913811126C06330A1F028F461307C
:10FE500049F0623059F008956530A1F078F06630CD
:10FE6000A9F0089560E089E090E013C060E08AE0C6
:10FE700090E00FC060E08BE090E00BC060E08CE0B1
:10FE800090E007C060E08DE090E003C060E08EE0AD
:10FE900090E02BCD08958091C913811126C0633065
:10FEA000A1F028F4613049F0623059F008956530CE
:10FEB000A1F078F06630A9F0089561E089E090E063
:10FEC00013C061E08AE090E00FC061E08BE090E059
:10FED0000BC061E08CE090E007C061E08DE090E055
:10FEE00003C061E08EE090E000CD08952091C91339
:10FEF000211108C0FC018281882321F061E088E0A3
:10FF000090E0F3CC08952091C913211108C0FC01A1
:10FF10008481882321F061E082E090E0E6CC0895BE
:10FF20002091C913211108C0FC018381882321F08D
:10FF300061E081E090E0D9CC08958091C9138111EE
:10FF400004C061E086E090E0D0CC08958091C913B0
:10FF5000811104C060E08BE090E0C7CC08958091EF
:10FF6000C913811104C061E087E090E0BECC089520
:10FF70008091C913811104C061E085E090E0B5CCA7
:10FF800008958091C913811104C061E08AE090E076
:10FF9000ACCC0895CF93DF93FC0125812223A1F1FE
:10FFA000EC018091C91381112EC06091B213709140
:10FFB000B3138091C2139091C3130E94CC3E109250
:10FFC000B8138091C91381110CC06091B91370915D
:10FFD000BA138091C2139091C3130E94CC3E109229
:10FFE000BF138091C91381110CC06091C01370912F
:10FFF000C1138091C2139091C3130E94CC3E109202
:020000021000EC
:10000000C8131092AA131D82DF91CF910895CF9348
:10001000DF93FC01258121111EC0EC018091C913E1
:10002000811117C08091AA13811113C022EC3DE702
:1000300048EB5BE060E070E08091C2139091C313E5
:100040000E941B3F9093B3138093B21381E080937F
:10005000AA1381E08D83DF91CF910895862F90912F
:10006000C913911101C021CC0895CF93C1E08091B3
:10007000C913811102C08C2F18DCCF5FC730B9F7CC
:10008000CF9108958091C913882329F06CED75E014
:1000900081E00C943C4084E090E0C9CB8091C9138E
:1000A000882329F068EE73E081E00C943C4060E026
:1000B00084E090E01ACC8091C91381111BC080911B
:1000C000AE138823B9F068EE73E081E00E943C40F3
:1000D0001092AE1325E03BE748E95AE360E070E098
:1000E0008091C2139091C3130E941B3F9093AD1354
:1000F0008093AC1308956CED75E080E00C943C4067
:1001000024EF31E0DB010E94A2C42FEF30E040E099
:1001100050E00E9478C2CA01B90164527A4F8F4FF1
:100120009F4F80E00C943C408091C913882331F0AC
:1001300060ED77E081E00E943C4055CD61E083E0D6
:1001400090E0D3CB2091C913211108C02091AB13AB
:10015000222321F002965ADD1092AB1308952091CC
:10016000C913222389F06FE676E080E00E943C40CC
:100170002CE03BE742E350E060E070E08091C21386
:100180009091C3130C941B3F2091AB13211105C018
:1001900002963CDD81E08093AB13089580E00E94DD
:1001A000634081E00E9463408091C913811103C0C4
:1001B00082E00E9463406CED75E080E00E943C406C
:1001C0006CED75E081E00E943C408091C913811183
:1001D0000CC08AE09AEAA1E0BB27ABBFFC016791A3
:1001E000769182E00E943C40F9C90895FC01848523
:1001F0009585978386838685978591878087808973
:10020000918993878287808D918D938B828B828D4C
:10021000938D958B848B848D958D978B868B08958C
:10022000FC01808991899387828782899389958748
:1002300084878489958997878687089526E00C941A
:10024000144A80911202882311F0599801C0599ADA
:100250009091120281E089278093120208951092F2
:100260009D1110921B071092120710921C071092FA
:100270001D0710921E0710921F0781E08093D60B76
:10028000409126075091270760E070E02EE431E8A6
:1002900080911307909114070C941B3F8091D90B08
:1002A000882361F18091D70A81111CC01092190B2B
:1002B00010921A0B10921B0B10921C0B10921D0B1C
:1002C00010921E0B1092210B8091D40B9091D50BA4
:1002D000DC01ED91FC910190F081E02D19951092D7
:1002E000D60B08952EE431E845E050E060E070E080
:1002F00080911307909114070C941B3F089560910F
:10030000E7137091E81380911307909114070E94EE
:10031000B43E882319F081E08093E613089560E0ED
:1003200087E00E94A14A1092D70B089561E087E010
:100330000E94A14A81E08093D70B0895CF93DF9369
:100340008091F413811110C084EF91E09093F31326
:100350008093F2138BE290E09093F1138093F0136B
:1003600081E08093F41320C08091F0139091F113F9
:100370008532910514F0049709C08331910514F07A
:10038000029704C0823091052CF001979093F113ED
:100390008093F0138091F0139091F11397FF04C0B4
:1003A0001092F1131092F013C091EF13CC2311F0BF
:1003B000B6DF01C0BBDF81E08C278093EF13C091D3
:1003C000F213D091F3131C161D0654F01092F4137F
:1003D000A6DF2EE032E84AEF50E060E070E007C0B0
:1003E0002EE931E8AE010D2E000C660B770B8091E3
:1003F0001307909114070E941B3F9093EE13809374
:10040000ED138091F0139091F113C81BD90BD09389
:10041000F313C093F213DF91CF9108950F931F93BD
:10042000CF93DF938091D80B882329F0DF91CF9170
:100430001F910F9183CF0091ED131091EE13C09196
:100440001307D0911407B801CE010E94B43E88234F
:1004500021F0B801CE010E94CC3EDF91CF911F91D7
:100460000F915DCFCF92DF92EF92FF921092D80B57
:1004700020911707309118074091190750911A07DA
:1004800060911C0770911D0780911E0790911F07B6
:100490000E94D5C26B017C0120E030E0A9010E94DE
:1004A0002FC187FD09C0C0921C07D0921D07E092A2
:1004B0001E07F0921F0708C010921C0710921D071C
:1004C00010921E0710921F07FF90EF90DF90CF90C1
:1004D000A5CFEF92FF921F93CF93DF9300D0CDB7BC
:1004E000DEB784E689838CE38A8388E28B8310916C
:1004F000E9131330E8F4E12EF12C10FF02C00FDFF6
:1005000001C014DFE1E0F0E0EC0FFD1FEE0DFF1D78
:10051000408150E060E070E029E632E88091130706
:10052000909114070E941B3F1F5F1093E91303C0B3
:10053000F6DE1092E9130F900F900F90DF91CF919C
:100540001F91FF90EF9008958091D70B882311F0B1
:10055000E6DE01C0EBDE9091D70B81E08927809326
:10056000D70B08950F931F93CF93DF939091EC13C4
:1005700080919D1191112AC0882309F44FC00091E8
:10058000EA131091EB13C0911307D0911407B8012F
:10059000CE010E94B43E882321F0B801CE010E9412
:1005A000CC3EC4DE22EB32E842EC51E060E070E089
:1005B00080911307909114070E94233F9093EB13AF
:1005C0008093EA1381E08093EC1353C0882329F0D1
:1005D000DF91CF911F910F91B7CF8091D70B8823D7
:1005E000B9F36091EA137091EB1380911307909126
:1005F00014070E94CC3E22EB32E844E150E060E078
:1006000070E080911307909114070E94233F90930C
:10061000EB138093EA131092EC132BC0C0911302DA
:10062000D09114022297D0931402C09313021C1687
:100630001D0674F4BE01772787E00E940C4BCC2383
:1006400021F081E08093D70B14C01092D70B11C01A
:100650006091EA137091EB13809113079091140746
:100660000E94CC3E5CDE8FEF90E09093140280936A
:100670001302DF91CF911F910F9108950F931F9354
:10068000CF93DF930091E2131091E313C091E41331
:10069000D091E513C00FD11FD093E513C093E4139D
:1006A000BE01772787E00E940C4BCC2321F081E02C
:1006B0008093D70B02C01092D70B10161106ECF5E1
:1006C0008091E0139091E113C817D9070CF485C00D
:1006D0008091E613882371F01092E1131092E013D9
:1006E0008CEF9FEF9093E3138093E21381E080936C
:1006F000DF1373C068E770E080E090E00E9412476B
:10070000DC01CB010A96A11DB11D9093E1138093EA
:10071000E01368E270E080E090E00E941247DC01A4
:10072000CB010A96A11DB11D66277727681B790B9F
:100730007093E3136093E21350C0012B09F44DC092
:100740008091E0139091E1138C179D070CF445C044
:100750008091DF13882311F10091E7131091E813C2
:10076000C0911307D0911407B801CE010E94B43E86
:10077000882399F1B801CE010E94CC3ED0DD1092C1
:10078000E5131092E4131092DF1380919D118823DA
:1007900021F1DF91CF911F910F91E4CE69E670E0D6
:1007A00080E090E00E941247DC01CB018A569F4F07
:1007B000AF4FBF4F9093E1138093E01368E270E076
:1007C00080E090E00E941247DC01CB010A96A11D57
:1007D000B11D9093E3138093E213DF91CF911F91AA
:1007E0000F91089560E088E00C94A14A61E089E2ED
:1007F0000C94A14A0F931F93CF93DF9360E08BE299
:100800000E94A14A0091DD131091DE13C0911307DD
:10081000D0911407B801CE010E94B43E882341F064
:10082000B801CE01DF91CF911F910F910C94CC3E76
:10083000DF91CF911F910F91089580912F07882309
:1008400061F08091D90B882341F081E08093D60B31
:1008500080912E070E94F36721CD0895CF93DF93F7
:10086000CDB7DEB765970FB6F894DEBF0FBECDBF2C
:1008700081E08093DA0B8091DA13882371F182E3AF
:1008800090E09A83898388E290E09C838B838EE654
:1008900090E09E838D8384EF91E098878F831D8AFB
:1008A00084E08F938DB79EB745970FB6F8949EBF9F
:1008B0000FBE8DBFADB7BEB7119685E1FE01319673
:1008C00001900D928A95E1F784EE9AE00E94FD92E4
:1008D0000FB6F894DEBF0FBECDBF65960FB6F89485
:1008E000DEBF0FBECDBFDF91CF9108952FB7F89433
:1008F0006091F6137091F7138091F8139091F913AA
:100900002FBF08951F920F920FB60F9211242F93AD
:100910003F938F939F93AF93BF938091F6139091E2
:10092000F713A091F813B091F9133091F51323E068
:10093000230F2D3720F40196A11DB11D05C026E817
:10094000230F0296A11DB11D2093F5138093F6137A
:100950009093F713A093F813B093F9138091FD0EC1
:100960009091FE0EA091FF0EB091000F0196A11D77
:10097000B11D8093FD0E9093FE0EA093FF0EB093D9
:10098000000FBF91AF919F918F913F912F910F9049
:100990000FBE0F901F9018950F931F93CF93DF9367
:1009A0000091ED131091EE13C0911307D09114072D
:1009B000B801CE010E94B43E8823A1F0B801CE0157
:1009C0000E94CC3E2FE731E848EB5BE060E070E04E
:1009D00080911307909114070E941B3F9093EE1390
:1009E0008093ED136091E7137091E81380911307E2
:1009F000909114070E94B43E81114BC01092E613EF
:100A00008FEF90E09093E5138093E4138FDC68E719
:100A100070E080E090E00E941247DC01CB010A9672
:100A2000A11DB11D9093E1138093E01368E270E083
:100A300080E090E00E941247DC01CB010A96A11DE4
:100A4000B11D66277727681B790B7093E3136093BA
:100A5000E2132EE333E844E150E060E070E080917F
:100A60001307909114070E94233F9093E8138093FB
:100A7000E7132FE731E848EB5BE060E070E080913E
:100A80001307909114070E941B3F9093EE138093DD
:100A9000ED13DF91CF911F910F9108958F929F9247
:100AA000AF92BF92CF92EF92FF920F931F93CF938B
:100AB000DF9320913107223008F078C07B018C0150
:100AC00080901C0790901D07A0901E07B0901F07F4
:100AD00020E030E0A901C501B4010E942FC1181621
:100AE00054F520E030E0A901C501B4010E94D3C350
:100AF000181654F420E030E048E452E4C501B40193
:100B00000E942FC11816D4F420E030E048E452E4EB
:100B1000C501B4010E94D3C318169CF420E030E054
:100B200048EC52E4C501B4010E942FC187FF09C0FF
:100B3000CBE4D0E008C0C0E0D0E005C0C2E3D0E024
:100B400002C0C4E6D0E08FEF8C0D823068F42097AD
:100B500039F06C2FC8010E94954D6C2FC7010CC055
:100B6000C8015EDBC70116C08DEF8C0D8330F0F439
:100B7000209779F06C2FC801DF91CF911F910F91D1
:100B8000FF90EF90CF90BF90AF909F908F900C947C
:100B9000954DC801DF91CF911F910F91FF90EF907C
:100BA000CF90BF90AF909F908F903ACBDF91CF9135
:100BB0001F910F91FF90EF90CF90BF90AF909F90BB
:100BC0008F9008958F929F92AF92BF92CF92DF92B3
:100BD000EF92FF92C0901C07D0901D07E0901E0777
:100BE000F0901F0720E030E0A901C701B6010E9484
:100BF000D3C320E030E040E05FE387FD0BC0C701D6
:100C0000B6010E94D6C24B015C010E94A2C397FDAF
:100C100027C010C0C701B6010E94D5C20E94A2C35E
:100C200097FD1EC06536710581059105DCF424E64B
:100C3000822F14C0C501B4010E94A2C3653671059C
:100C4000810591057CF420E030E040E05FE3C701DE
:100C5000B6010E94D6C20E94A2C384E6861B03C0CE
:100C600084E601C080E0FF90EF90DF90CF90BF90CE
:100C7000AF909F908F9008950F931F93CF93DF9322
:100C800000910C0710910D07C0911307D091140724
:100C9000B801CE010E94B43E882321F0B801CE01F4
:100CA0000E94CC3E8091D80B882339F01092D80B4B
:100CB000DF91CF911F910F91B1CBDF91CF911F9118
:100CC0000F910895EC981092D90B68EC70E082E0D7
:100CD0000C94286780912A07811105C080912E0706
:100CE000811101C0EFCF8091D40B9091D50B0E9460
:100CF0003D9581E08093D90B64E670E00C94286701
:100D000060E089E20E94A14A26EF33E842E350E026
:100D100060E070E080911307909114070C941B3FE2
:100D20001F920F920FB60F9211240BB60F922F93B2
:100D30003F934F935F936F937F938F939F93AF9363
:100D4000BF93EF93FF938091DC138823B1F0489910
:100D500018C0E8982AEF33E84CE251E060E070E018
:100D600080911307909114070E941B3F8091DB1321
:100D7000882339F00E946B7B04C0489B02C0E8982E
:100D800039DDFF91EF91BF91AF919F918F917F914D
:100D90006F915F914F913F912F910F900BBE0F90EC
:100DA0000FBE0F901F90189561E08BE20E94A14A40
:100DB000E89A2AEF33E848E853E160E070E0809178
:100DC0001307909114070E941B3F9093DE138093AA
:100DD000DD13089561E08BE20E94A14AE89A2AEFB0
:100DE00033E848E853E160E070E0809113079091A8
:100DF00014070E941B3F9093DE138093DD13089528
:100E00001092DA0B409124075091250760E070E0C2
:100E10002EE234E880911307909114070C941B3F45
:100E20008091A8139091A91380689093A91380933F
:100E3000A81308958091A8139091A91380619093AD
:100E4000A9138093A8130895FC018281882371F06F
:100E50008381882359F013828091A8139091A9135C
:100E600024E082279093A9138093A8130895FC018E
:100E70008281882371F0838181110BC081E083839B
:100E80008091A8139091A91384609093A9138093E3
:100E9000A8130895FC018481882371F0858188233B
:100EA00059F015828091A8139091A91328E0822708
:100EB0009093A9138093A8130895FC01848188233B
:100EC00071F0858181110BC081E085838091A81329
:100ED0009091A91388609093A9138093A813089503
:100EE0008091A8139091A91320E282279093A913CF
:100EF0008093A81308958091A8139091A9138062FC
:100F00009093A9138093A8130895DC01ED91FC91AF
:100F10000680F781E02D60E070E0199477FF03C050
:100F20007195619571096F3F710519F014F06FEFBC
:100F300070E08091A8139091A9138C7B917090938D
:100F4000A9138093A8138091A8139091A9136F30CF
:100F5000710514F480641FC06733710514F4816453
:100F60001AC06F3571051CF48164906114C0673834
:100F700071051CF4816490630EC06F3A71051CF416
:100F80008164906408C0673D71051CF481649065BC
:100F900002C0816490669093A9138093A81308956A
:100FA00080E094E09093A9138093A8130895809112
:100FB000A8139091A91392609093A9138093A813FA
:100FC0000895089508950895089508950895089539
:100FD00008950895089580E0089508950895089566
:100FE0000895089508950895089508950895089519
:100FF0000895089508950895089508950895089509
:10100000089580E00895089508950895FC0164838B
:101010000895FC0162830895FC01138214821582F5
:1010200016821782108611860895089508950895EE
:10103000FC0183810895FC0165830895FC016483AC
:101040000895FC0160870895FC0166830895FC0102
:10105000128213821482158261E086E10E94D04AD6
:1010600061E086E10E94A14AE2E7F0E080818160D0
:1010700080831092A9131092A81308951F920F92C3
:101080000FB60F9211240BB60F920F931F932F934D
:101090003F934F935F936F937F938F939F93AF9300
:1010A000BF93EF93FF93809102148F5F809302149C
:1010B00090910114891708F42EC1109202148091A6
:1010C000001490E08730910508F025C1FC018827C5
:1010D000E155FE4F8F4F0C9494C460E086E10E946E
:1010E000A14A80E48093011481E048C061E086E178
:1010F0000E94A14A88E08093011436C060E086E136
:101100000E94A14A8091FE139091FF1397FF05C0A2
:1011100088E18093011484E031C088E08093011459
:1011200083E02CC061E086E10E94A14A88E18093BF
:1011300001148091FD138F5F8093FD13803150F077
:101140001092FD1385E01AC061E086E10E94A14A79
:1011500088E0EDCF8091FE139091FF13880F991FC7
:101160009093FF138093FE1382E008C060E086E155
:101170000E94A14A88E08093011486E080930014C5
:10118000CAC061E086E10E94A14A80EC809301140C
:101190008091A8139091A9139093FF138093FE134D
:1011A0008091A8139091A91391FF1CC08091FC130A
:1011B000882369F08091A8139091A91322E09227C7
:1011C0009093A9138093A8131092FC130BC081E095
:1011D0008093FC138093FB138093FA138EE59BE0BE
:1011E0000E941B678091FA138823C9F08091FB133A
:1011F0008823A9F07BDB00915E0B10915F0B20919F
:10120000600B3091610BDC01CB01801B910BA20BB9
:10121000B30B8D369042A105B10508F070C08091E6
:10122000A8139091A91392FF12C08091FC138823F8
:1012300039F01092A9131092A8131092FC1307C052
:1012400081E08093FC131092FB131092FA138091AB
:10125000A8139091A91384FF14C08091FC138823D4
:1012600069F08091A8139091A91320E182279093AF
:10127000A9138093A8131092FC1303C081E08093FC
:10128000FC138091A8139091A91387FF13C080913C
:10129000FC13882361F08091A8139091A9138058C2
:1012A0009093A9138093A8131092FC1303C081E0BC
:1012B0008093FC138091A8139091A91390FF14C000
:1012C0008091FC13882369F08091A8139091A91351
:1012D00021E092279093A9138093A8131092FC13F6
:1012E00003C081E08093FC138091A8139091A9130F
:1012F0009093FF138093FE13109200140CC0109271
:10130000FA138091A8139091A91380649093A91364
:101310008093A81384CFFF91EF91BF91AF919F91DC
:101320008F917F916F915F914F913F912F911F917D
:101330000F910F900BBE0F900FBE0F901F9018953E
:10134000FF920F931F93CF93DF938C01C62FF42E40
:10135000D22F6AED70E0DC011A968D919C911B975B
:1013600055D5F80182859385DC01ED91FC910190C2
:10137000F081E02D6C2F1995F80182859385DC01B1
:10138000ED91FC910190F081E02D6F2D1995F80100
:1013900082859385DC01ED91FC910190F081E02D37
:1013A0006D2F1995EC2FF0E0BF0166527F4F6F0D46
:1013B000711D6D0F711D6F777727F80182859385F9
:1013C000DF91CF911F910F91FF9020C520E040E069
:1013D000B7CF65E4FBCF68E4F9CFCF93DF93FC018F
:1013E0002381222321F0EC0161E4F0DF1B82DF91F5
:1013F000CF910895CF93DF93FC012381211105C084
:10140000EC0160E4E3DF81E08B83DF91CF9108950D
:1014100063E5DCCFFC012581222311F060E5D6CF06
:101420000895FC012481222311F06CE3CFCF0895AD
:10143000FC012085222331F02185222319F0118619
:101440006BE3C4CF0895FC012085222339F0218568
:10145000211104C021E021876AE3B8CF0895FC017F
:101460002681222331F02781222319F0178269E394
:10147000ADCF0895FC012681222339F02781211167
:1014800004C021E0278368E3A1CF089567E39ECFDE
:101490006AE49CCF69E49ACF66E398CF65E396CF80
:1014A0006EE494CF64E392CF63E390CF242F462F72
:1014B0006CE446CF462F20E067E442CF462F20E081
:1014C00066E43ECF262F64E43BCFCF92DF92FF92BB
:1014D0000F931F93CF93DF938C01F62E443F81E04F
:1014E000580738F0413187E2580728F040E157E2C9
:1014F00002C044EF51E0243F81E0380738F0E901B1
:101500002131374228F0C0E1D7E202C0C4EFD1E078
:10151000CA01845F914022E3C22ED12CB6010E9401
:101520006DC4462F2F2D62E4C8010ADFCE01845F0F
:101530009140B6010E946DC4462F2F2D63E4C8016F
:10154000DF91CF911F910F91FF90DF90CF90F8CE58
:10155000242F462F62E5F4CE242F462F61E5F0CEEE
:10156000262F40E06FE3ECCE262F40E06EE3E8CE7E
:10157000262F40E06DE3E4CE462F20E06FE4E0CE7E
:1015800008950895FC01828193818830910529F4A2
:1015900010922B0110922A010895099721F41092BC
:1015A0002901109228010895FC01178A168A6CED12
:1015B00075E082810C940341CF93DF93EC011F8A85
:1015C0001E8A8A810E947C408B8D882331F08A811B
:1015D0000E94F3409A8F898F1B8EDF91CF910895DF
:1015E000DF92EF92FF920F931F93CF93DF93EC0163
:1015F0008A81893010F40E946340DD8C6B8D7C8D74
:10160000098D1A8DEA80FB8089E08E1508F466C08A
:101610000F30110538F001369DE6190728F000E675
:101620001DE602C00FE010E06F30710538F0613642
:101630008DE6780728F060E67DE602C06FE070E096
:1016400080E090E00E9433C120E030E04AE754E4BB
:101650000E943AC320E030E04CE852E40E9494C17A
:101660009B01AC0160E070E08AEF94E40E943AC311
:101670000E94A2C3FF2425E12E9DF0012F9DF00DB5
:101680001124E452FF4EDD2071F023813481AB013F
:1016900077FF04C044275527461B570B88279927F7
:1016A000841B950B0AC025813681AB0177FF04C0EE
:1016B00044275527461B570BCA014FB7F89455E1ED
:1016C0005E9DF0015F9DF00D1124E452FF4E108BE2
:1016D0000787328B218B948B838B4FBF9D8D6B8DB6
:1016E0007C8D8A819923F9F08A3058F495E1899F9D
:1016F000F0011124E452FF4E0581168116950795DD
:1017000002C00EEE12E041E00E94AA4061E070E0EB
:1017100080E090E00E94174C8A810E94F3400817F5
:101720001907A0F31EC08A3058F495E1899FF00193
:101730001124E452FF4E038114811695079502C0CF
:101740000AEC18E040E00E94AA4061E070E080E00E
:1017500090E00E94174C8A810E94F3408017910705
:10176000A0F38A810E947C40B8018A81DF91CF91E9
:101770001F910F91FF90EF90DF900C940341CF9356
:10178000DF93EC018A81893010F40E94634048EEB7
:1017900053E05B874A8720ED37E03D872C878CED4F
:1017A00095E09F878E87598B488B3B8B2A8B9D8B2F
:1017B0008C8BDF91CF910895CF93DF93EC017F8BDA
:1017C0006E8B888599856817790769F48A810E94EC
:1017D0007C408B8D882329F18A810E94F3409A8F67
:1017E000898F1B8E1EC0CE010E94224EEA81EA30F4
:1017F000B0F49C01C39714F022E330E02E3C8FEF4D
:10180000380714F42EEC3FEF8FB7F89495E1E99F79
:10181000F0011124E452FF4E318720878FBF81E011
:101820008B8FDF91CF9108950F931F93CF93DF9309
:101830008C01FC01778B668B0E94224EEC01F80133
:101840008281938188309105D1F4D7FF06C060E092
:101850008AE00E94A14A61E005C061E08AE00E943E
:10186000A14A60E086E00E94A14AD7FF03C0D1955B
:10187000C195D109D0932B01C0932A011BC00997B0
:10188000C9F4D7FF06C060E08DE00E94A14A61E084
:1018900005C061E08DE00E94A14A60E08BE00E94FB
:1018A000A14AD7FF03C0D195C195D109D093290191
:1018B000C0932801DF91CF911F910F910895CF938D
:1018C000DF93EC018A81893010F40E9463402EEC92
:1018D0003FEF3B872A8782E390E09D878C871F86B6
:1018E0001E86398B288B9B8B8A8B1D8A1C8A6EEEF9
:1018F00072E08A810E94EF406AEC78E08A810E945F
:10190000EB408CED95E09A8F898F1B8EDF91CF9104
:101910000895CF93DF93EC0121E03FEF3B872A87C7
:101920008FEF90E09D878C871F861E86398B288BD2
:101930009B8B8A8B1D8A1C8A61E08AE00E94D04AB8
:1019400061E086E00E94D04A61E08DE20E94D04AC8
:1019500061E08DE00E94D04A61E08BE00E94D04AB5
:1019600061E08EE20E94D04A8A819B818830910595
:1019700029F410922B0110922A0106C0099721F434
:101980001092290110922801DF91CF9108950F93B1
:101990001F93CF93DF93EC010E9476840C8D1D8DF5
:1019A0002E8D3F8DDC01CB01801B910BA20BB30B65
:1019B000853F9140A105B10548F06E897F89CE0130
:1019C000DF91CF911F910F910C949B4EDF91CF919E
:1019D0001F910F9108950F931F93CF93DF938C0165
:1019E000FC01178A168AEC01699640E068E0CE0196
:1019F0000E94319E4FE766E0CE010E94319E40E09A
:101A00006CE0CE010E94319E4FE767E0CE010E945C
:101A1000319E0E947684F801648F758F868F978F30
:101A2000DF91CF911F910F9108956F927F928F92C6
:101A30009F92AF92BF92CF92DF92EF92FF920F935D
:101A40001F93CF93DF938091A2149091A314DC0194
:101A5000ED91FC910084F185E02D1995B12C1816BB
:101A600019060CF0D1C0AA24A3948091A2149091DD
:101A7000A314DC01ED91FC910084F185E02D199512
:101A8000892B09F4C1C0C091651481E08C0F80934B
:101A900065148091A2149091A314DC01ED91FC9146
:101AA0000284F385E02D1995EC2FF0E0EB5DFB4E01
:101AB00080838A30D1F6E0906514F12C1092B20E3A
:101AC0001092B10E1092AD0E1092AE0E1092AF0E9B
:101AD0001092B00E1092AC0E1092AB0E1092AA0E95
:101AE00085E2C82E84E1D82E00E010E0D0E0C0E00E
:101AF0000E151F050CF06CC0F60191916F019D3021
:101B000009F463C09C3789F19A3009F052C0D33090
:101B100009F059C0CC2309F456C06C2E712CC301B6
:101B200001970E94026F7093B20E6093B10E0E94F3
:101B300076846093A5147093A6148093A714909351
:101B4000A81480910314882309F45BC08090B10E1F
:101B50009090B20EB8016619770985E294E10E946F
:101B6000749F8816990679F54CC08C2F90E0FC0183
:101B7000E455F04F1082D13099F068F0D230B1F4D2
:101B80000E94026F6093AD0E7093AE0E8093AF0E05
:101B90009093B00E0BC00E94026F6093AA0E06C015
:101BA0000E94026F7093AC0E6093AB0EDF5FC0E0DB
:101BB0000CC00F3311053CF4EC2FF0E0E455F04F6E
:101BC0009083CF5F02C0109224140F5F1F4F90CFFD
:101BD0008091241481110EC08091A70E9091A80EBF
:101BE00001969093A80E8093A70E60E087E80E946C
:101BF0000BA002C0BB24B39410922514109265145C
:101C000034CFA0922414E1CF8B2DDF91CF911F917F
